:020000040000FA
:1000000000040020F509000089060000D509000061
:10001000930600009D060000A706000000000000F7
:10002000000000000000000000000000190A0000AD
:10003000B106000000000000BB060000C50600007D
:10004000CF060000D9060000E3060000ED06000020
:10005000F7060000010700000B070000150700006D
:100060001F07000029070000330700003D070000BC
:1000700047070000510700005B070000650700000C
:100080006F07000079070000830700008D0700005C
:1000900097070000A1070000AB070000B5070000AC
:1000A000BF070000C9070000D3070000DD070000FC
:1000B000E7070000F1070000FB070000050800004B
:1000C0000F08000019080000230800002D08000098
:1000D00037080000410800004B08000055080000E8
:1000E0005F08000069080000730800007D08000038
:1000F00087080000910800009B080000A508000088
:10010000AF0800001FB500F003F88DE80F001FBD19
:1001100000F066BC10B54FF010208069401C20B183
:100120004FF01021886900F089FA10BDFC4A01687F
:100130001160121D41681160F94A10328168116026
:10014000121DC168116070471FB56FF0010000906B
:1001500040100390029001904FF010208069040B32
:1001600060095DF8200004F01F02012191408843DE
:1001700061094DF821006846FFF7D8FF1FBD2DE942
:10018000F04105460C461646002706E02846216841
:1001900000F066FA2D1D241D7F1CB742F6D3BDE882
:1001A000F08170B504460B464FF6FF710A4618E021
:1001B000B3F5B47F02D340F2671500E01D46284630
:1001C0001B1A00BF34F8026B751829462A44451ED5
:1001D0002800F7D18DB205EB114195B205EB124223
:1001E00000BF002BE4D188B200EB114190B200EBCC
:1001F000124241EA024070BD92B00446C94903C9A7
:10020000CDE90001FF22402102A800F08FFB0FCCB6
:10021000CDE90423CDE9020102A9202208465508B0
:1002200001EB850304E080C81D461B1F45F8047CD4
:100230009842F8D100BF102102A8FFF7B2FF00904A
:10024000AA208DF80400FFF77FFFFFF763FF4FF050
:100250001021896901F18000102202A9FFF78FFFA8
:100260004FF01021886908226946FFF788FF00F0E7
:10027000C9F901464FF0805000694FF08052526931
:1002800050430A68904201D8102070470020FCE7D4
:100290000146D1E9000200EB82024FF08050006974
:1002A0004FF080535B69584382420DD84FF01020C5
:1002B000406904234A6803FB0202980600699B0612
:1002C0005B695843824201D9092070474FF01020E2
:1002D0004069401C08B90F20F7E70020F5E770B52A
:1002E00005460C462E460BE0304600F0A7F9B4F563
:1002F000806F01D2002401E0A4F5806406F58056E9
:10030000002CF1D170BD2DE9F0410446206806288B
:100310006BD2DFE800F040031A305122A668E5688E
:10032000676829463046FFF7DAFF2A4639463046E5
:10033000FFF725FFAA003946304600F0CBFA10B986
:100340000020BDE8F0810320FBE700F07BFB4FF4C9
:100350008050754908600020F3E7201DFFF789FFF2
:1003600005460DB12846ECE700F06CFB6E4960686D
:1003700008600020E5E76568E668A768B2003946CE
:10038000284600F0A7FA8046B8F1000F01D10020FE
:10039000D7E70E20D5E74FF010208069401C08B940
:1003A0000420CEE7201DFFF773FF05460DB1284658
:1003B000C7E72046FFF720FF4FF010208069401C60
:1003C00008B90420BDE7201DFFF753FF05460DB116
:1003D0002846B6E7606828B9FFF7B6FEFFF79AFE31
:1003E00000F010F92046FFF707FF0720A9E770B5D6
:1003F00005460C46182D04D12068FFF784FF2060C5
:1004000002E00120206000BF00BF70BD2DE9FF4762
:1004100005464FF010204669A86806EB80074FEAB2
:10042000163807F6FF704FEA10390020009001904F
:100430000290039000BF0BE041095DF8211000F02D
:100440001F0301229A40114342094DF82210401C1B
:100450004045F1D348460BE041095DF8211000F01A
:100460001F0301229A40114342094DF82210401CFB
:100470008028F1D34FF010208069040B60095DF8EB
:10048000200004F01F0201219140884361094DF8CA
:1004900021006846FFF74AFEBDE8FF872DE9F041DD
:1004A00004464FF010204569A6686768B2003946D7
:1004B000284600F00FFA10B10020BDE8F0810120BD
:1004C000FBE70446606808B1012000E00020074611
:1004D0002046FFF7E3FF28B1FFF736FEFFF71AFECD
:1004E00000F090F82046FFF791FFBFB14FF01020C9
:1004F000D0F81480A5686668B6F5002F0BD2B5F564
:10050000002F08D229464046FFF7E9FE2A46314629
:100510004046FFF734FEFFF7FDFD00BF00F072F824
:1005200000060040680A00000000002004466568DC
:100530003C480560006800F05FFA4FF010208069C9
:10054000401C002843D04FF01020806900F1800447
:100550004FF0102085692879AA2837D1102120462C
:10056000FFF71FFE07462868B8422BD14FF0102036
:10057000806900F18001202208464FEA520C01EB0D
:100580008C0601230EE053B150F8049BB446361F8D
:100590005CF804CCE14502D14FF0010C01E04FF0D2
:1005A000000C6346B042EED163B1206810B104285C
:1005B00006D102E02046FFF784FF2046FFF7B6FF92
:1005C00000BFFEE7FFF7A6FD00F01CF800BF4FF0EC
:1005D00010204069401C50B14FF010204069006865
:1005E000401C20B14FF01021486900F005FA4FF48B
:1005F00080500068401C08B900BFFEE74FF48050EF
:1006000000F0FAF9BFF34F8F0748006800F4E0608C
:1006100006490843001D04490860BFF34F8F00BF1F
:10062000FEE70000000000200CED00E00000FA05ED
:1006300000BF134800680028FBD0704700B5014692
:100640000220104A1060FFF7F3FF0E48001D016002
:10065000FFF7EEFF00200B4A1060FFF7E9FF00BD37
:1006600000B502460120074B1860FFF7E1FF11605B
:10067000FFF7DEFF0020034B1860FFF7D9FF00BD36
:1006800000E4014004E5014008208F490968095849
:10069000084710208C4909680958084714208A49DE
:1006A0000968095808471820874909680958084700
:1006B0003020854909680958084738208249096867
:1006C000095808473C2080490968095808474020D4
:1006D0007D4909680958084744207B490968095839
:1006E0000847482078490968095808474C20764946
:1006F000096809580847502073490968095808478C
:100700005420714909680958084758206E490968FA
:10071000095808475C206C49096809580847602057
:1007200069490968095808476420674909680958F0
:100730000847682064490968095808476C206249DD
:1007400009680958084770205F490968095808472F
:1007500074205D4909680958084778205A49096892
:10076000095808477C2058490968095808478020DB
:1007700055490968095808478420534909680958A8
:100780000847882050490968095808478C204E4975
:1007900009680958084790204B49096809580847D3
:1007A000942049490968095808479820464909682A
:1007B000095808479C204449096809580847A0205F
:1007C0004149096809580847A4203F490968095860
:1007D0000847A8203C49096809580847AC203A490D
:1007E000096809580847B020374909680958084777
:1007F000B4203549096809580847B82032490968C2
:1008000009580847BC203049096809580847C020E2
:100810002D49096809580847C4202B490968095817
:100820000847C8202849096809580847CC202649A4
:10083000096809580847D02023490968095808471A
:10084000D4202149096809580847D8201E49096859
:1008500009580847DC201C49096809580847E02066
:100860001949096809580847E420174909680958CF
:100870000847E8201449096809580847EC2012493C
:10088000096809580847F0200F49096809580847BE
:10089000F4200D49096809580847F8200A490968F1
:1008A00009580847FC2008490968095808475FF4B7
:1008B0008070054909680958084700000348044941
:1008C000024A034B7047000000000020780A000035
:1008D000780A000040EA010310B59B070FD1042AF3
:1008E0000DD310C808C9121F9C42F8D020BA19BAFB
:1008F000884201D9012010BD4FF0FF3010BD1AB160
:10090000D30703D0521C07E0002010BD10F8013BB4
:1009100011F8014B1B1B07D110F8013B11F8014BDB
:100920001B1B01D1921EF1D1184610BD02F0FF032E
:1009300043EA032242EA024200F005B870477047DA
:1009400070474FF000020429C0F0128010F0030C31
:1009500000F01B80CCF1040CBCF1020F18BF00F8B2
:10096000012BA8BF20F8022BA1EB0C0100F00DB861
:100970005FEAC17C24BF00F8012B00F8012B48BFBF
:1009800000F8012B70474FF0000200B51346944663
:100990009646203922BFA0E80C50A0E80C50B1F1D7
:1009A0002001BFF4F7AF090728BFA0E80C5048BFEB
:1009B0000CC05DF804EB890028BF40F8042B08BF89
:1009C000704748BF20F8022B11F0804F18BF00F885
:1009D000012B7047014B1B68DB68184700000020A3
:1009E00009480A497047FFF7FBFFFFF78BFB00BD83
:1009F00020BFFDE7064B1847064A1060016881F3E7
:100A00000888406800470000780A0000780A000063
:100A10003B050000000000201EF0040F0CBFEFF3A8
:100A20000881EFF30981886902380078182803D11A
:100A300000E00000074A1047074A12682C3212688B
:100A40001047000000B5054B1B68054A9B589847A6
:100A500000BD0000EF03000000000020640A000059
:100A600004000000001000000000000000FFFFFF75
:040A70000090D0031F
:10100000E010002045AB0100452F0000B3AA01000D
:10101000452F0000452F0000452F00000000000074
:10102000000000000000000000000000A9AB01006B
:10103000452F000000000000452F0000452F000054
:1010400011AC010017AC0100452F0000452F000036
:10105000452F0000452F0000452F0000452F0000C0
:101060001DAC0100452F0000452F000023AC0100FE
:10107000452F000029AC01002FAC010035AC010068
:10108000452F0000452F0000452F0000452F000090
:10109000452F0000452F0000452F0000452F000080
:1010A0003BAC010041AC0100452F0000452F000082
:1010B000452F0000452F0000452F0000452F000060
:1010C000452F0000452F0000452F0000452F000050
:1010D000452F0000452F0000452F0000452F000040
:1010E000452F0000452F0000452F0000452F000030
:1010F000452F0000452F0000452F0000452F000020
:10110000452F0000452F000000F002F819F0F7FC11
:101110000AA090E8000C82448344AAF10107DA4552
:1011200001D119F0ECFCAFF2090EBAE80F0013F090
:10113000010F18BFFB1A43F0010318472C9C010054
:101140004C9C01000A4410F8014B14F00F0508BF35
:1011500010F8015B240908BF10F8014B6D1E05D083
:1011600010F8013B6D1E01F8013BF9D1641E03D05C
:10117000641E01F8015BFBD19142E4D3704700008B
:101180000023002400250026103A28BF78C1FBD890
:10119000520728BF30C148BF0B6070471FB500F031
:1011A00031F88DE80F001FBD8269034981614FF05E
:1011B0000100104470470000BD11000001B41EB4CE
:1011C00000B510F002FA01B40198864601BC01B0E6
:1011D0001EBD0000F0B44046494652465B460FB47F
:1011E00002A0013001B50648004700BF01BC864699
:1011F0000FBC8046894692469B46F0BC7047000073
:101200000911000019F078BC70B5F84C05460820AB
:101210002070A01C00F01BFA5920A080294620460F
:10122000BDE8704007F045B810B507F04CF8EF493D
:101230000020891E087010BD70B5EC4D0C46AD1E27
:101240000126297871B36038532871D2DFE800F0A5
:101250002F383D43484E53575D6270707070707008
:10126000676C71787C7F858B9095999DA1A8ADB3B3
:10127000BBC2C9F2F8FFEEEDECEBEA707070707073
:10128000E9E8E7E6E5E4E3E2E1E0707070707070D1
:10129000DFDEDDDCDBDAD9D8D7D6D5D4D3707070F9
:1012A000D2D1D000602802D043F201009AE1D4E903
:1012B000000107F05BF92060002800D12E7070BD9E
:1012C000D4E9000107F0DCF98CE12088616880B284
:1012D00007F01FF986E1D4E9000107F062FA81E125
:1012E000D4E90112207807F075FA7BE194E8070051
:1012F00007F091FA76E1206807F0B0FA72E12088F1
:10130000616880B207F0CEFA6CE1D4E9000107F021
:10131000E6FA67E1D4E9000107F0FAFA62E1207821
:10132000616802F06DFE5DE1206802F0BFFE59E1E8
:101330005AE1237B2179A268206802F0CDFE51E1B9
:10134000206802F059FF4DE102F033FC4AE12088A9
:10135000616880B203F07DF844E12088217980B291
:1013600003F0EFF83EE1207840B203F0FAF839E1FB
:10137000208880B200F07FFA34E1206800F08DFA16
:1013800030E1206800F015FA2CE1206800F041FA05
:1013900028E1208982B2D4E9000100F09EFA21E11F
:1013A000D4E9000100F0E8FA1CE12088616880B20D
:1013B00004F06AFA16E1D4E902232088217980B288
:1013C00004F043FB0EE12088217980B2A26804F08A
:1013D000E8FC07E1D4E90112208880B204F05BFD4B
:1013E00000E1211D20880EC980B204F0B9FDF9E0AA
:1013F000F2E0ECE0E6E0DEE0D9E0D1E0C7E0C0E01A
:10140000B6E0AFE0A6E09DE095E08DE084E07DE011
:101410006FE068E05FE055E04DE071E045E03EE000
:1014200037E02EE027E023E01DE019E014E00EE0B5
:1014300006E0FFE72088616880B204F0CCFDD1E0CF
:101440002088227A217980B203F098F8CAE02088B7
:1014500080B203F096F8C5E0206803F097F8C1E089
:1014600002F088FBBEE094E8070003F0F7F8B9E06B
:1014700002F069FBB6E02088616880B203F0A1F950
:10148000B0E0A088A26881B2208880B200F06BFF33
:10149000A8E02088616880B200F0A8FFA2E0208860
:1014A000616880B200F0B0FF9CE02088616880B283
:1014B00000F0B8FF96E0D4E90112208880B200F075
:1014C000C6FF8FE0208982B2A08881B2208880B2D6
:1014D00000F0C2FF86E02089616882B2208880B275
:1014E00000F0DBFF7EE02088616880B200F0E6FF5C
:1014F00078E0A08881B2208880B201F040F871E0E5
:101500002088616880B201F047F86BE0D4E90112ED
:10151000207806F0ADF865E0A088A26881B2208846
:1015200080B206F0B5F85DE0211D20880EC980B2BA
:1015300006F0AFF856E0D4E90112208880B206F038
:10154000C3F84FE0A088A26881B2208880B206F07C
:10155000D0F847E0A088A26881B2208880B206F067
:1015600017F93FE02088616880B206F06CF939E035
:10157000208982B2A08881B2208880B206F06DF9FD
:1015800030E02088616880B206F08DF92AE0208979
:10159000E36882B22088616880B206F0ECF921E04D
:1015A000211D20880EC980B206F0C2FA1AE0206818
:1015B00006F06CFB16E0D4E90112208880B206F038
:1015C00076FB0FE0208880B201F030FC0AE0208832
:1015D00080B201F04AFC05E0D4E90112208880B213
:1015E00001F054FC206070BD266070BD0A00002030
:1015F00010B504460021012000F034F80021182025
:1016000000F030F800210B2000F02CF80221192006
:1016100000F028F802210D2000F024F802210E200D
:1016200000F020F802210F2000F01CF80221C81F52
:1016300000F018F80321162000F014F803211520FB
:1016400000F010F82046FFF7DFFD002010BD7921E3
:1016500001807047FFF7E8BD0A487047FFF7ECBD0F
:10166000704770474907090E002806DA00F00F009E
:1016700000F1E02080F8141D704700F1E02080F8B0
:101680000014704703F90043FD4800210160818088
:1016900070472DE9FF418046FA480D4692B01C463E
:1016A0001946834206D3F848814207D3F7480068B9
:1016B000814203D2102016B0BDE8F081012001F074
:1016C0007AFD0028F7D101268DF842604FF4C05012
:1016D000ADF84000002210A9304605F088FC002833
:1016E000E9D18DF842604FF42850ADF84000002752
:1016F0001C216846099719F0A2F99DF82400ADF85D
:10170000345020F00F00401C20F0F00010308DF815
:1017100024009DF82500ADF8367020F0FF008DF80C
:1017200025009DF8260007AA20F00600801C40F046
:1017300001008DF826009DF800000BA940F0020082
:101740008DF800001F20ADF8380009A80C9010A8F3
:101750000B90CDF83C80684605F02FFA0028AAD1FE
:10176000C74DBDF81C0007AA28808DF8426042F6DC
:101770000120ADF840009DF826000BA920F00600DE
:10178000801C20F001008DF826000220ADF8340006
:10179000ADF8380014A80F90684605F00EFA00283E
:1017A00089D1BDF81C006880291D204600F010F981
:1017B00081E73EB504460820ADF80000B1488442F8
:1017C00006D3B148844205D3B0480068844201D2B0
:1017D00010203EBD2146012001F0EDFC0028F8D18B
:1017E0002088ADF804006088ADF80600A088ADF848
:1017F0000800E088ADF80A00A14801AB6A4680887D
:10180000002105F02FFEBDF800100829E1D00320CB
:101810003EBD1FB50446002002900820ADF8080028
:101820009848CDF80CD0844206D39748844206D31A
:1018300096480068844202D2102004B010BD90483F
:1018400002AA81884FF6FF7005F0A2FF0028F4D1AC
:10185000BDF80810082901D00320EEE7BDF80010FC
:101860002180BDF802106180BDF80410A180BDF890
:101870000610E180E1E701B582B00220ADF800007A
:101880007F4802AB6A464088002105F0EBFDBDF8B9
:101890000010022900D003200EBD1CB500210091CC
:1018A0000221ADF800100190B0F5000F06D3B0F1A1
:1018B000805F05D375490968884201D210201CBD9C
:1018C0006F486A4641884FF6FF7005F061FFBDF82A
:1018D00000100229F3D003201CBD2DE9FF4117465B
:1018E000684A0E460546914206D368486649006834
:1018F0008E4204D3864202D2102004B0DCE61F2FB1
:1019000001D90C20F9E75E4C954227D38D4201D3D3
:10191000854223D3208803A905F062FD0028ECD17D
:1019200028788DF80D00208803A905F03AFD0028DD
:10193000E3D100909DF800009DF80D1040F00200EA
:101940008DF80000090703D040F008008DF8000072
:101950002088694605F0BFFC0028CED1ADF80470A0
:101960002088334601AA002105F07CFDBDF8041053
:10197000B942C2D00320C0E77CB50C4600210091DB
:10198000019122884149ADF8002001904FF40003F5
:1019900009685D0128B1984209D3A84201D3884261
:1019A00005D39C4203D3AC4203D38C4201D2102016
:1019B0007CBD00B152B132486A4601884FF6FF70D3
:1019C00005F0E6FEBDF8001021807CBD0C207CBD3A
:1019D00030B593B0044600200D460090142101A8B4
:1019E00019F02DF81C2108A819F029F89DF800001D
:1019F000CDF808D020F00F00401C20F0F00010308F
:101A00008DF800009DF8010006AA20F0FF008DF877
:101A100001009DF8200001A940F002008DF820008F
:101A200001208DF8460042F60420ADF8440011A8CC
:101A300001902088ADF83C006088ADF83E00A08899
:101A4000ADF84000E088ADF842009DF8020020F0BB
:101A50000600801C20F001008DF802000820ADF87F
:101A60000C00ADF810000FA8059008A805F0A5F827
:101A7000002803D1BDF818002880002013B030BD25
:101A80001000002000B00100000000201C00002019
:101A900070B50D46007804991446042804D0052832
:101AA00033D019F000F870BDA88B0E2200EB400077
:101AB00002EB4000188033200880002CF3D0A88B64
:101AC000A081002613E0A87F012814D006EBC600F1
:101AD00005EB400106EB460204EB4202088CD08184
:101AE0001020223110320DF0BDFD761CB6B2A08957
:101AF000B042E8D870BD05EB860106EB460204EB68
:101B00004202088CD0810220EBE7A88B102200EB68
:101B1000C00002EB4000188034200880A87F012814
:101B200009D0022807D018F0BEFF002CE2D0A88B05
:101B3000A081002613E0A073F7E7A87F012812D048
:101B400006EBC60005EB400104EB40000A8C028264
:101B500010221230223118F0D9FE761CB6B2A089BC
:101B6000B042EAD870BD05EB860106EBC602088CD0
:101B700004EB420222311082022012320DF072FD7B
:101B8000EBE72DE9F04105780E20DDF818C001F1F2
:101B9000200402F10E074FF00008022D07D0032D9C
:101BA0002ED0062D6BD018F07EFFBDE8F081CD8BD6
:101BB00005EB850600EB460018803120ACF80000EC
:101BC000002AF2D0087F9581801FC6B214E06168B8
:101BD0002088388031F8020BF88031F8020B388108
:101BE000BA1C30460DF03EFD06B118B187F80480EE
:101BF000A7F8028008340A376D1EADB2E7D2D4E7E9
:101C0000CD8B05EB850600EB460018803220ACF842
:101C10000000002AC9D0087F9581401FC6B22AE083
:101C20006168228811F8010BFA803A79430860F361
:101C3000000263F34102830863F38202C30863F383
:101C4000C302030963F30412430963F345128309D2
:101C500063F386123A71C009787131F8020B38814A
:101C60003A4630460DF0FEFC18B187F80280A7F81E
:101C7000008008340A376D1EADB2D1D295E7087FD7
:101C8000CD8B801E86B206F10800684310301880A4
:101C90003520ACF80000002A87D0958102F11007AA
:101CA000D68107EBC5080BE020883880C7F8048090
:101CB00032464046616818F029FE0834B0440837BF
:101CC0006D1EADB2F0D270E72DE9F0471D46089EBB
:101CD0000C4681462AB1607E00F58070D080E08B92
:101CE000108199F800000E274FF000084FF0100AFD
:101CF0000C2874D2DFE800F0A10616232C354454DA
:101D00006A747474207F9146082803D0032801D098
:101D100018F0C9FE2F8030200CE000BFA9F80C801D
:101D2000BDE8F087207F9146042801D018F0BBFE63
:101D30002F8031203080B9F1000FEFD1F0E7207F04
:101D40009146042801D018F0AEFE2F803220F1E732
:101D5000207F9146022801D018F0A5FE2F80332065
:101D6000E8E7207F1746022801D018F09CFE3420B7
:101D7000A5F800A03080002FD2D0A7F80C80CFE7C4
:101D8000207F1746042801D018F08DFE3520A5F8D5
:101D900000A03080002FC3D04046A7F80C8013E08D
:101DA000207F1746052803D0062801D018F07BFEB7
:101DB0001220288036203080002FB1D0E08BB881EF
:101DC000A7F81080B9F80200F881A9E7207F9146B2
:101DD000072801D018F067FE2F803720AAE72CE0F3
:101DE0004FF0140018804FF038001700308097D063
:101DF000E08BB881A7F8128099F80000092806D076
:101E00000A280BD00B2810D018F04DFE88E7207F51
:101E10000C2801D018F047FE01200CE0207F0D288F
:101E200001D018F040FE042005E0207F0E2801D0EC
:101E300018F039FE0520B87372E718F034FE6FE72A
:101E400070B50C46054601F01EF920B10078222835
:101E500004D2082070BD43F2020070BD052128465F
:101E60000BF065FD206008B1002070BD032070BD3F
:101E7000FFB585B007461720ADF80800089814464E
:101E80000D46032628B908A93846FFF7D9FF0028D0
:101E90003AD14DB100220321384600F04BFFA8B3E0
:101EA0000898007890BB06E02078092822D00F28F7
:101EB0002DD018F0F8FD002000900246019003ABF1
:101EC000BDF80810384600F02BFC08B118F0EBFD07
:101ED000089802A9801DC4E901072046039A07F06B
:101EE000FAFA40B3072824D2DFE800F01A182323B7
:101EF000211C1E00072600223146384600F01AFF3A
:101F00000028D8D143F2040009B0F0BD06E0002259
:101F10000321384600F00EFF0028CCD11120F3E752
:101F20000020F1E70820EFE743F20300ECE7072089
:101F3000EAE70320E8E703980090BDF808300422A0
:101F40003146384600F0B8FD0028DDD1002DDBD049
:101F500008990D70D8E710B588B01C46AAB10423C3
:101F60008DF800301388ADF80C305288ADF80E2093
:101F70008A788DF812200988ADF8101000236A467F
:101F80002146FFF775FF08B010BD1020FBE72DE9D3
:101F9000F041074600780C4612283FD2DFE800F0F7
:101FA0003E383816113B09090909090909090909C7
:101FB00009090CB918F077FD607840F008006070EE
:101FC0002EE0002CF8D118F06EFDF5E7B888052159
:101FD00086B230460BF0ABFC05460CB118F063FD41
:101FE0000DB918F060FD3146A81D07F06DFA06F036
:101FF000A9F8040007D0607840F00800607066809F
:1020000006F07EF80DE01321304602F09AFA19E04E
:1020100018F049FD04E018F046FD01E018F043FD1A
:1020200084B1607800070DD52078582220F00F0089
:10203000C01C20F0F00090302070394604F11800E8
:1020400018F0A9FC0020B0E5002100F8061B07F0FD
:1020500038BA0A460146901D07F03CBA70B50546ED
:1020600005210BF064FC040001D118F01CFD294689
:10207000A01DBDE8704007F027BA2DE9FE4F4FF0D4
:102080000009ADF80890ADF8049047880C46054665
:102090009346052138460BF04AFC060001D118F0A2
:1020A00002FD24B1A780A4F80690A4F80890297E28
:1020B00004F112003827C91E4FF001084FF0360A0C
:1020C00000900F2973D2DFE801F0EEED726308B2E1
:1020D0006C73852DBBCFEF9A9A003078012801D020
:1020E00018F0E1FCA88B0E2101EBC001ADF8041043
:1020F0003021ADF80810002C13D0A08100200DE095
:1021000004EBC00132790A747288CA8105EB80023F
:10211000401CD38B4B82128C8A8280B2A18981426F
:10212000EED8F1E03078012801D018F0BCFCE88B43
:102130000E2101EBC001ADF804103021ADF80810FC
:10214000297F091FC9B20091002CEAD0A081002785
:102150001AE000BF05EBC70A04EBC70808F10E023E
:10216000DAF8241000980DF07DFA18B188F8109074
:10217000A8F80E90BAF82010A8F81210BAF8221099
:102180007F1CA8F81410BFB2A089B842E2D8BBE007
:1021900002A8009001AB224629463046FFF778FCA2
:1021A000B2E03078072808D018F07DFC05E0A9E0FF
:1021B0003078072801D018F076FCE88BADF808A03D
:1021C0001230ADF80400002C39D0A98BA1817188A0
:1021D000E18124E03078082801D018F064FCA88B55
:1021E00000F10E01ADF804103721ADF80810002CF5
:1021F00025D0A081AA8B04F10E00296A4EE0E88B5D
:10220000123080B23921ADF80400ADF80810ECB3FB
:10221000A98BA181287E102807D00221A173E98B08
:102220002182EA8B296A009838E00121F6E702A8AA
:10223000009001AB224629463046FFF7A2FC63E03E
:102240003078092801D018F02EFC1420ADF80400D5
:10225000ADF8087024B3A98BA181A4F81290A4F85A
:10226000109084F80E804FE030780A2801D018F0E2
:102270001AFC288CADF808701430ADF804007CB15D
:102280000421A173A98BA181E98B00E037E02182B1
:10229000298C61822A8C04F11400696A18F036FBDB
:1022A00032E001E014E01CE030780B2801D018F097
:1022B000FAFB1420ADF80400ADF8087024B3052132
:1022C000A173A4F80C90A4F81090A4F812901BE04D
:1022D00002A8009001AB224629463046FFF7F4FCE5
:1022E00012E00D203A21ADF80400ADF8081034B129
:1022F000A4F80680A4F8089084F80C9004E0ABF8E9
:10230000000015E018F0CFFBBDF80400ABF80000AA
:1023100074B1BDF808002080BDF804006080287EFC
:10232000032805D0102803D0112801D086F800908A
:102330000020BDE8FE8F2DE9F84356880F46804601
:102340001546052130460BF0F2FA040001D118F0D1
:10235000AAFBA41D33462A4639464046009407F09E
:1023600037FABDE8F8832DE9F0438DB00D461446E9
:10237000814607A9FFF764FD002814D14FF6FF76C8
:1023800001274FF420588CB103208DF80000102055
:10239000ADF8140008A802460690204605A90DF0E5
:1023A00080F978B107200DB0BDE8F0830820ADF8C2
:1023B0000C508DF812708DF80000ADF80E60ADF87D
:1023C00010800CE00798A1780171218841808DF878
:1023D0001270ADF80C50ADF81080ADF80E606A4682
:1023E00001214846079BFFF743FDDCE708B50122C2
:1023F0008DF8022042F60202ADF800200A460223C0
:102400006946FFF7A8FD08BD08B501228DF8022036
:1024100042F60302ADF800200A4603236946FFF79F
:102420009AFD08BD00B587B079B102228DF8002071
:102430000A88ADF80C204988ADF80E1000236A46D2
:102440000421FFF715FD07B000BD1020FBE709B11F
:10245000062380E50720704770B588B00D46144606
:10246000064607A9FFF7ECFC00280ED17CB1062038
:10247000ADF80C508DF80000ADF80E40079B6A4691
:1024800007215C803046FFF7F3FC08B070BD0520E3
:102490008DF80000ADF80C50F0E700B587B059B1E9
:1024A00007238DF80030ADF80C20049100236A4614
:1024B0000821FFF7DDFCC6E71020C4E770B5002453
:1024C00088B0172391B10A78062A20D2DFE802F0FB
:1024D0001F04041503171523DB1E9DB2CB880BB117
:1024E0008E681EB1AB4203D90C20CEE71020CCE79A
:1024F000042A04D08B8853B901E00620C5E7012ADD
:1025000013D0022A05D0042A1CD0052A2AD007207D
:10251000BBE709228DF800204A88ADF80C20CA8854
:10252000ADF80E208968049123E00C228DF800207C
:102530004A88ADF80C20CA88ADF80E2089680924B5
:10254000049116E00D228DF800204A88ADF80C2089
:102550008A88ADF80E20CA88ADF8102089680A2450
:10256000059106E00E228DF8002049788DF80C10B8
:102570000B2400236A462146FFF77AFC85E700B565
:1025800087B00F228DF80020ADF80C1000236A46AA
:102590001946FFF76DFC56E700B587B071B102220E
:1025A0008DF800200A88ADF80C204988ADF80E108F
:1025B00000236A460521FFF75BFC44E7102042E751
:1025C0004FF0E0224FF400410020C2F88011224970
:1025D0000870224990020860704730B51E4D0446CD
:1025E0002878A04218BF002C03D0002818BF18F08C
:1025F0005AFA2878A04208BF30BD2C701849174AF3
:102600000020F4B1174DDFF860C0131F012C04D077
:10261000022C0CD018F047FA30BD08600220086088
:10262000CCF800504FF040701060186030BD08606A
:1026300003200860CCF800504FF4000010601860D0
:1026400030BD086008604FF06070106030BD00B5AC
:1026500018F029FA00BD00001600002008F501401E
:1026600000F50040D002002014F500402DE9F047AD
:102670008246DDE9087807F10B00C5B29946164697
:102680000C46504600F035FCA84207D2072E02D077
:102690001120BDE8F08743F20400FAE7607B1E28B2
:1026A00001D318F000FAA07800061BD4A8F10401A9
:1026B000C81E0022027028F8047C28F8029C5046AC
:1026C0000BF0E9FA5FEA000801D118F0ECF93F1DC0
:1026D000B9B2404600F088FC08B918F0E4F9504659
:1026E00008F0C4FF207B617B0844491CC0B26173C1
:1026F0001E2801D31E38C0B200EB40002044072E34
:102700008673C17B21F00F01C173057404D0608909
:10271000401B60810020BCE72089401B2081F9E735
:102720002DE9F04385B01D46DDE90C871646894644
:102730000BF0B1FA040001D118F0B5F909F1040069
:1027400082B26946204600F04DFCF8B1BDF80800A1
:10275000042801D218F0A7F91EB1BDF80800001F27
:10276000308015B10198C01D2860BDF8100008B177
:1027700018F099F90020B8F1000F01D0A8F8000076
:1027800007B13860002005B0BDE8F08343F20400D3
:10279000F9E72DE9F04F0F46054687B016465088F9
:1027A00003210BF0C4F8040001D118F07CF94FF0BC
:1027B00000098DF80890A078400601D118F073F94F
:1027C000042F53D3297841F30000401C06D16278CE
:1027D0006B789A424AD12278120747D04FF0010B0A
:1027E0004FF00208142939DA4FF6FF7A012933D065
:1027F000122902D0132931D11CE00C2F2ED1A1783F
:1028000001F07F01012929D0207820F00F00401C21
:102810002070687860708DF808B0A888ADF80C005A
:10282000E888ADF80E002889ADF810006889ADF889
:10283000120016E0062F11D1207820F00F00207032
:10284000718801200FF0E3F88DF80880ADF80CA036
:10285000A888ADF80E0004E0062F0AD09DF80810F5
:10286000B9B17088324602A901F054FA07B0BDE848
:10287000F08F207820F00F002070718801200FF079
:10288000C6F88DF80880A888ADF80C00ADF80EA049
:10289000E7E70028EAD0768827464C46CDF8009036
:1028A00005AB002206213046CDF80490FFF738FF33
:1028B00008B118F0F8F8059805231A4680F800B01A
:1028C00069784170A0F8028084800621CDE900106B
:1028D00039463046FFF7CAFE0028C7D018F0E3F8A3
:1028E000C4E72DE9FF470F468146014615463846A5
:1028F000FFF721FDC0B2082851D10026ADF80860CD
:10290000688803210BF013F8040001D118F0CBF80C
:1029100001230021207B627B0EE000BF00EB400C16
:10292000A4449CF80EC09C4501D1491CC9B2401C6E
:10293000C0B21E2800D10020521ED2B2EED211B970
:102940001720ADF8080000960196688803AB0022B6
:10295000BDF80810FFF7E4FE08B118F0A4F80095E0
:1029600002AA49463846039B04F001F9C0B2052883
:102970001CD2DFE800F0031B14161400BDF8080099
:1029800000280CD003990423CDE9000168880122B6
:102990002146FFF76BFE002801D018F084F8BDE84F
:1029A000FF87687840F010006870F8E718F07BF84F
:1029B000F5E70020F949024621F81020401C0828BC
:1029C000FAD37047817821F0FF018170017821F0FE
:1029D0000F010170012141700021416001734173B9
:1029E000704770B50D4603210AF0A1FF040001D124
:1029F00018F059F8A078012D65F30600A07002D0F8
:102A0000022D02D003E0EE2000E066202081CC20E1
:102A1000608170BD7047014601200EF0F8BF3EB5E1
:102A20008DB2032128460AF082FF040001D118F07C
:102A30003AF82078002220F00F00207002208DF854
:102A400000004FF6FF70ADF80400ADF806006946CF
:102A5000284601F05FF93EBD2DE9F04105460C46E0
:102A600000270078012190463E46B1EB101F01D0AF
:102A700018F019F8287E03280AD018F014F800BFBF
:102A8000A8F800600CB1278066800020BDE8F081C6
:102A9000EA8B702702F10A0086B254B16888A080E0
:102AA000A88B2081E28004F10A00296A17F02EFF2A
:102AB000E6E7A8F80060E8E72DE9FC410F461C4670
:102AC000164680460321089D0AF031FF010008D018
:102AD00033463A464046CDE90045FFF7C7FDBDE81D
:102AE000FC8143F20200FAE72DE9F04102468068DA
:102AF000938930F8031F1B1F45889942C6D1042DC6
:102B00001FD0052D29D0062D1FD0402DBED3061D68
:102B10000F461446284600F0F2F90828B6D020786F
:102B200020F00F00401C20F0F00010302070032037
:102B30002076A583E7832662607840F00800607005
:102B4000A4E7BDE8F041001DCBE6031D5088BDE8B9
:102B5000F0410A46194602F0B2BBBDE8F041001D43
:102B600017E6FEB50D46064603210AF0E0FE040016
:102B700010D0207800F00F00012809D0002000902C
:102B80000246019002AB0C213046FFF7C9FD20B18F
:102B90001120FEBD43F20200FEBD02981221052362
:102BA000017061781A46891C41700821418029888A
:102BB00081806988C180A9880181E98841810C21CF
:102BC000CDE9001021463046FFF750FD08B117F05F
:102BD0006AFFF0230022314601200EF07AFE2078B1
:102BE00020F00F00401C20706078801C6070002076
:102BF000FEBDFEB50D46064603210AF098FE040010
:102C000006D0207800F00F00012804D00820FEBD77
:102C100043F20200FEBD002000900246019002AB8C
:102C200006213046FFF77CFD08B11120FEBD029859
:102C30001321052301706178417002214180858054
:102C40000621CDE900101A4621463046FFF70EFD59
:102C500008B117F028FF207820F00F002070002026
:102C6000FEBD2DE9F0470D46824603210AF05FFEC6
:102C700004004FF0000801D117F015FF607BA84257
:102C80002CD217F010FF29E0207B00EB40010E1939
:102C9000401CC0B2B77B96F8109020731E2801D15B
:102CA00000202073607B401E6073F07BC00704D05F
:102CB0005046042F17D017F0F6FEF17B11F00E0FDF
:102CC00006D0C1F34201504604290FD017F0EBFEA5
:102CD000072F0ED0618901EB090060816D1EEDB2F6
:102CE000D2D24046D5E402F07FFBE6E702F044FB97
:102CF000EEE708F10100218900F0FF0801EB09006F
:102D00002081EBE710B503210AF011FE040001D188
:102D100017F0C9FE207B617B0844C0B220731E28D7
:102D200001D31E38207300206073A07840F080002B
:102D3000A07010BD2DE9F0410D461746064603214F
:102D40000AF0F5FD040003D03DB11FB1062002E0FA
:102D500001209BE60820A84201D817F0A4FE2A46CD
:102D60002146304600F0C5F82221B0FBF1F0C6B292
:102D700037B32EBB207B617B1EE000BF00EB40021F
:102D80002244937B072B03D0D37B13F00E0F07D085
:102D9000401CC0B21E280CD00CE0000050070020E0
:102DA00000EB40002044C07B65F34300D07339B989
:102DB00004E00020491EC9B20029DFD117F073FEDC
:102DC000304663E62DE9F0410D4603210AF0AFFDE0
:102DD000040001D117F067FE681E052801D317F023
:102DE00062FE1E23227B607B002111E002EB420683
:102DF0002644B77BAF4206D1F37B491C23F0010385
:102E0000F373C9B21346521CD2B21E2A00D100225B
:102E1000401EC0B2EAD21E2B06D203EB4300204470
:102E2000C27B42F00102C27308462FE610B5044689
:102E3000402801D2072010BD00F061F8082802D018
:102E40004FF4445010BD0021334802E0491C0829CA
:102E500003D230F81120002AF8D1082903D020F835
:102E60001140002010BD042010BD10B5402801D233
:102E7000072010BD00F043F8082805D0264A00219D
:102E800022F81010084610BD052010BDFEB51546ED
:102E90000C00064605D025B16188402903D20720E1
:102EA000FEBD1020FEBD208808B1172801D90C20D6
:102EB000FEBD084600F023F8082818D00020009036
:102EC00001900246218802AB3046FFF729FC00281A
:102ED000EED122882946029817F018FD029800903A
:102EE0002388628807213046FFF7E6FDFEBD0520F6
:102EF000FEBD072A01D048897047088970470146FE
:102F00000020054A02E0401C082803D232F81030A5
:102F10008B42F8D170470000500700200DF03BBDF8
:102F20000449002008604FF0E0210220C1F880022F
:102F300070470000FC1F00400E4A12680C498A428C
:102F40000AD118470B4A1268094B9A4204D101B5BD
:102F50000EF032FB03BC8E46074909680958084742
:102F600006480749054A064B70470000000000006C
:102F7000BEBAFECA8C00002004000020E010002031
:102F8000E010002070B50C46054606F0E9FD21462C
:102F90002846BDE8704007F0C3BD10B50EF08CFEAA
:102FA0000EF095F9FFF70CFB16F000FB0EF084FD18
:102FB000BDE810400EF010BE08B5DDF808C0009363
:102FC000634609F09BFF08BD134610B50A46194633
:102FD00009F08EFF80B210BD09F0BEBF0AF02AB919
:102FE0000AF03AB909F0BABF0AF022B800220AF092
:102FF000DDB80AF05EB80AF097B80AF03FB970473A
:1030000010FFFFFFDBE5B15100B001007900FFFFC9
:1030100030B5FB4D044610280BD0112C07D02846A4
:10302000122C817808D0132C0BD017F03CFDAC701B
:1030300030BD17F038FDFAE71129F8D017F033FD4D
:10304000F5E71129F3D017F02EFDF0E7EC4810B5A5
:10305000C17894B0A9B117218DF800104168CDF85E
:1030600002100089ADF8060009A9684608F0AAF91F
:103070000446112802D00CB117F015FD14B02046FB
:1030800010BD3221E8E702210AF051BC2DE9F041E0
:1030900094B01D4690460E460746FFF7F4FF040025
:1030A0000BD02078222804D3A07FC0F34010A84280
:1030B00006D1082014B0BDE8F08143F20200F9E720
:1030C00037208DF80000ADF802703DB101208DF879
:1030D00004008DF805608DF8068002E000208DF870
:1030E000040009A9684608F06DF9A07F65F3451052
:1030F000A0770020DEE730B50446A1F120000D46A0
:103100000A2854D2DFE800F005080E1F272D3B41A6
:10311000474D17F0C8FC4CE02078202849D117F023
:10312000C2FC46E0B6480178032942D080781328D3
:103130003FD0207824283CD025283AD0232838D0E6
:1031400017F0B1FC35E02078222832D0232830D87F
:1031500017F0A9FC2DE0207822282AD017F0A3FC34
:1031600027E02078222824D0242822D0262820D006
:1031700027281ED029281CD017F095FC19E02078AC
:10318000252816D017F08FFC13E02078252810D0C2
:1031900017F089FC0DE0207825280AD017F083FC71
:1031A00007E02078282804D017F07DFC01E017F014
:1031B0007AFC257030BD30B50B8840F67B444FF665
:1031C000FF72022801D0934204D09D1FA54224D251
:1031D000022802D04D88954203D04D88AD1FA542EC
:1031E0001BD24C88A34218D88B88B3F5FA7F14D22F
:1031F000022802D0C888904205D0C88840F677459A
:103200000A38A84209D2C888904208D0944206D011
:103210005B1C6343B3EB800F01DB072030BD002054
:1032200030BDF0B5774988423DD3784A764D126873
:10323000A84201D3904236D3047934B1082C02D885
:10324000067B082E05D90720F0BD037B002BFAD0A2
:10325000F6E734B103688B4225D3AB4201D39342E6
:1032600021D336B183688B421DD3AB4201D3934245
:1032700019D300230AE0076857F823708F4212D34E
:10328000AF4201D397420ED35B1CDBB29C42F2D813
:1032900000230CE0846854F823408C4203D3AC42F2
:1032A00003D3944201D21020F0BD5B1CDBB29E42DE
:1032B000F0D80020F0BD10B5028943F6FD73111F50
:1032C000994212D2418904290FD3B1F5804F0CD80D
:1032D00091420AD80178890705D5406818B1FFF7EF
:1032E000A0FF002800D1002010BD072010BDF0B5C0
:1032F0000024059D10B1A94203D851E009B900206E
:10330000F0BD0920F0BD055D8DB107197E78112E45
:103310003FD00FDC0A2E3CD2DFE806F03B16242417
:103320002A2A2C2C3333025D72BB641CE4B28C421B
:10333000F9D3E4E71C2E2CDAA6F11206042E28D2CB
:10334000DFE806F027271018022DDAD1BD781D70AE
:10335000072D01D26D0701D40A20F0BD157845F084
:10336000010515E0EE43F60707E0012D07D010E058
:103370000620F0BD2E07A6F18056002EF5D060463F
:10338000F0BD1578AE0701D50B20F0BD45F0020564
:103390001570055D641C2C44E4B28C4202D9B0E780
:1033A0004FF4485C8C42AED3A9E710B504784CB119
:1033B000012243F20223012C07D0022C0CD0032C53
:1033C00014D10FE000220A7012E00A7082790324FF
:1033D000B4EB921F0AD10BE00A708479B2EB941F10
:1033E00004D105E00A708279920901D0184610BD17
:1033F00050F8012F41F8012F80888880002010BDEF
:10340000A801002000B00100000000201C000020E6
:1034100008B538B1FEA06B4600680090487903EB10
:10342000901000781070086842F8010F888890802A
:1034300008BD30B50C46097895B0222902D2082083
:1034400015B030BD28218DF80010ADF80200132A08
:1034500003D03B2A01D00720F2E78DF8042009A908
:10346000684607F0AFFF050003D121212046FFF792
:1034700042FE2846E4E700B595B023218DF8001000
:10348000ADF802001088ADF804005088ADF80600D1
:10349000D088ADF80A009088ADF808000020ADF89B
:1034A0000C00ADF80E0009A9684607F08BFF15B0B7
:1034B00000BD70B50E46050003D0002109200EF0B6
:1034C000A6FAD44C0120022EE0701DD0032E01D0AC
:1034D00017F0E9FA0621201D0DF092FF607A20F026
:1034E000C0006072FFF7B2FD608A00280BD0002D8B
:1034F00009D083000122002109200EF0EAF90928F1
:1035000001D017F0D0FA70BD0321E01D0DF078FF57
:10351000607A20F0C00040F040006072E01C02F0D1
:103520004FF9DFE72DE9FF410220BA4E8DF8040084
:103530000027F08AADF80600B84652E001A80AF06C
:1035400054F9050006D0F08A90B3A6F81680ADF8BD
:10355000068044E0039C2078212840D0A07F01070A
:1035600027D504F122000090628EBDF808002146A4
:1035700004F1340301F074FB050004D0112827D0B6
:1035800017F091FA24E0A07F20F00800A077E07FF8
:10359000410861F3000094F8201061F3C700E07760
:1035A0002078282825D129212046FFF7A4FD20E0F6
:1035B0001DE0400713D5BDF80800214604F10E02B6
:1035C000FFF759FF050005D0112801D017F06BFA5D
:1035D00000250EE0A07F20F00400A07709E07F1C0A
:1035E000FFB202200AF04CF9401CB842A6D8052DC3
:1035F00007D0BDF80600F082052D04D0284604B09F
:1036000059E5A6F816800020F9E72DE9F0470400F7
:1036100001D117F048FA20787E4E20F00F00801C70
:1036200020F0F0007030207060680178091F1129C7
:103630000CD2DFE801F0F2090B54F10B0DF1F13976
:103640000B0B0B0BF27BF20017F02DFABDE8F087A5
:1036500087883846FFF717FD050001D117F023FAD8
:103660006078212140F008006070307D40F0040057
:1036700030752846FFF73FFD3846FFF7CCF938464E
:10368000FEF7ECFC384603F0F6F9394602200EF05E
:10369000BEF9A87F20F01000A877FFF743FF0028AD
:1036A000D4D017F000FAD1E785882846FFF7EBFC65
:1036B00008B917F0F8F960688078012801D017F090
:1036C000F2F9606881792846FFF7CBFA0028BDD06F
:1036D000617841F0080161706168C880B6E786884A
:1036E0003046FFF7D0FC050001D117F0DCF9607817
:1036F000314640F0080060706068C08828816068CA
:103700000089688160684089A88102200EF07FF9F5
:103710000020A875A87F00F00300022896D1FFF7CB
:1037200001FF002892D017F0BEF98FE780783C287F
:1037300003D0002502280BD000E00125002728B186
:103740003C2803D0022801D017F0ADF917B184E06E
:103750000127F4E7607840F008006070307D40F0A9
:1037600008003075F5BB60680221878838460AF08A
:10377000D5F80546032138460AF0D0F882460521DF
:1037800038460AF0CBF88146042138460AF0C6F8DC
:1037900080460DB917F087F9BAF1000F01D117F083
:1037A00082F9B9F1000F01D117F07DF9B8F1000FDE
:1037B00001D117F078F922212846FFF79CFC6068B8
:1037C0008079012838D04FF00208A87F68F3010003
:1037D000A8776068C08A28816068008B688160680B
:1037E000408B00E02BE0A8816068C079E8756068D4
:1037F0008168A9618089A8836068807B687060683F
:1038000050F80F1FC5F802108088E880A87F05E0F7
:103810000302FF01A80100202DE031E000F00301C8
:103820003846FFF7DEF8B8F1010F08D0B8F1020F03
:1038300013D017F038F909E74FF00108C5E73078E1
:10384000032801D017F02FF9002108460EF0DFF809
:10385000BDE8F047012000F0E7BFB078132801D0A1
:1038600017F021F9002107200EF0D1F8BDE8F0474C
:103870001120FFF7CDBB2046BDE8F04701F05BBC4F
:10388000607840F008006070E0E62DE9F0470546FA
:10389000007800270009DFF8ACA691460C463E46AA
:1038A00001287DD000234FF6FF71022879D0072828
:1038B0000BD00A2876D017F0F6F800BFA9F8006000
:1038C0000CB1278066800020C0E6686802780D2A67
:1038D0003BD006DC042A66D0072A40D00A2A7DD1D4
:1038E00006E0122A42D0132A4AD0142AF7D1BDE0AA
:1038F00011270726002C72D0B0F80480A4F80480A9
:1039000068688079A0719AF81410404621F004018B
:103910008AF8141004210AF014F8052140460AF030
:1039200010F8002140460AF00CF8012140460AF048
:1039300008F8032140460AF004F8022140460AF044
:1039400000F8404607F07CFEB8E701270926002C66
:10395000D1D08088A080686880792072AEE7122775
:103960000E268088214600F08CFFA7E71A2707263D
:10397000002CC0D04088A08068680079A0719DE7C5
:1039800081783C293AD010271E26002CB3D080889D
:10399000A0806868C08A20836868C08AE08203E0EB
:1039A0007BE0A5E073E033E06868A21D008B6083D4
:1039B0006868408BA0836868417F607D61F3000088
:1039C00060756968497F490861F3470060756968F7
:1039D000C8790831FFF71CFD696801E056E086E010
:1039E000887B04F10D020F31FFF712FD68688079C2
:1039F00010B10120207506E00220FBE719270726F9
:103A0000002C74D0A3719AF8141021F008018FE0F3
:103A10001B272E26002C6AD0A1806968A21D481D94
:103A20000B7901461846FFF7F3FC686890F82B0005
:103A300060736868C0780428A07B14D020F001006F
:103A4000A07369681F22C97861F34200A073696896
:103A5000C97A61F3C700A073696804F10F000C31E3
:103A600016F054FF2AE740F00100E9E71E270E2672
:103A7000ECB3A1806868E21D407AA0716968C81C37
:103A80008B7801461846FFF7C3FC17E74A462146E4
:103A90002846BDE8F04701F0CDBC287E012804D0BF
:103AA000022814D016F0FFFF08E71D270E26F4B1F8
:103AB0006888A080A88BE080E88B2081288C6081BA
:103AC000688CA0819AF8141021F0200130E01227B0
:103AD0000E26688800F0D5FE4CB1687800F007002B
:103AE0000328BFD19AF8141021F0020120E027E04A
:103AF000287E062821D2DFE800F0040E0E0303031F
:103B0000C4E719270726DCB1A180A3719AF8141025
:103B100021F001010CE0192707268CB1A180287E35
:103B2000012808D00320A0719AF8141021F0100188
:103B30008AF81410C2E60220F5E716F0B4FFBDE6DD
:103B4000A9F80060BFE610B5FE4894B0807813284D
:103B500002D0082014B052E422208DF8000009A9F8
:103B6000684607F02FFC0446002107200DF04FFFA8
:103B70002046EFE700B5F34895B08078122801D0D1
:103B8000082094E41E208DF8000000208DF802002B
:103B90008DF8030009A9684607F014FC0028F0D14D
:103BA000002107200DF033FF1120FFF731FA00202C
:103BB0007DE400B5E34895B00078022801D00328E1
:103BC00018D11B208DF82C0000208DF82E0069469E
:103BD0000BA807F0F7FB002804D19DF801001B2873
:103BE00001D0032063E4002108460DF010FF9DF88A
:103BF000020008B108205AE4012000F015FE002060
:103C000055E42DE9F0410027CE4C0A287FD2DFE8A9
:103C100000F0057E1C7E7E7E7E453C6CFFF7C9FF72
:103C2000002832D104F08EFA00282ED0017821F03D
:103C30000F01891C21F0F00120310170077604F09A
:103C40005FFA207D40F001001EE08EB23046FFF7A3
:103C50001AFA050001D116F026FF2878212814D081
:103C600004F070FA98B1017821F00F01891C21F05D
:103C7000F00110310170022101764680AF7504F029
:103C80003FFA207D40F002002075BDE8F081294612
:103C90003046BDE8F0411322FFF7CBBBA578122DCB
:103CA00004D0132D05D016F0FEFEEEE7FFF762FFFD
:103CB00001E0FFF748FF0028E7D104F043FA0028AD
:103CC000E3D0017821F00F01891C21F0F0012031AF
:103CD0000170122D07D00221017604F011FA207D27
:103CE00040F01000D0E70121F6E7607A0121B1EB46
:103CF000901F02D1022105E009E0800901D016F0F1
:103D0000D2FE0321BDE8F0410020FFF7D2BB16F040
:103D1000CAFEBAE72DE9F04114460D00074601D16D
:103D200016F0C1FE2878012804D0022823D016F00E
:103D3000BAFEAAE73846FFF7A6F9060001D116F049
:103D4000B2FE0220B075207820F00F00801C20F019
:103D5000F000103004F8010B207840F0080004F85F
:103D6000170B95E8070084E807007648017D41F0CD
:103D70002001017589E73846FFF785F9060001D172
:103D800016F091FEA9884FF6FF70814209D1EA88AA
:103D9000824206D131463846BDE8F0411322FFF792
:103DA00048BB814201D1E88898B1207820F00F000B
:103DB000801C20F0F000103004F8010B207840F057
:103DC000080004F8170B95E8070084E807000020B6
:103DD00006E078230022394602200DF07AFD01200A
:103DE000B07552E730B50C46574995B08C423DD37B
:103DF0005749564B0A689C4201D3944236D300235C
:103E000001212038062867D2DFE800F00326474B5F
:103E1000515F002108200DF0D3FD10B1112015B025
:103E200030BD24208DF80000D4F80200CDF8020047
:103E3000A0798DF8060009A9684607F0C3FA0500C5
:103E400033D108230022114618460DF042FD082800
:103E50002BD016F028FE28E0606848B1B0F5000FBE
:103E600004D3B0F1805F03D3904201D21020D6E793
:103E70003C208DF800002088ADF802006088ADF885
:103E8000040009A9684607F09DFA05000DD1606895
:103E900058B1BDF82810018007E0206801F0D0FC7F
:103EA00002E0204600F001FD05462846B7E73D2028
:103EB0000CE000BF8DF8021002E000BF8DF8023068
:103EC00009A9684607F07EFAEEE734208DF8000075
:103ED0002078C007F2D0EDE70720A0E730B54FF417
:103EE000000295B00C46914242D3194953019C42BD
:103EF000096801D38C423BD32038052841D2DFE842
:103F000000F0032D2D2F2D002088FFF7BCF820B1E5
:103F10000078222804D2082081E743F202007EE7DD
:103F200025208DF830002088ADF8320001A90CA8BA
:103F300007F048FA0028EFD1DDF80A10C4F80210A3
:103F400008E00000A801002000B0010000000020EF
:103F50001C0000209DF80E10A17160E706205EE7AE
:103F6000206848B1904203D3984203D3884201D2DB
:103F7000102054E701F058FCFD48408AA080002042
:103F80004DE707204BE7FA480A30704710B5182173
:103F9000F74816F032FD012000F046FC1120FFF733
:103FA00037F8F34C0020211D60744FF4617060827B
:103FB000E01C04F08CF9D4F80300C4F80A00B4F84B
:103FC0000700E081607A2074FFF740F808B116F02E
:103FD0006AFDFDF759FBBDE8104001F072B810B55D
:103FE00004463C2116F009FDA07F20F00300A077D5
:103FF000202020700020A07584F8210010BD70479B
:104000002DE9FC410646DB480D46814206D3DA48DD
:10401000854206D3D9480068854202D21020BDE807
:10402000FC81D34C16B1012E38D12CE0D4F803001A
:104030000090B4F80700ADF804008046677A8DF868
:104040000670E11C2846FFF7B0F90028E7D1FEF71B
:10405000FDFF30B10099C4F80310A4F8078067721F
:10406000DDE7287808B1012808D1D4F80300C4F8A6
:104070000A00B4F80700E081607A2074002109206A
:104080000DF0C5FC0FE0097841B1012906D00229E5
:1040900006D0032904D043F20220C0E70720BEE780
:1040A0000120FFF706FA66740020B8E700B5B0F506
:1040B000000F06D3B0F1805F05D3B049096888428C
:1040C00001D2102000BDAA490246CB78091D18462E
:1040D000FFF79EF9002000BD2DE9F0419AB00500E0
:1040E0004FF000008DF85C008DF858008DF8280026
:1040F0008DF86000A148144688469E499E4A006893
:104100001E4605D08D420AD3954201D3854206D37F
:1041100044B18C4203D3944204D3844202D210208F
:104120001AB0B2E555EA040018D01F270AAB17AA47
:10413000414628460097FFF7DAF80028F0D118AB7F
:1041400016AA314620460097FFF7D1F80028E7D19C
:104150009DF85800C00703D00A20E1E70720DFE7F9
:1041600001AF7DB11A208DF804008DF8068042461B
:104170002946F81C16F0CAFB0BA901A807F022F982
:104180000028CDD17CB120208DF804008DF8066088
:1041900032462146F81C16F0B9FB0BA901A807F01E
:1041A00011F90028BCD172499DF828004870002000
:1041B000B6E770B506460A200C460870154611464B
:1041C000204607F0FFF830B93821217020462946F3
:1041D00007F0F8F820B1082801D143F2032070BDA0
:1041E0002A462146304600F08AFB0446082801D1C1
:1041F00016F059FC204670BD2DE9F041044660A13F
:1042000096B0D1E900015B4A00279442CDE9140140
:1042100010D35A48584B01689C4201D38C4209D3B1
:104220002078012809D16068904203D3984204D3D2
:10423000884202D2102016B027E54D4D287801287B
:1042400001D00820F7E7072009F023FB18B92078F0
:1042500030B1012804D0287D10F00C0F07D101E007
:104260000420E8E7C10702D1A846800701D5112044
:10427000E1E7208A43F6E172A0F120019142217822
:1042800007D3012944D1002842D1618A00293FD1B6
:104290000FE0022901D0032901D1A02838D3012938
:1042A00007D098F80110C90703D0618A81B3B429F7
:1042B0002ED8217831B1012908D0022904D0032950
:1042C00026D115E0002516E0022514E008B9608A21
:1042D00060B104256068007868B101280AD002281E
:1042E00008D0032806D043F20220A4E70125F1E715
:1042F000032500E00127207A30B1012806D00228EA
:1043000007D0032870D106E0002605E0012603E06F
:104310006AE0022600E003260DB1022D13D196B10A
:10432000E06818B1FEF77DFF002884D198F80100FD
:10433000800702D043F201207DE7022D03D1022E37
:1043400052D0032E50D018208DF82C00208AADF8C2
:104350002E00208AADF830008DF8325098F8031006
:1043600000204FF0010879B101296ED10FE0000063
:10437000A801002000B00100000000201C00002067
:1043800007060504030201008DF8330001E08DF8F3
:1043900033808DF83470217801291ED0CDF8350096
:1043A000ADF839008DF83C60207DC0F34002014635
:1043B00062F35F01C0F3800041EA800014A9085C49
:1043C0008DF83B0080B169460BA806F0FBFF002882
:1043D0008BD15DB1022D09D011E0606850F8011F4A
:1043E000CDF835108088DBE7072024E73EB1E06890
:1043F00028B16A460BA9FFF7DCFE00289CD11B20E0
:104400008DF82C008DF82E8069460BA806F0DAFF97
:10441000002891D19DF801001B2816D1052D09D245
:10442000DFE805F0030305050300032000E0022098
:1044300000F0FAF9012D0AD0608A40B10022830011
:10444000114610460DF045FA08B10320F3E60020AE
:10445000F1E62DE9FC410C0007464FF0030609D0B8
:10446000F84884426BD3F848844203D3F748006885
:10447000844264D33846FEF706FE050004D028784F
:10448000222804D20820CAE543F20200C7E5A87F2B
:1044900000F0030C2CB121466046FEF78CFE0600AE
:1044A000F1D1EB48BCF1010F06D0BCF1020F18D0DE
:1044B00016F0F9FA3046B2E5AA7D2146012A02D06B
:1044C000007D800701D51120A9E529B96846FDF7CF
:1044D000A0F90028D7D169463846FEF742FB0646C8
:1044E000E8E7A97D022914D1007D800611D424B10A
:1044F000A87F40070BD4002100E001213846FEF7D9
:1045000078FB0600D6D1A875002CD3D002E0112686
:10451000D0E7A4B1224629463846FEF7ACFF06464E
:104520001128C7D1A87F4107C4D4216845F80E1FC0
:104530006168696040F0040028740026BAE7102022
:104540006DE570B50C460546FEF79DFD010005D0F2
:1045500022462846BDE87040FEF76BBF43F20200DA
:1045600070BD00B595B031218DF800108DF80200B6
:1045700009A9684606F026FF15B000BD0123FEF725
:1045800085BD00231A461946FEF780BD70B5044666
:10459000AC4894B0844206D3AB48844206D3AB48BF
:1045A0000068844202D2102014B070BD2046FEF78D
:1045B00082FE0028F8D1A6488178112901D0082070
:1045C000F2E7017DC90601D51120EDE71D218DF827
:1045D00000102178002501F001018DF802102189D9
:1045E000ADF804106189ADF8061021780126C1F3F9
:1045F00040018DF80910C07818B1012804D00320BB
:10460000D2E78DF8085001E08DF8086009A96846E6
:1046100006F0D8FE0028C7D12078800707D560684B
:1046200028B109AA6946FFF7C4FD0028BCD11E20A5
:104630008DF800008DF802608DF8035009A96846D6
:1046400006F0C0FE0028AFD1A08900F00CF90400EC
:10465000AAD11220FEF7DCFC2046A5E7F0B5050044
:104660007A4816460C467749774A006895B005D0D7
:104670008D420FD3954201D385420BD38C4209D38F
:10468000944201D3844205D38E4203D3964204D38D
:10469000864202D2102015B0F0BD6D4F387D10F06B
:1046A000180F01D1400701D51120F4E72046FEF78D
:1046B00002FE0028EFD12078C0F34001294302D048
:1046C000800702D50DB10720E5E731460220FEF74D
:1046D00072FD0028DFD1B878112803D0122801D04C
:1046E0000820D8E7062009F0D4F818B1B8781228C5
:1046F00002D005E00420CEE7FFF73CFA0028CAD13B
:104700002078800707D5606828B109AA6946FFF7B5
:1047100050FD0028BFD121208DF800002089ADF880
:1047200002006089ADF8040020784FF00101C0F369
:1047300040008DF80600207882074FF0000015D465
:104740002A7842B1012A09D0022A07D0032A05D0CB
:1047500043F202209FE78DF8070001E08DF8071073
:1047600055F8012F0292AA88ADF80C20FA781AB1F8
:10477000012A04D003208EE78DF80E0001E08DF8A9
:104780000E103188ADF810107188ADF81210B18894
:10479000ADF81410F188ADF81800ADF81610ADF8AA
:1047A0001A0009A9684606F00DFE00288CD1A089E0
:1047B00000F059F8040087D11320FEF729FC2046A9
:1047C00069E730B595B00C460546B1F5000F06D344
:1047D000B4F1805F06D31D480068844202D21020E5
:1047E00015B030BD2846FEF74EFC38B101782229BD
:1047F00002D3807F800604D40820F1E743F2020050
:10480000EEE713208DF80000ADF8025009A96846C4
:1048100006F0D8FD0028E3D19DF92A107F2901D0A8
:104820002170DDE70520DBE730B5094D040011D02C
:10483000012C05D0022C10D0032C0ED016F033F929
:104840002C7030BD00B00100000000201C000020D2
:10485000A801002016F027F9F2E728780128EFD008
:1048600016F021F9ECE710B548B18300002211469B
:1048700007200DF02EF8072801D0032010BD0020DE
:1048800010BD70B50C0006460ED0FEF7FCFB05000F
:1048900001D116F008F9A6802889E08028892081B6
:1048A00068896081A889A08170BD10B50446006840
:1048B00058B13749884206D33649884205D336492C
:1048C0000968884201D2102010BD00F0A0FFA08826
:1048D000324C6082607C01280FD1002109200DF04C
:1048E0006FF800B10120617A0122B2EB911F01D172
:1048F000022100E00321FEF7DCFD002010BD2DE9C0
:10490000F047002592460C460646A8464FF001099E
:104910000B2721E0306850F82500007820B10128ED
:1049200005D00720BDE8F08784F8028001E084F814
:104930000290306850F8250050F8011FC4F80310A9
:104940008088A4F8070027705146204606F03AFDFB
:104950000028E7D16D1CEDB23079A842DAD80025E5
:1049600039270FE0B068102250F82510A01C15F070
:10497000CDFF27705146204606F024FD0028D1D1F6
:104980006D1CEDB2307BA842ECD80020CAE70000D5
:1049900000B00100000000201C000020A801002041
:1049A000F749884206D3F749884205D3F649096892
:1049B000884201D2102070470178C1F38201042996
:1049C00007D84178072904D38278102A01D88A426F
:1049D00001D207207047C178490702D40079400707
:1049E00001D5062070470020704710B513785C0889
:1049F000C37F64F30003C37710784309087863F337
:104A00000410087013789B0863F343000870507813
:104A1000087310BD30B500240C70C37803F0010397
:104A20000B70C57805F002052B430B70C57805F0B7
:104A300004052B430B701470017901F00101117012
:104A4000037903F0020319431170007900F00400A8
:104A50000143117030BD70B514460D46064603F093
:104A600071FB80B10178142221F00F01891C21F023
:104A7000F001A03100F8181B214615F08CFFBDE8AD
:104A8000704003F03DBB29463046BDE8704013221C
:104A9000FEF7CFBC70B514460E46054603F052FB38
:104AA00070B1017821F00F01891C21F0F001203153
:104AB0000170458021880183BDE8704003F020BB70
:104AC00031462846BDE870401322FEF7B2BC10B54F
:104AD000AE4C94F8300000280DD104F120014FF6BF
:104AE000FF72A1F110000AF011FD08B115F0DBFF13
:104AF000012084F8300010BD2DE9FF5F0646DDE996
:104B00000E5B1C4617461421284615F098FF00211D
:104B1000DFF87482CBF80010F8074FF400094FF06B
:104B2000805A12D02068484549D3504503D3D8F85D
:104B30000010884243D31230286020681430686027
:104B40002068A8602168CBF80010B8072CD56068F1
:104B500038B1484533D3504503D3D8F800108842C4
:104B60002DD3019979B3FFF70EFA0168C6F85C11ED
:104B70008188A6F86011807986F86201FFF7A7FFA7
:104B8000DFF808B20BF1200BC5F80CB062685AB11F
:104B900096F85C0106F25D111032FEF739FC102226
:104BA0005946606815F0B2FE780715D5A0684845EB
:104BB00005D350450FD3D8F8001088420BD21020EF
:104BC00004B0BDE8F09FFFE70028F8D0E860606817
:104BD000C6F85801E8E728610020F1E730B505463E
:104BE00008780C4620F00F00401C20F0F001103136
:104BF00021700020607095F8210028B103280CD0A6
:104C000004280ED015F04FFF20780121B1EB101FC2
:104C100002D2E87FC008607030BD21F0F000203083
:104C200002E021F0F00030302070EDE710B510B157
:104C300090F8644044B1554890F8344000205CB18D
:104C400008601060186010BD00F164040C6000F191
:104C50009001BC301160F5E74C4C34340C60F0E747
:104C600030B595B00C462C2518998DF80050ADF84C
:104C70000200B3B11868019058680290ADF80C209A
:104C800010220DF10E0015F041FE09A9684606F04C
:104C900099FB002803D1A17F41F01001A17715B045
:104CA00030BD00200190E8E72DE9F04F0646008A6C
:104CB00095B080B20D468346FEF7E5F90446334FC2
:104CC0003078283FDFF8C4904FF000084FF02B0AEF
:104CD0000E2872D2DFE800F071F3070E4675809A55
:104CE000B0F4F1F0EFEE15B0324621465846BDE87B
:104CF000F04FB0E6A07F00F00300012806D00021AD
:104D0000584608F014FE050004D101E00121F7E740
:104D100015F0C9FE99F86010090602D5D9F86400AB
:104D20000EE08DF82CA069460BA806F04BFB08B1ED
:104D300015F0B9FE16490198B0FBF1F201FB120023
:104D4000A8617068A862B068E8622078252801D060
:104D500015F0A9FE324621465846FFF77CFE15B0F5
:104D6000BDE8F08FA07F00F00300012806D00021ED
:104D7000584608F0DCFD06000ED10BE00121F7E7F4
:104D800000B00100000000201C0000205C02002098
:104D900040420F0015F087FE2078252804D0307897
:104DA00040F001003070DAE702202870B068A86097
:104DB000B06818B185F80480D1E77FE1012028713F
:104DC000CDE78DF800A0FE49684606F0FBFA08B171
:104DD00015F069FE032016E02A208DF8000010224D
:104DE0000DF10200716815F091FD10220DF1120015
:104DF000B16815F08BFDF249684606F0E3FA08B198
:104E000015F051FE042028706F60A8E7B06808B95B
:104E100015F049FEE07F400701D515F044FEB0686B
:104E200000903379062204215846FDF745FE0028FC
:104E300095D015F038FE92E70CB915F034FE04F168
:104E4000220010220546716815F060FD28212046D9
:104E5000FEF751F9A07F00F0030002280CD10023D7
:104E60001A46214658460095FFF7FAFE112809D048
:104E700029212046FEF73FF9317AE07F61F3C70030
:104E8000E0776CE7A07F000701D515F00CFEA07F4E
:104E900040F00800A077A4F83280C4F83480C4F849
:104EA0003880E07F014660F34101E177307A84F891
:104EB000200054E7FEE073E069E04EE000E02AE005
:104EC000A07F00F00300012806D00021584608F01A
:104ED0002EFD040004D101E00121F7E715F0E3FD08
:104EE0008DF800A0B649684606F06CFA08B115F0D6
:104EF000DAFDB348808824F8390F1220287004F2B4
:104F00002310686034F809092882AD486C613C3090
:104F1000C5E9029023E70CB915F0C5FD20782128DA
:104F200089D93079012802D002280AD103E0E07F34
:104F300040F00400E07799F8601041F0010189F831
:104F40006010324621465846FFF785FD15B02046D1
:104F5000BDE8F04F2321FEF7CEB8012204215846C8
:104F6000FDF7E8FE00288CD0132028701721297146
:104F7000CDF8008002AB00225846CDF80480FDF742
:104F8000CFFB08B115F08FFD0298A860E7E6042179
:104F90005846FDF717FF00288BD114202870DEE655
:104FA000A07F00F00300012806D00021584608F039
:104FB000BEFC050004D101E00121F7E715F073FD07
:104FC00095F83800410639D5A17FC00701F00301EB
:104FD0000ED0D5F854215AB195F83730107C63F3D0
:104FE00047001074E37FD5F8542163F30000107478
:104FF00095F8380000070ED5D5F850215AB195F82C
:105000003730107C63F347001074E37FD5F85021EC
:1050100063F30000107495F83800820701D5022967
:1050200003D0C0060AD5012908D1D5F8582195F832
:10503000300005F131011032FEF7EAF905208DF854
:10504000000095F838008DF801005D48703802784E
:1050500022F00F02921C22F0F002203202704278FD
:1050600022F00702D21C4270A0F802B0BDF8001076
:10507000018303F0D1F92078252806D0212808D013
:1050800015F011FD2078222803D922212046FEF7B1
:1050900032F8A07F00F00300012809D00021584613
:1050A00008F04FFC00283FF47EAE15F0FCFC56E6FD
:1050B0000121F4E7716881F8008050E615F0F3FCF7
:1050C0004DE670B53E4C00252C3414F8600F20F0EE
:1050D0008000207065600AF0A6F939493C31A1F1E1
:1050E000100003F027F904F8305C70BD70B50D4670
:1050F000FDF7C9FF040001D115F0D5FC4FF4B271E2
:10510000284615F09CFCA07F00F0030001280AD07F
:105110005FF0020105F1E8000AF086F9002801D0ED
:1051200015F0C1FC70BD0121F4E70A46014602F109
:10513000E8000AF090B970B5054640689AB0017869
:1051400008290DD00B2903D00C2938D101218171F8
:10515000686886883046FDF796FF04003BD138E04A
:1051600046883046FDF78FFF040001D115F09BFC07
:105170002078212823D0282826D1686802210C30E5
:1051800000F042FF00B368680821001D00F03CFFFA
:10519000D0B12D208DF80000ADF80260102204F18E
:1051A000220101A815F0B2FB09A9684606F00AF928
:1051B00008B115F078FC29212046FDF79CFF01E09D
:1051C000300200201AB070BD687840F008006870A6
:1051D000F5E715F068FCA07F00F00301022902D179
:1051E00020F01000A077207821280BD06868817902
:1051F00009B1807890B1A07F00F00300022859D057
:1052000015F051FCA07F00F003000228D7D1FEF773
:1052100089F90028D3D015F046FCD0E7687840F033
:1052200008006870E07FC00701D0042000E0032080
:1052300084F821002078292817D02428E2D131468B
:1052400006200CF0E4FB22212046FDF754FFA07F4E
:1052500000F0030001282BD00021304608F071FB3C
:105260000028CFD015F01FFCCCE7A07F00F0030092
:10527000012806D00021304608F059FB050004D172
:1052800001E00121F7E715F00EFC25212046FDF78E
:1052900032FF11208DF8500014A905F1E8000AF042
:1052A000D1F80228AED00028ACD015F0FCFBA9E75D
:1052B0000121D2E7687840F008006870A2E72DE984
:1052C000F0418CB0164688460746FDF7DCFE040028
:1052D0004FD0207822284CD323284AD0E07F4007A3
:1052E00047D4A07F00F00300012806D000213846F3
:1052F00008F01DFB050002D00BE00121F7E7A07FBD
:1053000000F00300012804D10121384608F006FB13
:10531000054601AB02AA03A92846FFF787FC0398BC
:1053200008B915F0C0FB45B10398E8354561207810
:10533000222806D0242804D007E0039900204861E1
:1053400003E025212046FDF7D6FE03980D210170CC
:1053500047620671C0F808800299C1600199016135
:1053600004A90AF08FF8022803D0002801D015F014
:105370009AFB0CB0BDE8F08130B589B00546FDF769
:1053800082FE017822292DD9807F00F003000128B8
:1053900006D00021284608F0CAFA040004D101E032
:1053A0000121F7E715F07FFB13208DF80C0000209A
:1053B00017210090024601908DF8101002AB28468C
:1053C000FDF7AEF908B115F06EFB0298059003A940
:1053D00004F1E8000AF036F8022803D0002801D0D2
:1053E00015F061FB09B030BD10B586B00446FDF77D
:1053F0004AFE017822291BD9807F00F00300012892
:1054000006D00021204608F092FA040004D101E001
:105410000121F7E715F047FB14208DF800006946DD
:1054200004F1E8000AF00EF8002801D015F03BFB6B
:1054300006B010BD2DE9F0470546002700789046DC
:1054400000090C463E46BA46022875D0072802D00D
:105450000A280AD142E068680178082906D00B2999
:105460002BD00C2929D015F01EFB2AE114271A266F
:10547000002C79D04088A080FDF705FE5FEA000986
:1054800001D115F010FB99F81700A21D09F11801C0
:10549000FDF7BEFF68688089E08168684168216126
:1054A00080686061207E20F0060040F001002076D8
:1054B00099F81E0040F040013BE018270826002C18
:1054C000D7D08088A080FDF7DEFD050001D115F062
:1054D000EAFAA11D2846FFF781FBF2E00CB1288D06
:1054E000A080287E01287CD0022804D0032827D061
:1054F00015F0D9FAE5E01C270726002C34D0A08847
:10550000FDF7C1FD5FEA000901D115F0CCFA287F53
:1055100000F003000128A0790FD020F00100A07155
:10552000297F890861F34100A07199F81E0040F0BD
:10553000800189F81E10C4E0B7E040F00100EEE7FA
:1055400013270B26002C0FD0A088FDF79CFD814669
:10555000807F00F00300012807D00021A08808F018
:10556000E6F9050005D102E08EE00121F6E715F02D
:105570009AFA99F81E0000F00300012838D0E96A71
:10558000887800F003000128A07933D020F00100D2
:10559000A0718A78920862F34100A0710A7862F3E0
:1055A0008400A0714A7862F34510A07184F807A0C6
:1055B000C87820724A79607A530862F3000063F376
:1055C00041009208097962F382006072A07A4A0869
:1055D00061F3000062F34100890861F38200A07268
:1055E00000E00AE099F8000023286AD92621B1E0FA
:1055F000A96AC5E740F00100CAE7297F0122F948FE
:1056000002290DD017270C26F4B301290DD0032948
:1056100018D0042919D0052917D015F044FA20E034
:10562000192707268CB3A27104E0A271E17921F059
:105630000301E17110F8601F4A08520062F306018D
:1056400001700EE00220A07107E0687F052900F0DC
:105650000F0040F08000A0711DD0E07920F0030021
:10566000E071A088FDF70FFD05460078212828D0BD
:10567000232801D015F017FAA87F00F003000128B5
:1056800011D00021A08801E00AE01AE008F059F9E1
:10569000222128465FE0E07920F00300401CDFE78C
:1056A000A8F8006012E00121ECE70CB16888A08046
:1056B000287E03282AD004280BD005284ED015F0C8
:1056C000F2F9A8F800600CB1278066800020BDE8E0
:1056D000F08715270C26002CE2D0A088FDF7D3FC1C
:1056E000807F00F00300012806D00021A08808F088
:1056F0001EF9050004D101E00121F7E715F0D3F907
:105700000622A11DA86905F09CFEDAE716270726E8
:10571000002CC5D0A088FDF7B6FC8146807F00F044
:105720000300012806D00021A08808F000F9050038
:1057300004D101E00121F7E715F0B5F92878C0069A
:1057400001D5022000E00120A07199F80000232873
:10575000B7D927214846FDF7CEFCB2E717270C261C
:10576000002C9DD0A088FDF78EFC6D7E5FEA0009BD
:1057700001D115F098F9C4F806A0A4F80AA084F89D
:1057800006A0207A40F00300207299F81F1061F300
:1057900082002072680694D5E079EA0840F004009F
:1057A000E071E17AA07A62F3000165F300006A0813
:1057B00062F34100A072280960F34101E17280E7C1
:1057C00030B504468079012591B0B5EB901F01D02A
:1057D00015F069F9FFF77BF94FF6FF7009908148E2
:1057E0008DF8005020300190201D0290601C0C901C
:1057F0000BA9684609F046FE08B115F054F90C985B
:105800000188A4F801108078E07011B030BD10B5A7
:10581000744C30B10146102204F1200015F076F8E6
:10582000012084F8300010BD10B50446FFF74FF991
:105830006C4920461022BDE81040203115F066B8B2
:1058400070B5684C0025D0B16749884206D36749D6
:10585000884205D366490968884201D210250CE0C8
:10586000062105F0D5FD411C06D0606614F8600FD6
:1058700040F08000207000E00725284670BD14F835
:10588000600F20F08000F5E72DE9F0418EB00C00AC
:1058900080464FF0000709D0534884421BD3534839
:1058A000844203D352480068844214D34046FDF733
:1058B000EAFB050003D02878222814D103E043F244
:1058C00002000EB056E544B9A87F010603D500F0EA
:1058D0000300022801D01020F3E7A87FC10601D4FD
:1058E000010702D50CB10820EBE73E4991F86010A2
:1058F000C90701D01120E4E7E97F490701D50D2050
:10590000DFE700F00300022805D124B12046FFF7AD
:1059100047F80700D5D1A87F00F00300012806D082
:105920000021404608F003F8060002D00CE00121F7
:10593000F7E7A87F00F0030001280BD000214046C4
:1059400007F0ECFF060007D0A87F00F00300022854
:1059500004D009E00121F2E70420B2E724B1224695
:1059600031462846FFF741F80DAB1A4603A93046E9
:10597000FFF75CF9039808B915F095F803980E2124
:10598000017006F1E801C0F824808160A97F01F070
:10599000030101292FD06CB302210171311DC160B7
:1059A0003178C1F3420101743178C1F300114174BF
:1059B000217801F00102817C62F301018174EA7FA8
:1059C00062F382018174A178C17405AA04A92046FA
:1059D000FFF720F803989DF8141001759DF810103A
:1059E00041751FE05C02002000B0010000000020B3
:1059F0001C00002012E001210171217801F0010258
:105A0000017B62F3010101732278520862F3820183
:105A1000017324212846FDF76EFB0BE00321017181
:105A20000521017325212846FDF765FBA87F20F09D
:105A30008000A87707A9039809F024FD022802D066
:105A400008B115F030F838463BE72DE9FF4F934693
:105A5000F84A89468FB09A4607CA0BAB4FF0000848
:105A600083E80700CDF80080CDF804800F98FDF79B
:105A70000AFB050006D02878262806D0082013B097
:105A8000BDE8F08F43F20200F9E7A87F00F00307BA
:105A9000012F02D0022F09D00BE0B9F1000F08D17D
:105AA0005846FEF77DFF0028E9D102E0BBF1000F68
:105AB00016D14846B9F1850F1CD008DC90B1812879
:105AC00012D0822812D0B9F1830F09D110E08628B4
:105AD00012D0882812D0892812D0B9F18A0F11D09B
:105AE0000720CCE700260EE001260CE002260AE0A3
:105AF000032608E0052606E0062604E0082602E064
:105B0000092600E00A26A87F00F00300012806D03D
:105B100000210F9807F00BFF040004D101E00121E0
:105B2000F7E714F0C0FF012F0FD1B9F1000F0CD12E
:105B30005A4621462846FEF758FF9BF8020001907E
:105B40009BF8000000F0010000900020207101216E
:105B50008DF81410211D06910EB12671FAE0012F67
:105B60000CD0D4E90A610223894601220020A060FA
:105B700005F11700022A1AD0012119E0D4E90A968A
:105B800001230222032131702178C1F300117170C9
:105B9000B178DDF804C086F803C0DDF800C021F05C
:105BA00004016CF30101B17070713071DEE7002106
:105BB00004EB81010861681C022B01D0012100E087
:105BC000002104EB81010861B07800F00300012896
:105BD0005DD199F8020000F00300012857D199F82F
:105BE0000400019099F805000090012F1ED0307933
:105BF0008DF8080070798DF80C0000BF9DF8082022
:105C00000198009902409DF80C0000EA010B52EA4D
:105C10000B003CD088498A4506D388498A4515D36C
:105C2000874909688A4511D2102028E702AA03A9EA
:105C30005846FEF7EFFE9DF80800019908403071C4
:105C40009DF80C00009908407071D7E704F5A87121
:105C500004F13C00022FCDE9000135D05FF00001D6
:105C60000AF10C032046FEF747FF0028DDD104F5BA
:105C7000AA7104F15000012FCDE9000126D00021C6
:105C800053465A462046FEF737FF0028CDD199F8F3
:105C90000200400702D4E87FC0072FD00BA8012FD5
:105CA00016D099F8001030F811002178C1F34201A4
:105CB0004900C84010F0030080462AD0012816D0C1
:105CC000B8F1020F0FD114E00121C9E70121D7E794
:105CD0002178C1F3420130F8110099F80010490011
:105CE000C84000F00308B8F1030F05D006E0022019
:105CF00000E0012080460CE04FF00208012F08D19F
:105D0000E87FB17860F38201B1702078C0F342007F
:105D100030702078EF2220F00100207099F80110F7
:105D200001F0010142EA011108402070C00621D4AF
:105D3000B8F1020F1ED0B8F1010F1DD00020A061F4
:105D4000E0612062606204F11800A060E87F20F04A
:105D50000100E87705A904F1E80009F073FB18B128
:105D6000022801D014F09FFE25212846FDF7C3F933
:105D7000002084E6032008E00D2104F11B0014F04C
:105D80003CFE04F11800A06004208DF81000E87FAC
:105D900004AA40F00100E87729460F98FEF77AFE42
:105DA000D8E7F0B587B015460F0004460CD022485E
:105DB000854206D32148854206D3214800688542A2
:105DC00002D2102007B0F0BD2046FDF75CF90600B6
:105DD00004D03078272804D00820F3E743F20200EB
:105DE000F0E7B07F00F00300012806D00021204634
:105DF00007F09DFD040004D101E00121F7E714F054
:105E000052FE00202FB1022F08D0012F1AD00720F8
:105E1000D8E701218DF80410A06021E004F11803F7
:105E2000A3608DF8040010222946184614F06EFD78
:105E300016E0000084AC010000B00100000000206A
:105E40001C00002004F11801A1608DF80400A0617D
:105E5000E061206260620621284605F0D9FAA0615F
:105E60002078C10711D020F00100207002208DF8A9
:105E7000000004F1180002906946D03009F0E2FAFF
:105E8000022802D008B114F00EFE25213046FDF79D
:105E900032F9002096E7F8B515460E460746FDF79D
:105EA000F2F8040004D02078222804D00820F8BD9D
:105EB00043F20200F8BDA07F00F00300022802D0E8
:105EC00043F20500F8BD56498E420DD3554A564857
:105ED000964202D303689E4206D38D4204D3954274
:105EE00004D30068854201D21020F8BD00953288A5
:105EF000B31C21463846FEF7B3FE112810D0002807
:105F0000F3D12A7CE17F62F30001E1772A7C520819
:105F100062F3C701E177A17F21F08001A177F8BD8D
:105F2000A17F0907FBD4D6F802006063D6F806000B
:105F3000A063308860861022294604F1220014F004
:105F4000E5FC287CE17F60F34101E177287C400893
:105F500084F82000A07F40F00800A0770020DAE756
:105F600070B594B00D46064613B1072014B070BD4D
:105F7000FDF789F8040007D02078222802D3A07FFB
:105F8000400604D40820F1E743F20200EEE7A5B191
:105F90002D208DF80000ADF802601022294601A8DE
:105FA00014F0B4FC297CE07F61F30000E077297CE9
:105FB000490861F3C700E07704E02E208DF8000067
:105FC000ADF8026009A9684605F0FCF9A17F21F04F
:105FD0004001A177CAE710B50C46FDF754F858B157
:105FE000B4F5000F06D3B4F1805F08D30E490968F9
:105FF0008C4204D2102010BD43F2020010BD214695
:10600000FEF7ECFD002010BD05E000BF10F8012BED
:106010000AB100207047491E89B2F7D201207047AB
:1060200000B00100000000201C00002018B18178A1
:1060300001293CD101E010207047018842F602138B
:10604000C81A4FF48072994233D01CDC42F6010327
:10605000A1EB030099422CD00CDCF9B1B1F5C05F83
:1060600027D06FF4C050081823D0A0F57060FF3817
:106070001DD11EE001281CD002281AD0FF2818D0FC
:10608000904214D115E0904213D008DC012810D0C2
:1060900002280ED0FE280CD0FF2808D109E0A0F578
:1060A0008070013805D0012803D0022801D00020DB
:1060B00070470F2070470B2826D008DC1BD2DFE882
:1060C00000F01C2025251A25292325271E0011282C
:1060D0001CD008DC0C2817D00D281DD00F2815D097
:1060E000102808D110E0822809D0842810D08528F3
:1060F00010D0872812D00320704700207047052059
:10610000704743F203007047072070470F20704725
:1061100004207047062070470C2070474FF4505001
:10612000704707280DD2DFE800F00406040C0C08C5
:106130000A00002070471120704707207047082090
:10614000704703207047007810F00F0204D0012A36
:1061500005D0022A0AD10EE0000907D108E00009A3
:10616000012805D0022803D0032801D0072070475A
:106170000870002070470620704738B1012809D008
:1061800002280FD0032815D007207047087820F088
:10619000FF0016E0087820F00F00401C20F0F0000F
:1061A00010300EE0087820F00F00401C20F0F000C6
:1061B000203006E0087820F00F00401C20F0F000AE
:1061C000303008700020704738B50C46050041D0CB
:1061D0006946FFF7B8FF002819D19DF80010208804
:1061E00061F38B2020806946681CFFF7ACFF002814
:1061F0000DD19DF80010208861F30D302080A97822
:10620000C1F34101012903D0022904D0072038BD80
:1062100020F0200001E040F02000208080B210F447
:10622000406F04D0A978C90861F38E30208080B215
:1062300010F4405F07D0A978090961F3CF302080BE
:1062400010F4405F02D12088400403D5208840F03C
:1062500040002080002038BD70B504460020088032
:1062600015466068FFF7B0FF002816D12089A18984
:10627000884211D860688078C0070AD0B1F5007FE5
:106280000AD840F20120B1FBF0F200FB1210288086
:1062900007E0B1F5FF7F01D90C2070BD01F20121AB
:1062A0002980002070BD10B50478137864F30003D2
:1062B00013700478640864F3410313700478A4082D
:1062C00064F3820313700478E40864F3C303137067
:1062D0000478240964F3041313700478640964F3E4
:1062E000451313700078800960F38613137031B181
:1062F0000878C10701D1800701D5012000E0002006
:1063000060F3C713137010BD028812F4406F02D0FF
:10631000C2F3812306E012F4405F02D0C2F30133DE
:1063200000E001230A8863F38B220A80008810F4BE
:10633000405F02D0C0F3013006E010F4406F02D09D
:10634000C0F3812000E0012060F30D320A80704725
:106350002DE9F04792B00D00804613D0B8F1000F40
:1063600014D01221284614F048FB03AAFF21012073
:1063700004F069FE0024264637464FF420596FF496
:10638000205A6DE0102012B0BDE8F0870720FAE730
:106390009DF8160001280AD1BDF8140048450BD01D
:1063A00010EB0A000AD001280CD002280CD0042CD3
:1063B0000ED0052C0FD10DE0012400E00224BDF821
:1063C000126008E0032406E00424BDF8127002E025
:1063D000052400E00624BDF81210414540D12C747C
:1063E00086B34FF005090DF134080EAACDF80090E0
:1063F000CDE9012810230022FF21304604F0BFFE22
:10640000F0B9BDF834002A46C0B20EA909F02AF945
:10641000B0B9AE81B7B108AECDF80090CDE9016852
:1064200013230022FF21384604F0A9FE40B9BDF82D
:106430003400F11CC01EC0B22A1D09F013F910B1BE
:106440000320A0E70AE0BDF82100E881062C05D171
:106450009DF81600A872BDF814002881002092E76C
:1064600003A804F0F8FD002892D0FFF724FE8AE785
:10647000002805D0F74A012903D0022903D00320C0
:106480007047518800E09188814201D10020704717
:10649000072070472DE9F0438BB00E46DDE91298D6
:1064A00005461C461746142103A814F0C8FA01201B
:1064B0008DF810008DF80C008DF81180ADF8147077
:1064C00064B1A178C90709D08DF81600E088ADF84D
:1064D0001A00A088ADF81800A068079001F032FEFD
:1064E000040023D06580002017210090024601900F
:1064F000ADF8201009AB2846FCF712F9002812D19C
:1065000008368DE8700008AA494603A8099B04F0E4
:10651000D8F806466078000701D501F0F1FD5EB1BC
:106520003046FFF7FEFD0BB0BDE8F083132128468F
:10653000FEF707F80320F6E709980090BDF8203031
:10654000042201212846FCF7B7FAECE770B50646AD
:106550008AB000200D46059005240490069003A9FA
:1065600000940790CDE901010246102329463046E8
:1065700004F005FE68B904A9009108A8CDE901401E
:10658000BDF80C3000222946304604F009FC0028F2
:1065900001D0FFF790FD0AB070BD04F0CFBA2DE92D
:1065A000FC470546002700780C46B846B9460C283B
:1065B00078D2DFE800F0C4060E32DB6363859EBF4D
:1065C000A3AF0CB114F06FFA288980B201F02FFF4D
:1065D000B7E0A888042180B2814607F0A8F90646F2
:1065E0000CB114F060FA0EB914F05DFA494606F1E8
:1065F000080003F0CFFC01F0A5FD040008D060788E
:1066000040F008006070A4F8029001F079FD99E074
:1066100013214846FDF795FFA8E00CB914F043FAA2
:106620006088042107F083F9060001D114F03BFAD9
:10663000A6F80090002029791DE000BF05EBC002FC
:10664000128992B2130707D5D30605D505EBC10011
:1066500030F8020C308006E052040AD5307105EBA8
:10666000C000C08870806078022740F00800607029
:1066700067E0401CC0B28142E0D862E0E888ADF833
:1066800000000CB914F00FFABDF80000000404D5A6
:106690002878062807D005282ED0607840F008001A
:1066A00060704EE04BE06088042107F040F906007E
:1066B00001D114F0F8F986F80490A88870801BE0E6
:1066C0000CB914F0F0F96088042107F030F90600E5
:1066D00001D114F0E8F906F1080004F083FA90F013
:1066E000010F02D1E88800042BD560880227F080D2
:1066F000D3E70CB914F0D7F90227CEE70CB914F0A0
:10670000D2F9022761880122204601F0C5FE4FF030
:106710000108C2E7A88986B20CB114F0C4F9686810
:1067200000902889ADF8040001226946304601F046
:10673000D0FE06E0002CB0D114F0B5F9ADE714F0AE
:10674000B2F99CB16078000710D5B8F1000F0DD1F7
:106750002078582220F00F00001D20F0F00080303B
:106760002070294604F1180014F015F93846BDE8E8
:10677000FC872DE9F04F054687B00C46007E0A31B4
:10678000019104F10C010027039190461631821EFD
:106790003E46BB464FF0010A0291082A7DD2DFE84F
:1067A00002F0FC047C32327FBDFD6888042107F0D2
:1067B000BEF85FEA000901D114F075F9B9F80000DC
:1067C00010B152270726F0E051271E26002C7DD05D
:1067D0006888A08084F806A099F80400019905EB68
:1067E000C000C08BFFF7B4FD002870D199F80400F9
:1067F00005EBC000C08B208199F8040005EBC000B8
:10680000408CA083ECE0B5F82290062824D1E88BD8
:10681000000421D5512709F1220086B2002CD6D0E0
:10682000A88B0399FFF794FD002874D16888A08095
:106830000220A071A88B208184F80AA0288CE08314
:10684000A4F820904A46696ADDF8080014F05EF862
:10685000C6E00000C4020020502709F1200086B2E3
:10686000002C33D0A88B0199FFF772FD002852D17C
:106870006888A080A88BE080287E06280ED00220A1
:106880002072288CA083E88B4A46C00B6072A4F863
:106890001E9004F12000696AD8E79FE00120EFE72D
:1068A0006888042107F043F8B5F822A05FEA0009E0
:1068B00001D114F0F8F809F1080004F093F990F010
:1068C000010F02D1E88B000424D501E042E022E070
:1068D0000AF1220086B25127E4B36888A080A88B11
:1068E0000399FFF735FD002815D10220A071A88B70
:1068F00020810420A072288CE083A4F820A05246B6
:10690000696A029814F002F889F804B0A98BA9F812
:10691000021065E0032007B0BDE8F08F6888FCF73F
:10692000B2FB82466888042107F001F88146BAF17B
:10693000000F01D114F0B7F8B9F1000F01D114F034
:10694000B2F8B9F80600A0F57F41FF3903D051270E
:10695000222602E035E05027202694B36888A080E4
:10696000502F07D00220A071287F04F1080101F008
:1069700041FA35E0287FA11D01F03CFA9AF8211078
:10698000CDE9001BB9F80220688800234946FFF7CB
:1069900081FD0028BFD123E000E016E0FE49A88B6E
:1069A000C988814205D15427062654B16888A08041
:1069B00016E05327082624B16888A080A88BE080C1
:1069C0000EE0FFE7A8F800600FE055270726002C2F
:1069D000F8D0A88BA08084F806B001E014F063F82A
:1069E000A8F800600CB127806680002093E7EA4990
:1069F00000200870704730B585B00C4601F00EFAE3
:106A00000546FF2801D114F04EF8002020802071A7
:106A100060804FF6FF70E080294604F1080003F023
:106A2000ABFA6A462946012004F00DFB16E000BFD0
:106A3000BDF80400000711D5BDF806002946FFF790
:106A400085FDBDF80400FF2340F01000ADF8040000
:106A5000BDF806002946019A04F026FC684604F0B9
:106A6000FAFA0028E4D005B030BD0A46014602F12A
:106A7000080003F095BA70B50546042106F057FFEB
:106A8000040001D114F00FF8294604F10800BDE814
:106A9000704003F07FBA2DE9F0418AB00D46804680
:106AA000FCF7F1FA060006D03078222806D208203A
:106AB0000AB0BDE8F08143F20200F9E70421404644
:106AC00006F035FF07460DB1A88878B101208DF892
:106AD000140002208DF8180000248DF819403DB1F3
:106AE000A888ADF820002868079004E00920DFE7B7
:106AF000ADF82040079401F025FB050024D0A5F84F
:106B000002801721ADF80C10009404AB002240461F
:106B10000194FBF705FE0028CAD107F10800009593
:106B2000CDE9018096F8211003AA05A8049B03F083
:106B3000C8FD04466878000701D501F0E1FA4CB1C0
:106B40002046FFF7EEFAB3E713214046FDF7F9FCC4
:106B50000320ADE704980090BDF80C300422012119
:106B60004046FBF7A9FF4FF6FF71F980A0E72DE93A
:106B7000FF5F83460E9E9846914677888A46384640
:106B8000FCF781FA05460421384606F0D0FE04469B
:106B90000DB913F088FF0CB913F085FF0834CDE967
:106BA0000274CDE9008695F821104B4652465846AE
:106BB00003F026FA04B0BDE8F09F2DE9F04F9BB03A
:106BC0000D464FF000097449ADF82490ADF83490AB
:106BD000ADF83090A1F804900446ADF80C90ADF8F3
:106BE0001090ADF81890ADF8149008781646CB4682
:106BF000012808D0022806D0032804D0042802D097
:106C000008201BB088E6654884426AD3654F644A11
:106C10003968944201D38C4263D38046454560D3A2
:106C20009246554501D38D425BD3606878B14045AB
:106C300057D3504501D3884253D360892189884274
:106C400002D8B1F5007F01D90C20DAE7814608AA05
:106C500004A92846FFF700FB0028D2D16868807895
:106C6000C0F3410002280FD1BDF8100010F4405FBE
:106C70000AD0286940B1B0F5000F32D3B0F1805F7F
:106C800002D3396888422CD303A92069FFF79CFA04
:106C90000028B6D1206948B160788007BDF80C00A3
:106CA00000F4405001D5E8B300E0D8BBBDF80C00BB
:106CB000810618D510F4405F60680AD098B1B0F52D
:106CC000000F0ED3B0F1805F04D33968884208D337
:106CD00000E040B1404504D3504504D339688842B0
:106CE00001D210208DE705A96069FFF76DFA002831
:106CF00087D1606940B1BDF81400C0F3812101293A
:106D000037D110F4405F34D006A9A069FFF75CFAD0
:106D100000289AD1BDF8140080062AD4BDF81800C6
:106D2000810600E025E024D4A16931B1C0F38121BE
:106D300001291ED110F4405F1BD0E06818B1007823
:106D4000B8B11C2815D20EAA611C2046FFF7ABFA79
:106D500001278DF84E7042F60300DA46ADF84C007C
:106D60004FF4806B0DF13B0219A9286808F099FCDB
:106D700008B1072045E79DF8640014A9C01CCDF8B0
:106D800000A0CDE901A100F0FF08002308F20122D4
:106D9000594613A808E00000C402002000B001001A
:106DA000000000201C00002004F097F830BBBDF864
:106DB00050000B90FE482A8929690092CDE9011004
:106DC0006B89BDF820202868049904F086F801003A
:106DD0007ED1DFF8DCB35546ABF1040B0521BBF8DF
:106DE0000400ADF839000EA88DE8230043460022C8
:106DF000FF21BDF8500003F0D3FF10B1FFF75BF99E
:106E0000FFE69DF838004FF0020A01064FF480605B
:106E1000804622D501468DF84E704FF42450ADF8CF
:106E20004C00ADF81C5062789DF81C00002362F302
:106E300000008DF81C006278CDF800A0520862F3C3
:106E400041008DF81C0007AACDE9012540F203227C
:106E500013A804F042F801003AD1606840B32069F9
:106E600060B903A904A8FFF74FFA6078800705D43A
:106E7000BDF80C0020F44050ADF80C008DF84E70B9
:106E800042F60110ADF84C00208940F20121B0FB20
:106E9000F1F201FB120261680CABCDF80090CDE974
:106EA0000113002313A8039904F017F801000FD170
:106EB0002078C10601D480062CD5ADF81C5060693D
:106EC00068B905A904A8FFF71FFABDF8140000E08F
:106ED00077E020F4406000F58060ADF81400BDF864
:106EE00014008DF84E7040F0C800ADF8140042F662
:106EF0000210ADF84C000DA907AACDF800A0CDE90D
:106F00000121002340F2032213A8059903F0E5FFB5
:106F1000010056D12078C0072AD0ADF81C50A069D6
:106F200058B906A904A8FFF7EFF9BDF8180020F436
:106F3000406000F58060ADF81800BDF818008DF8CD
:106F40004E7040F04000ADF8180042F60310ADF866
:106F50004C0009A907AACDF800A0CDE90121002322
:106F600040F2032213A8069903F0B7FF010028D1CD
:106F7000E06850B38DF84E7042F60410ADF84C0046
:106F8000E0684146002302788DF85C2040788DF857
:106F90005D00E06807224088ADF85E00E068007997
:106FA0008DF86000E068C088ADF8610017A8CDE9F1
:106FB000002002954FF4027213A803F08EFF010027
:106FC00003D00B9800F02CFF1BE603218BF8001078
:106FD0005EB1BBF804003080BDF830007080BDF8B1
:106FE0003400B080BDF82400F080002009E670B5C0
:106FF00001258AB016460B46012802D0022814D17A
:1070000004E08DF80E504FF4205003E08DF80E5040
:1070100042F60100ADF80C0053B104AA08A91846C5
:107020004FF4806408F03DFB20B107200AB070BD2A
:107030001020FBE704A99DF820205D48CDE9002140
:10704000801E02900023214603A802F2012203F0D1
:1070500044FF10B1FFF72FF8E8E75548001F0EB1C5
:107060004188318005700020E0E770B594B0044697
:1070700001268DF83E6041F60100ADF83C0012AAF1
:107080000FA93046FFF7B3FF00284AD12078484CBB
:10709000C0074FF00005A4F1040444D01C2102A84D
:1070A00013F0CDFC9DF808008DF83E6040F0200004
:1070B0008DF8080042F60520ADF83C000E959DF8CD
:1070C0003A00119520F00600801C8DF83A009DF8DA
:1070D00038006A4620F0FF008DF838009DF839002E
:1070E00009A920F0FF008DF839000420ADF82C002C
:1070F000ADF830000EA80A9011A80D900FA80990C5
:10710000ADF82E5002A8FFF758FD002809D1BDF8B0
:107110000000E080BDF804002081401C60812570E3
:10712000002014B070BDE5802581BDF84800F4E76B
:107130002DE9F74F8B461E490026091F9EB00A789D
:10714000012A05D0022A03D0082021B0BDE8F08F23
:107150004A88824201D00620F7E789465A4501D184
:107160000720F2E701218DF866104FF0000842F683
:10717000020AADF84410ADF864A008F580624FF63D
:10718000FF710F92ADF84E10FF208DF86A801AAA99
:107190008DF84C00ADF84610ADF868801292CDF82D
:1071A000508011A803F07EFF00242546274601E009
:1071B000C80200200AAA052111A803F076FF78B1C1
:1071C000822856D1F4B3EDB3ADF85C409DF842008F
:1071D000ADF85E508DF80C8017AC01285DD064E0EE
:1071E0009DF82E00F7B1012852D1BDF82C10514561
:1071F0001AD116AA06A905208DE80700BDF82A00B5
:1072000010230022FF2103F0BAFF90BBBDF8580005
:10721000042801D0062846D1BDF81810594537D1A9
:107220000F2092E7012833D1BDF82C00B0F5205F84
:1072300003D042F6010188422AD1B9F80210BDF804
:107240002A0000E027E0814201D1012700E0002769
:1072500004B17DB158451BD116AB06AA05218DE8B6
:107260000E00044610230022FF2103F088FF00B91E
:1072700002E02DE035460BE0BDF85800022801D0B1
:10728000102810D1C0B210AA06A908F0EBF950B925
:10729000BDF82A608BE7052057E703A910A8221D37
:1072A00008F0FFF908B103204FE79DF80C00002318
:1072B000001DC2B220988DF80C200092CDE901404B
:1072C00019A80F9903F009FE10B9022289F80020CD
:1072D000FEF7F1FE39E710B50B46401E86B084B2CA
:1072E00003AA00211846FEF7DEFF04AA052103A821
:1072F0008DE8070001230022FF21204603F050FD06
:107300000446BDF81000012801D013F0CCFB204644
:10731000FEF7D1FE06B010BDF0B587B00E460446AC
:10732000FE4F3878032804D0042802D0082007B084
:10733000F0BD04AA03A92046FEF78EFF0500F6D192
:1073400060688078C0F34100022812D1BDF80C00BB
:1073500010F4405F0DD0206958B1B0F5000F06D38E
:10736000B0F1805F05D3EE490968884201D2102050
:10737000DDE7208905AA21698DE807006389BDF84A
:1073800010202068039903F0A8FD10B1FEF793FECA
:10739000CDE716B1BDF814003080042038702846BF
:1073A000C5E738B50C00054609D000236A46FF2121
:1073B00003F051FF28B100BFFEF77DFE38BD10205D
:1073C00038BD69462046FEF7FFFE0028F8D1A078B8
:1073D000FF2100F001032846009A03F065FFEBE768
:1073E0001FB50C0009D06B4601AA002103F033FF42
:1073F00028B1FEF760FE04B010BD1020FBE70020AE
:107400002080A070BDF8040002A9C0F38120FEF71F
:10741000B4FE50B99DF808002070BDF8040002A920
:10742000C0F30130FEF7A9FE08B10320E3E79DF8A1
:1074300008006070BDF80410A078CA0B62F3041055
:107440008A0B62F3C300A070890601D5022100E017
:10745000012161F342009DF8001061F30000A0706B
:107460000020C8E77FB5144603AA05250292CDE99E
:1074700000350A462388FF2103F092FCBDF80C106A
:107480002180FEF718FE04B070BD2DE9F04393B0E3
:107490004FF000060C008146ADF80C60354619D05F
:1074A000E06828B1A068A8B10188ADF80C1006808A
:1074B0004846FBF7E8FD88B10078222870D348469B
:1074C00000F0ACFC80460421484606F030FA070084
:1074D00009D106E0102013B0BDE8F08343F20200AA
:1074E000F9E713F0E0FAA078012803D0022801D0D0
:1074F0000720F0E7208838B1401E80B204AA414638
:1075000003F0A1FDA8BB3CE043F20300E3E700BFAA
:10751000BDF81610228891420DD29DF81A004FF046
:10752000000501282FD1BDF81800A0F5205103391E
:1075300029D1012527E002D185B36D1C02E001D9D4
:10754000022D02D0032D1ED322E09DF81A1001292E
:1075500019D1BDF8181042F602028B1A91421DD0C3
:1075600008DCB1F5205F19D06FF42050C1420AD178
:1075700014E025E0012B11D0B3F5807F03D1032562
:1075800006E04FF4505804A803F065FD0028BFD072
:10759000822801D0A0B904E0022D11D140469AE71B
:1075A0002BE0E06898B1052203A9CDE90002029121
:1075B000A2882088BDF80C30FF2103F0F1FB10B148
:1075C000FEF779FD87E7A168BDF80C000880BDF8DB
:1075D0001400C00602D543F201407CE7089818B1B8
:1075E000BDF81C00022801D0032074E70898A17898
:1075F0000078012903D080070FD408206BE7C0076B
:10760000FBD0002207214846FBF794FB10B1072569
:10761000022004E043F204005DE7022503208DF818
:10762000300020881721ADF83400ADF82C100096FA
:107630000AAB002248460196FBF772F80028AED14B
:10764000CDE90069083702970BAA05210CA80A9B0F
:1076500003F037F810B1FEF764FD3CE70A9800909C
:10766000BDF82C30042229464846FBF725FA32E7BC
:1076700070B5064615460C460846FEF7D7FC0028AE
:1076800005D12A4621463046BDE87040AFE470BDC2
:107690004EE570B51E4614460D0013D094B16168D6
:1076A00081B10121FEF7E4FE00280CD12068FEF72D
:1076B000BDFC002807D1324621462846BDE870406F
:1076C000FFF77BBA102070BD70B515460C000ED0C8
:1076D0000221FEF7CDFE00280AD12068FEF7A6FCA5
:1076E000002805D129462046BDE8704014E6102048
:1076F00070BDF8B514460E460546B2F5000F3ED3F0
:107700000748B4F1805F016801D38C4237D36068C9
:1077100080B1044A904232D3034A07E0C4020020F9
:107720001C00002000B0010000000020904201D3A6
:10773000884224D3A5F57F40FF3803D02846FBF7C5
:10774000A2FC58B1284600F069FB0546304600F01F
:107750000FFB002804D1606818B112E043F2020068
:10776000F8BD00236A462946304603F074FD10B187
:10777000FEF7A1FCF8BDBDF80000800601D4102082
:10778000F8BD6188224630466368FFF76BFEF8BD9E
:107790002DE9F74F4FF4000986B0144607464A45D5
:1077A00007D34FF0805AFC4E544505D330688442CD
:1077B00002D2102009B0C9E4384600F02FFB4FF682
:1077C000FF7B05465F4501D0FF2D0AD0002304AAA8
:1077D0002946079803F03FFD30B100BFFEF76BFC70
:1077E000E8E743F20200E5E7BDF81000C00602D565
:1077F00043F20140DEE74FF0050803A90027CDF86A
:107800000080CDE9017162885B462946079803F044
:10781000B6FC010015D1606848450FD3504502D32E
:10782000326890420AD3CDF80080CDE90107238861
:1078300062882946079803F0A2FC0146BDF80C00B7
:1078400020800846CAE739B1D44B0A881B899A427E
:1078500002D843F20300704717E610B586B0CF4C4C
:107860000423ADF81430E3883BB124898C4201D263
:10787000914204D943F203004CE506204AE5ADF8F5
:107880001010002100910191ADF8003002218DF817
:10789000021005A9029104A90391ADF812206946CE
:1078A000FFF7F3FD36E52DE9FE4F82468120BC4F00
:1078B0000C468DF80800B94246D3DFF8E882DFF8BD
:1078C000D892444503D3D9F8000084423CD35046B3
:1078D000FBF7D9FB06000FD03078222836D30022E0
:1078E00001215046FBF726FA50B10421504606F01C
:1078F0001EF8050008D105E043F20200BDE8FE8F46
:107900001120FBE713F0CFF805F1080002F05EFB51
:107910002178012903D0022904D00720EEE782074D
:1079200014D502E010F0340F10D0241DA278D20735
:107930000ED0E28862B1A268BA4205D3424507D3AD
:10794000D9F800309A4203D21020D7E70820D5E7B3
:10795000228802AB00F0DBF90028CFD19DF8081097
:1079600096F82100CDE900016A8823462946504651
:10797000FEF790FDC2E72DE9FF4F89B01E46154680
:107980000C464FF000090F460998FBF77CFB30B11D
:107990000078222806D208200DB0BDE8F08F43F20F
:1079A0000200F9E7B00801D00720F5E7032E00D167
:1079B0000026099800F032FA83464FF6FF7A34B376
:1079C000022D78D37648844214D3764A724B94427F
:1079D00002D319688C420DD304EB0508B8F1010FEE
:1079E0000AD0A8F10101814204D3914204D318685E
:1079F000814201D21020CFE7AD1EAAB221465046E7
:107A000003F030FD38F8021C884254D1ADB263480F
:107A1000B10702D50189491C00E001211FFA81F854
:107A2000F10701D0068900E0564603AA59464046B0
:107A300003F009FB4FF0050A0BE0788810283AD8CC
:107A400009F1040108441FFA80F9A94533D804EB71
:107A5000090757B339884145EFD349E0BDF8101005
:107A60000A0745D57CB304EB090709F104027B88BA
:107A70001FFA82F8102B1ED803EB0802AA421AD86C
:107A80003A88904217D1C80617D504EB0801CDE912
:107A9000001A08AA029238880022594603F080F999
:107AA00020B1FEF708FB77E705E021E07888BDF814
:107AB0002010884201D00B206EE7798801EB080086
:107AC0001FFA80F907E0FFE7C90604D55946FEF71B
:107AD0003DFD00288FD1BDF81000FF2320F01000DD
:107AE000ADF81000BDF812005946049A03F0DCFB13
:107AF00003A803F0B0FA18B9BDF81200B042ADD92E
:107B00000421099805F013FF040001D112F0CBFF06
:107B100022885AB10025CDE900A52B4621460998B7
:107B2000FEF7B8FC0028BED1258035E7002033E7FA
:107B30002DE9F04F89B01E4617000D464FF00004A6
:107B400027D0B10801D0072034E6032E00D100264B
:107B500000F064F98046FF2826D0E5B14FF400021A
:107B6000954216D353010C499D4202D308688542C1
:107B70000FD3388800EB050CBCF1010F17D0A5F12D
:107B8000010C6044904204D3984210D309688842A3
:107B90000DD210200EE60AE01C000020C4020020D6
:107BA00000B001000000002043F2020002E6A249FA
:107BB000B00701D5488900E00120F2074FF6FF79B0
:107BC00002D04989491E00E049468EB204AA4146C6
:107BD00003F039FA0DF10C0B4FF0050A34E000BF49
:107BE000BDF8141009072FD50023CDE900A3CDF867
:107BF00008B04B460022414603F0C1FAE8B9F5B19E
:107C0000BDF80C103A8821442819091D8A422ED348
:107C1000BDF8162020F8022BBDF80C2020F8022B0E
:107C2000CDE900A0CDF808B0BDF81600BDF80C30C5
:107C30000022414603F0A3FA08B10320BAE5BDF8DB
:107C40000C002044001D84B204A803F004FA20B103
:107C5000822806D0FEF72FFAACE5BDF81600B04238
:107C6000BED934B175B13988A01C814203D20C2031
:107C7000A0E505209EE522462946484603F0F2FB92
:107C800029190880A41C3C80002093E5B0F5000F62
:107C900006D3B0F1805F05D368490968884201D2F4
:107CA00010207047644949890180002070472DE900
:107CB000F0411446804651EA040013D04FF4000608
:107CC0005E4D770189B1B14217D3B94202D328681A
:107CD000814212D3404603F019FB30B1BDE8F041B8
:107CE000FEF7E9B90720BDE8F08174B1B44204D3CE
:107CF000BC4204D32868844201D21020F3E7214615
:107D00004046BDE8F041FFF76BBB0020EBE770B5E4
:107D10008AB1A2F201168124D5B2112E1AD224D230
:107D2000DFE806F0230C0F23202314201223232046
:107D30002020202320000020187014E0022914D0F5
:107D400010E0012911D00DE0C00600E080060028F7
:107D50000BDA07E0A2F5C0701F2803D9A2F2FD12CA
:107D6000022A02D81D70002070BD1C70072070BD53
:107D700000B585B06946FEF7EBFA00280AD19DF8F8
:107D80001000082832D2DFE800F0042F2F2F2F0731
:107D90000704032005B000BD9DF80200012808D1AA
:107DA000BDF80000B0F5C05F1ED06FF4C051C842EE
:107DB0001AD09DF80600012805D1BDF80400A0F5F1
:107DC0002850052810D99DF80A00012810D1BDF8C7
:107DD0000800B0F5245F07D0A0F52450023803D086
:107DE000012801D0022803D10F20D3E712F05BFE57
:107DF0000020CFE770B50C4605461A21204612F048
:107E0000FCFD0020208035B1012D02D012F04BFE88
:107E100070BD062000E00520A07070BD05F050BDCB
:107E200010B50C4603F0DEF808B112F03CFE204617
:107E3000BDE81040FEF73FB9C40200201C0000203E
:107E40007CB50A460546694605F0B0F904460AE0E5
:107E5000002201A9284605F0A9F904469DF804006E
:107E600008B112F020FE2CB19DF80000411E8DF8E3
:107E70000010EDD220467CBD2DE9FF4F9FB0FB499D
:107E8000DDE92C9A06000396D1E90001CDE909014C
:107E9000507A117A9B4608441546C7B20ED000248A
:107EA000F01C20F00300B04201D012F0FCFD288845
:107EB0000399401C1FFA80F814B108E00124EFE791
:107EC00008F0FF0007F072FB08B112F0ECFD039917
:107ED0003A4601EB0810C01C20F00301D5F81080D1
:107EE000039144B9002008701FFA88F002F01FFFC8
:107EF00008B112F0D8FD0399234601EB0800039066
:107F0000A87A297A3A460844C1B203A800F04FFD86
:107F10000398C01C20F003000390697A00912B7A2B
:107F2000AA7A04B1002002A905F0CDFB08B112F035
:107F3000BAFDBDF8081003983A4608442E99C01CB3
:107F400020F00300CDE90210CDE9009A04B1002031
:107F50005B4606A905F076FD08B112F0A4FDBDF858
:107F6000181003980844C01D20F00700811B0390DF
:107F70002098002C016045D101222C21BC4805F03D
:107F800039FBFBF70AF8BB4C6178A06803F0F5FBFE
:107F9000E068401E07280BD830218DF82C108DF892
:107FA0002E000BA804F08BFE10B114A803F0AAFC5D
:107FB00000211E22084601F07DFAFBF7E7FFFAF7E1
:107FC000F8FCFEF714FD09AB00220521AAA0F9F781
:107FD00060FB08B112F067FD05F10C00FFF745F8F2
:107FE00008B112F060FD4FF47F71A54812F027FD33
:107FF000A348012180F8F913022180F8FA13062121
:1080000080F8FB1323B0BDE8F08F10B59C4CA0782E
:10801000092801D312F047FD2078C0EBC00004EB23
:10802000001010F8041F21F0FF010170417821F0C9
:108030000701C91C21F0180141700121E17010BD38
:108040002DE9F0474FF0000914460D46A3F80090C3
:10805000072851D2DFE800F050040B19125020001D
:1080600021462846BDE8F0471A46FAF7F5BC2146F6
:108070002846BDE8F0471A46FBF707BC21462846CC
:10808000BDE8F0471A46FEF774BB21462846BDE816
:10809000F0471A46F9F7F1BF28784FF0000806219B
:1080A0001F464646B1EB101F01D012F0FCFC287EA3
:1080B00058B1012811D012F0F6FC3E8014B1A4F89A
:1080C000008066804846BDE8F0874FF00208092628
:1080D00084B1A88BA080A87F0AE04FF00308142683
:1080E00044B16888A080286AE060A88C2082287F3C
:1080F0002072E2E73E80E5E712F0D5FC0320E2E7DC
:1081000070B55F4CE07800281BD020780025C0EBCC
:10811000C00004EB0010407900F00700011991F84D
:10812000F803401E81F8F8032078401CC0B220708C
:10813000092800D12570A078401CA07009F04EF8E5
:10814000E57070BD4E4890F8FB03002800D05CE756
:1081500070472DE9F8434A4D5FF00006D5F8F40367
:1081600068B1FFF7EFFF002876D07022D5F8F4133E
:1081700012F011FCFFF7C4FFC5F8F463EEE795F8C1
:10818000F903002868D0FFF740FF0446384805F09F
:1081900043FA606008B912F086FC606803F036F9B3
:1081A00088B12046FBF731FA6078010706D520F048
:1081B0000700401C6070FFF7A3FFCFE72C48616801
:1081C00005F033FACAE72A48616805F02EFA6846D6
:1081D00000F028FC00286AD10321BDF8000005F05A
:1081E000A6FB8046BDF8000005F042FD0746B8F149
:1081F000000F01D112F057FCD8F8040010B100783C
:10820000FF2854D0FFF701FF0446001D81460146B8
:10821000384605F053F918B1D9F80000067001E0AE
:1082200012F041FCA08A08B112F03DFCD4F8049091
:1082300089F80060BDF8000060802046FAF754FC21
:10824000384605F06CF908B912F02DFC607801078A
:1082500003D4C00607D415E029E020F00700801CF5
:108260006070FFF74DFFC8F8049077E790AC01000D
:1082700020070020180000206E52463578000000CC
:1082800024030020D8F8040040B10178491C11F003
:10829000FF01017091D112F006FC5FE70021384622
:1082A000FFF7CEFD002888D112F0FDFB56E7BDE8B0
:1082B000F88310B5FE4CC4E90201AFF2691001F079
:1082C0008EF8607010BDFA4900200870704730B514
:1082D00005464FF080500C46D0F8A41095B0491CCC
:1082E00005D1D0F8A810C9430904090C08D050F8EA
:1082F000A01F01F0010129704168216080680FE032
:108300002B208DF8000009A9684603F05BF808B13E
:1083100012F0C9FB012028700A982060BDF82C00DB
:10832000A0802878002803D0607940F0C0006071F8
:1083300015B030BDF0B54FF080540746D4F880003A
:1083400095B00D462B26401C0BD1D4F88400401C60
:1083500007D1D4F88800401C03D1D4F88C00401C0D
:108360000BD0D4F880003860D4F884007860D4F85A
:108370008800B860D4F88C0018E08DF82C6069464D
:108380000BA803F01FF808B112F08DFB01983860BC
:10839000029878608DF82C6069460BA803F012F8FB
:1083A00008B112F080FB0198B8600298F860D4F828
:1083B0009000401C0BD1D4F89400401C07D1D4F895
:1083C0009800401C03D1D4F89C00401C08D054F8FD
:1083D000900F286060686860A068A860E06818E096
:1083E0008DF8006009A9684602F0ECFF08B112F0B0
:1083F0005AFB0A9828600B9868608DF8006009A9FC
:10840000684602F0DFFF08B112F04DFB0A98A86041
:108410000B98E86015B0F0BD30B5A64C0546D4F811
:10842000F40308B112F03FFBC4F8F45330BD38B583
:108430000546032105F07BFA0446284605F018FCA2
:1084400005460CB912F02FFB606820B10078FF28B8
:1084500001D112F028FB69462846FFF7F1FC08B964
:1084600012F021FB60680099884201D10020606011
:10847000904C94F8FA03022801D312F014FB94F8FC
:10848000FA03401CC0B284F8FA03012803D18848DB
:10849000407800F0C4FF38BD70B50446A1F57F40B8
:1084A00016460D46FF3801D112F0FDFA012E02D01A
:1084B00012F0F9FA70BD207820F00F00801D20F036
:1084C000F0006030207000202076A5830120A07786
:1084D00070BD70B515460C460646FFF733FE90B1E9
:1084E000017821F00F01891D21F0F0016031017048
:1084F00046800121017621680162A1888184057787
:10850000BDE87040FCE53046BDE870401321FCF743
:1085100018B870B50C460546B1F5000F06D3B4F196
:10852000805F05D362484068844201D2102070BD4C
:108530002846FAF7A8FD28B1284605F0ACFB05004F
:1085400005D102E043F2020070BD12F0ACFA2846F9
:10855000FAF742FD2221B0FBF1F0C0B2062801D9A2
:10856000801F00E000202070002070BD2DE9F04F3A
:108570000D464F49044685B0087810B1082005B073
:1085800041E54B494C4848604FF400018C420AD306
:108590004A01944201D3844205D38D4203D39542CC
:1085A00003D3854201D21020E9E7617A227A8B1841
:1085B000FF2B2BD82088FE2828D8082B01D904208F
:1085C000DDE700B90A202080206908B94FF4B060C7
:1085D00002EB820601EB810306EBC20606EB4306C3
:1085E00001EB410302EB420703EB470707EBC7032D
:1085F00003EB430A06EBC60303EB43082061D828CC
:1086000001D20920BBE7A07A884201D90720B6E74A
:10861000606800F0A0F95FEA0009B0D11FFA88FB9A
:108620000097CDE901B61FFA8AF3224603A9FFF7A6
:1086300023FCDFF87C8003992A68D8F80400014401
:10864000914202D90C20296099E70097CDE901B643
:108650001FFA8AF3224604A9FFF70EFCDDE90301A5
:10866000884201D012F01FFA0498D8F80410084488
:10867000C8F804002860012088F8000048467EE71A
:108680002DE9F05F0F464FF4000104468F421BD3E3
:10869000DFF81CB04A019742DBF8040001D387429F
:1086A00012D364B18C420FD3944208D3844205E0C4
:1086B0001800002024030020F010002004D3E01C48
:1086C00020F00300A04202D01020BDE8F09FFB483C
:1086D0004FF00008817899B141788246C1EBC10121
:1086E00000EB0115B7F8009015F8040F3B4600F0B9
:1086F0000F0000222946FFF7A3FC060004D013E078
:10870000A7F800800520E0E794B13988494501D9F0
:108710000C260DE028783B4600F00F002246294643
:10872000FFF78EFC060005D00C2E01D0A7F80080C4
:108730003046CAE79AF801005446401CC0B28AF895
:108740000100092801D184F80180A078401EA070A2
:10875000687800F0070101290CD0022904D0032910
:1087600019D012F0A0F9E3E7C006E1D46888FFF75A
:108770005EFEDDE7D248696804F057FF94F8F9031C
:10878000401CC0B284F8F9030128D1D19BF8010044
:1087900000F045FECCE794F8FB03401C8AF8FB038D
:1087A000C6E7C84A30B490420ED3C84AC64C526895
:1087B000A04201D3904207D3B1F5000F04D3B1F129
:1087C000805F04D3914202D2102030BC704730BC8D
:1087D00006F023BFBB4B10B599420ED3BB4BBA4C2E
:1087E0005B68A14201D3994207D3B2F5000F04D3CD
:1087F000B2F1805F03D39A4201D2102010BD02284B
:1088000003D0102801D0092010BD06F02BFF00284E
:10881000FAD0052010BD70B5AA4B984216D3AB4BC9
:10882000A94C5B68A04201D398420FD34FF40004D7
:10883000A1420BD36501A94201D3994206D33AB1B3
:10884000A24203D3AA4203D39A4201D2102070BDA0
:1088500006F027FF0028FAD0072070BD10B594B0AD
:108860000446B0F5000F06D3B4F1805F06D39748F5
:108870004068844202D2102014B010BD0F208DF841
:10888000000009A9684602F09DFD0028F4D19DF87A
:108890002C002070BDF82E006080BDF83000A08054
:1088A0000020E9E730B4A9B14FF40004A1420DD390
:1088B000864A6501A942536801D3994206D30A68E2
:1088C000A24203D3AA4203D39A4201D210207CE7EA
:1088D0008A8812B130BCFEF7DEB8092075E7794A04
:1088E000914206D3784A914205D3784A5268914220
:1088F00001D210207047421E1E2A01D800F0CFB8C6
:10890000A0F120021F2A01D8FBF76CBA072070479C
:10891000B1F5000F11D36D4AB1F1805F526801D3F8
:1089200091420AD3431E1E2B0FD8664B994204D3A3
:10893000654B994203D3914201D210207047012820
:1089400001D10620704707207047A0F120021F2A9E
:10895000F9D8FBF7C3BAF0B500280AD0594B9842B2
:1089600006D3594B984205D3584B5B68984201D2C5
:108970001020F0BD83784678057833442B448C185A
:108980009C4206D147790379C0781F440744BC4212
:1089900001D00720F0BD954205D1904203D18E420F
:1089A00001D18B4201D00620F0BD0020F0BD2DE9A1
:1089B000F0410646022012B101EB4200401DC7B251
:1089C0003068C01C20F0030232602BBB3B483B46A2
:1089D0000A21283808F04BFF002408E00A2C11D2A5
:1089E000DFE804F005070509090B0B050505384804
:1089F00004E0384802E0384800E0384808F058FF02
:108A0000054601E012F04FF8A54201D012F04BF8F4
:108A1000641CE4B20A2CE1D3306800EB071030602C
:108A2000BDE8F0812DE9F04194B080463A208DF800
:108A30002C0069460BA802F0C5FC08B112F033F80F
:108A400043F2040600246D4622E02F19B87DC107C9
:108A500006D0400704D405EB4400C088FAF752F969
:108A6000164890F8FA0388B1B87D80070ED505EB5B
:108A700044000022C0880621FAF75CF930B105EB0A
:108A800044000026C188A8F8001005E0641CE4B288
:108A90009DF80400A042D8D8304614B0C0E700B515
:108AA000084A95B0914206D3074A914218D3074A23
:108AB0005268914214D2102015B000BD240300204A
:108AC0002007002000B00100000000201800002056
:108AD000033C00001F2A0000852F0000D5F4000091
:108AE000012802D0022810D123E00A78022A04D0FB
:108AF000012A02D043F20500DEE7487828B10328B6
:108B000003D8897809B1032901D90720D4E7022ABB
:108B100002D0012A09D104E0022806D1022904D199
:108B200005E0032801D1032901D00620C4E7002075
:108B3000C2E7087800F001008DF80200487800F0E4
:108B400001008DF803000878C0F340008DF80400A0
:108B50004878C0F340008DF80500087880088DF84B
:108B60000600487880088DF8070088788DF808009E
:108B7000C8788DF8090008798DF80A003E208DF834
:108B8000000009A9684602F01DFC95E730B44FF0DB
:108B9000E02001234FF4006C0021C0F880C11D02C9
:108BA000C0F880511C06C0F88041DD4A82F80014EC
:108BB000D21E82F80014DB4A82F80014DA4A5360AD
:108BC0009360C2F84011C2F84411C2F84811C0F8CD
:108BD00080C2C0F88052C0F88042C0F800C1C0F81E
:108BE0000041136030BC704770B401204FF0E023A7
:108BF000C6024FF0000CC3F880610402C3F8804144
:108C00000506C3F88051C84A50609060C7480168A3
:108C10000029FCD1C2F840C1C2F844C1C2F848C121
:108C2000C3F88062C3F88042C3F8805270BC7047BA
:108C30004FF0E0204FF40061C0F88012C910C0F876
:108C400080127047002804BFB9487047012804BF4C
:108C5000B8487047022804BFB748704700B511F004
:108C600022FF002000BD08B5AF49002230B1012825
:108C700022D002282ED011F016FF08BD4FF480300C
:108C8000C1F80803C1F84803AC4B1A60C1F8402191
:108C9000AB4BC1031960AB49C1F808034FF0E023A7
:108CA0000012C3F88001A8480260C1F84021C1F851
:108CB0000022A648027008BD4FF40030C1F8080336
:108CC000C1F84803A2480260C1F8442199480068ED
:108CD000009008BD4FF48020C1F80803C1F8480394
:108CE0009C480260C1F8482193480068009008BD84
:108CF00070B5DFF834C204260025012430B1012804
:108D00003CD0022852D011F0CEFE70BD881E20F05B
:108D10007F414FF48030CCF80803CCF84051CCF8B8
:108D20004403CCF84015012B14BF00210121874BCF
:108D3000597084494C60CC60DFF81CC2CCF80050FC
:108D4000864D4FF0020CC5F800C0DFF814C2CCF815
:108D50000060DFF8F4C13D32CCF80020C1F80042D9
:108D60004FF0E02C8A15CCF88022C1F80403CCF82F
:108D7000002108047B4908601C7070BD7A484FF4DC
:108D80000032012B09D100BFC0F84051CCF80423B8
:108D9000CCF84423C0F8401570BDCCF80823C0F8C7
:108DA0004051CCF84423C0F8401570BD6F484FF4D3
:108DB0008022012BF1D1E7E75C480068704770B56D
:108DC000594CD4F84001002501280AD1D4F80803F1
:108DD00010F4803F05D04FF48030C4F80803C4F885
:108DE0004051D4F8440101280DD1D4F8080310F4FF
:108DF000003F08D04FF40030C4F80803C4F84451D1
:108E0000012007F0EEFCD4F84801012818BF70BD1E
:108E1000D4F8080310F4802F08BF70BD4FF48020F1
:108E2000C4F80803C4F84851BDE87040022007F0B8
:108E3000D8BC46490878E0B1414A4FF00040106084
:108E4000404AC00BC2F8080303124FF0E02C002088
:108E5000CCF880313C4B1860C2F84001C2F80002E7
:108E600008704A78002A08BF70474870002007F051
:108E7000B8BC032007F0B5BC4FF0E0214FF0807084
:108E8000C1F8000270474FF0E0214FF08070C1F848
:108E9000800270474FF0E0214FF40010C1F800024B
:108EA00070474FF0E0214FF40010C1F88002704786
:108EB000244801214160C1604FF0E0218015C1F8D4
:108EC00080027047410A43F609525143C0F308003B
:108ED00010FB02F000F5807001EB50207047430B4F
:108EE00048F2376C03FB0CF31B0C4FEA432CC1F820
:108EF00000C0DFF87CC003FB0C031E484CF2F72CCB
:108F00005843400D10FB0CFC0CEB432303F580731E
:108F10005B1213700A6810440860704707F052BD76
:108F20000BE000E018E000E000B0004004B50040B5
:108F30004081004044B1004048B1004040B500408D
:108F400008F50140008000404085004028000020D6
:108F500044B5004048B50040048500400885004005
:108F60001085004004F5014004B0004008B0004006
:108F7000F7C2FFFF6F0C010010B5EFF3108000F097
:108F8000010472B6CB484178491C417040780128F1
:108F900001D108F043F9002C00D162B610BD70B5C4
:108FA000C44CE07848B90125E570FFF7E5FF08F00B
:108FB0003DF920B1002008F018F9002070BD4FF0F5
:108FC0008040A571C0F80453F7E770B5EFF3108047
:108FD00000F0010572B6B74C607808B911F063FD76
:108FE0006078401E6070607808B908F01BF9002DA9
:108FF00000D162B670BDAF4810B5C17821B1002173
:109000008171C170FFF7E1FF002010BD10B504466B
:1090100008F00CF9A749C978084000D00120206069
:10902000002010BD2DE9F05F0026A24C082104228B
:10903000102320270125B046E6714FF0020A0D28C3
:109040002CD2DFE800F007090C0E101214161F21B5
:1090500024262800657123E084F805A020E06271D1
:109060001EE061711CE063711AE0677118E001266F
:1090700016E0FFF781FF00BF08F0D8F80028FBD00A
:1090800002260DE0627100E06171E57108E0637134
:10909000FBE76771F9E740206071F6E711F003FD27
:1090A00008F0D1F848B108F0D5F8B04205D1304603
:1090B00008F0D4F80028FAD032E04FF08047FD6085
:1090C000C7F804817C490E60C7F804A3BD60C7F8E7
:1090D0001081DFF8E8B1DBF80010C94341F300115B
:1090E00001F10109DBF8001041F01001CBF800108C
:1090F00000E020BFD7F804010028FAD0304608F07D
:10910000ADF80028FAD0B9F1000F05D1DBF8001056
:1091100021F01001CBF80010C7F808A3C7F80481AC
:10912000E07960B108F082F8074608F065FA6FF060
:10913000004117B1C4E9021001E0C4E902011EB107
:1091400084F80480BDE8F09F2571BDE8F05F00F071
:109150008FB810B5044608F06FF828B155490120C2
:10916000C8704A78521C4A702046BDE8104059E742
:109170002DE9F0414FF08045D5F80801002601287F
:1091800003D1C5F8086108F030F8D5F804010128CA
:1091900001D1C5F80461D5F800010127454C01282B
:1091A0000ED1C5F80061A07918B1002008F01DF8B3
:1091B000A671207820B108F039F808B12F61A770A6
:1091C000207930B3D5F81001012824D1C5F81061F9
:1091D0006F61E079B0B108F029F8804608F00CFA28
:1091E000B8F1000F01D0E16800E0A168411A02293E
:1091F00002DA11F1020F0EDCB8F1000F01D0E060CD
:1092000000E0A060FFF7B8FE08F010F810B12F6181
:10921000A77000E02770D5F80C0101280AD1A078CA
:1092200008B911F040FCC5F80C61A6702670BDE8C5
:10923000F041CAE6BDE8F08170B51E4DE87808B986
:1092400007F0F0FF01208407A061A87858B100BFA3
:10925000D4F80C0120B9002008F000F80028F7D15C
:109260000020C4F80C014FF0FF30C4F8080370BDB3
:109270002DE9F0411927BC07C4F808734FF0000826
:10928000C4F80081C4F80C8107F0D0FF094E012515
:1092900010B12561B57000E03570FFF76DFEC4F8C0
:1092A00004730549707920310860A561C4F8108104
:1092B0006561BFE72C0000201805004010ED00E0BC
:1092C00010B50D2000F069F8C4B26FF0040000F092
:1092D00064F8C0B2844201D011F0E5FB36490120A8
:1092E000086010BD70B50D2000F041F8334C00202F
:1092F000C4F800010125C4F804530D2000F042F821
:1093000025604FF0E0216014C1F8000170BD10B578
:109310000D2000F02CF82948012141600021C0F8FF
:109320000011BDE810400D2000F02CB8234910B505
:10933000D1F80001012802D011F0B5FB10BD1E4884
:10934000001D00680022C0B2C1F80021BDE8104035
:1093500008F077B810B51948D0F800110029FBD0F3
:10936000FFF7E4FFBDE810400D2000F00BB800F05F
:109370001F02012191404009800000F1E020C0F867
:109380008011704700F01F020121914040098000C8
:1093900000F1E020C0F880127047002806DA00F0E3
:1093A0000F0000F1E02090F8140D03E000F1E02040
:1093B00090F800044009704704D5004000D00040F8
:1093C0004FF0E0214FF00070C1F88001C1F8800239
:1093D000354B402283F80024C1F80001704700B5E6
:1093E00002460420314903E001EBC0031B7933B18D
:1093F000401EC0B2F8D211F056FBFF2000BD41F86C
:10940000302001EBC00100224A718A7101220A71E9
:1094100000BD264A002102EBC0000171704710B563
:109420000446042801D311F03EFB204800EBC4049D
:109430002079012801D011F036FB6079A179401C18
:10944000C0B2814200D060714FF0E0214FF0007057
:10945000C1F8000210BD70B51348042590F800044F
:10946000124E4009124C022819D011F01CFB16E0D4
:10947000217806EBC1000279012A08D1427983796B
:109480009A4204D04279827156F8310080472078A0
:10949000401CC0B22070042801D3002020706D1E33
:1094A000EDB2E5D270BD000019E000E060070020D9
:1094B0003C000020F84B586019721A80C90011F066
:1094C000BEBA0021018070474FF6FF720280032070
:1094D00008F09DBA70472DE9F04F0E46017804461A
:1094E0004FF0010A0AFA01F047F2FF1100EA010801
:1094F0006168154697B00888A0F57F42FF3A06D00C
:10950000B8F1000F07D047F2FE12104203D001203D
:1095100017B0BDE8F08F40EA080008804FF000095E
:10952000A5B185F8009023780027052003220221A9
:10953000DFF864B3102B75D2DFE803F0740D131C51
:109540002F4A515A31A5A175A9F1F0EF20780B28C7
:10955000E9D00420DCE72970A089A5F80100328059
:109560001DE104212970A189A5F80110E189A5F860
:10957000031082E006202870A089A5F80100E08988
:10958000A5F80300208AA5F80500A28AE81DA169B4
:1095900011F0BCF9A08AC01D6FE008212970217864
:1095A000082901D110212970A189A5F80110E189AC
:1095B000A5F8031030806A1D694604F1100006F01A
:1095C00070F800287ED130889DF80010084454E0DF
:1095D0000A202870A089A5F801003280AAE00C2199
:1095E0002970A189A5F80110E189A5F80310B7E059
:1095F000A2890AEB420081B23088884262D30529F1
:1096000060D30E202870002008E0236905EB400C91
:1096100033F81030401CACF8013080B29042F4D3E3
:109620003180BCE0CAE09BF809005A46002873D09C
:10963000401E5072227BDBF80400236900EBC20558
:10964000AA882868D3F800C00244A2F1080042F8B2
:1096500008CC5A6842608DF800108DF80190286897
:109660000290A888ADF8040000216846F8F78FFC46
:10967000A5F80490002E01D0484630808FE028786D
:1096800040F080012970287840F040012970287846
:1096900020F03F0012302870A189A5F80110E2895E
:1096A000E81C216911F032F9E089C01C308028786B
:1096B00041063FD5000672D58DF800A08DF80190C7
:1096C000308800E026E0001DADF804000295E18935
:1096D000E81C08440390001D04909BF808008DF8D6
:1096E000140000216846F8F752FC074630880C3019
:1096F0003080022F01D007B363E09DF81420DBF81F
:1097000004109BF80830584601EBC2019A4201D27E
:109710008A882AB1042754E030E02BE022E00DE0F3
:10972000427A521C8BF809200D6030888880A6F898
:10973000009046E06168A089888030E0287820F0B9
:109740003F0016302870A089A5F80100E089A5F82F
:109750000300228A681D616911F0D8F8208A401D33
:109760003080E7E7287820F03F0018302870207B11
:10977000687055E760680188090401D4052720E076
:10978000C088A189884201D006271AE01E202870CF
:10979000A6F800A06068018821F400410180B8F1BA
:1097A000000F0ED0BBF80000002283000320A16848
:1097B00008F08FF861682078887007E0A6F80090BC
:1097C00003276068018821EA0801018038469FE686
:1097D0002DE9FF4F97B00C46249E70B117280CD886
:1097E0003288A2F57F43FF3B07D02278530601D48D
:1097F000120604D508201BB08BE60720FBE74FF0CC
:1098000000098DF800908DF801902278831E02F0F7
:109810003F0CA0F1010A611C4D461FFA8AF702AA0B
:10982000BCF1200F79D2DFE80CF089107861786CF8
:1098300078AA78CD78F778FC78F478F378F27878AD
:1098400078F178F078EF78EE7889052876D10420E1
:109850008DF80000B0788DF804006088ADF806003F
:1098600020798DF80100607800F03F000C282BD0A3
:109870000ADCA0F10200092860D2DFE800F0145FE2
:10988000175F1C5F1F5F2200122826D006DC0E28FF
:109890001DD01028DAD11DE08007002016281FD027
:1098A0001828D3D11FE03078800701E030784007D6
:1098B000002843DA37E130780007F9E73078C0064E
:1098C000F6E730788006F3E730784006F0E7307846
:1098D0000006EDE73088C005EAE73088C004E7E716
:1098E00030888004E4E730884004E1E73178890774
:1098F00024D50328AAD105208DF80000B4F8010072
:10990000D2E031784907F3D5062817D3617898B2A9
:10991000012903D0022999D102E01FE1022700E0CA
:10992000102706218DF8001061788DF80610ADF82B
:109930000490A11C904607F102091BE097E000BFCC
:1099400031F8022BA0F1020AA8F800208B463A4613
:1099500008F1020010F0DAFF08EB070202F102083A
:10996000BDF80420AAEB0700521C0BEB070180B2E4
:10997000ADF804208145E3D9002878D1D3E03078D0
:10998000000774D507208DF800001FFA8AF1ADF8A2
:109990000490601C0DF106020FE000BF30F8023B9E
:1099A00022F8023B30F8023B22F8023B091FBDF8C7
:1099B000043089B25B1CADF804300429EED20029D2
:1099C00055D1B0E03178C90651D502284FD30820CF
:1099D0008DF80000ADF8069061789BB28DF8041008
:1099E000A01C0CE0078822F8047B871C80C25B1A4D
:1099F000BDF8067008447F1C9BB2ADF80670994212
:109A0000F0D9A3BB8FE070E075E065E04FE042E085
:109A10001DE012E005E0FFE73078800627D5092039
:109A200003E03078400622D50A208DF80000B08887
:109A3000ADF80400ADF8067007E03078000616D5E2
:109A40000B208DF80000ADF8047002916BE03188B6
:109A5000C9050CD502287FD30C208DF8000099B2DF
:109A6000ADF8069063788DF80430A01C10E073E028
:109A7000078822F8027B478822F8027B071D80C2F4
:109A8000C91ABDF8067018447F1C89B2ADF806707B
:109A90008B42EDD993E73188C9045DD501285BD1AC
:109AA0000D208DF80000B088ADF804003BE031884F
:109AB000890451D505284FD30E218DF80010B188A7
:109AC000ADF80410B4F80310401FADF80800601D95
:109AD000ADF80610039026E0318849043CD50128F2
:109AE0003AD10F208DF800001DE03188090433D4ED
:109AF000B4F80110F18003282ED3217801F03F0142
:109B00001B2925D011218DF80010318841F4004126
:109B1000A6F80010B4F80110ADF80410C01EADF89E
:109B20000600E01C0290207800F03F001B2809D0BE
:109B30001D2807D003201A9907F069FF308800F428
:109B40000040308068461999F8F721FA284652E615
:109B500010218DF80010DDE70725F7E70825F5E768
:109B600000B597B0032806D18DF8000001910021BF
:109B70006846F8F70CFA17B000BD00002DE9FF4F5A
:109B80008DB09346DDE91A56DDF8749004464FF027
:109B9000000A082A06D0E06901F029F858B110201F
:109BA0003070BCE02888092140F01000288089F836
:109BB0000010022717E0E16901208871E2694FF483
:109BC00020519180E1698872E06942F601010181CA
:109BD000E16900208873288840F020002880112047
:109BE00089F800000427307809900A20307004F1C9
:109BF000180009F1020802250B9001F053FA002029
:109C000066E000BFBBF1100F06D1022D04D0A8EB17
:109C10000A00BDF80C204280BDF80E001099884261
:109C200003D9F649097A0E9104E003D1099909B1E3
:109C300031701FE0A8F800001C980088A0EB050018
:109C4000A0EB070083B2C7F1FF00984200D20346A1
:109C50000E980AAA08EB07018DE8070094F8201077
:109C6000BDF80E00002201F08AFA307030B1C0B2A7
:109C7000832858D0BDF80E0020833DE0089828B115
:109C8000DE48006800790A282BD335E0BDF82800AB
:109C9000C11901F0FF0A022D0ED099F801105145AB
:109CA00003D1BDF81820824208D0D4488A46006803
:109CB0000178032908D021E089F801A0CF48006885
:109CC0000178042906D008E000790A2816D201207C
:109CD000089006E0BDF80E10818005EB0A00D04424
:109CE00085B203AA0E990B9801F0DFF920B91C98F0
:109CF0000088401BB84285DA022D0BD0BBF1100F53
:109D000004D1A8EB0A01BDF80C0048801C9805801E
:109D100000203070B94800680078032803D0002084
:109D200011B0BDE8F08F0220FAE72DE9F0410546B9
:109D3000406B1346002758B3491F8EB2698FA1F5B7
:109D40007F42FF3A05D0421892881144891D8CB297
:109D500000E00024A1192A8F0831914216D820442E
:109D6000B3F8011020F8021BB3F8031020F8021B0F
:109D7000324620F8026B591D10F0C8FD6C87696BE4
:109D800000202144B61D3144088002E0092700E08C
:109D900083273846BDE8F08110B50B88048F9C42BC
:109DA0000CD9446BE018048844B1848824F400443E
:109DB000A41D23440B801060002010BD822010BD24
:109DC0002DE9F04788B00025904689468246ADF8D7
:109DD0001050052745E0039806888088000440D489
:109DE000A8F8006005A80097CDE901504FF4007372
:109DF00000224946304601F0C2F9040038D1BDF8CE
:109E00001000ADF81800039804888188B44214D17A
:109E10000A0412D4CDE9005721F40041029541F41F
:109E2000804342884946204600F0BAFF04000BD127
:109E30000398818841F40041818003AA06A9504615
:109E4000FFF7AAFF0400DED0CDE900570398029582
:109E5000BDF8143000880022494600F0A1FF822C92
:109E600006D103AA04A95046FFF796FF0400B2D01A
:109E7000ADF8105004E00398818821F400418180FE
:109E800003AA04A95046FFF787FF0028F3D0822CCD
:109E900003D0204608B0BDE8F0870020FAE730B5CF
:109EA0000446406B97B0002570B10B208DF8000080
:109EB000208FADF80800606B039101900021684687
:109EC000FCF76DFB8DF800504FF6FF7065636087FF
:109ED000258717B030BD2DE9F041044686B00E4607
:109EE000616B00200C9D174600292AD0012B28D138
:109EF0002A4631462046FFF763FF002821D1002F74
:109F00001FD0A04634460026ADF8106005270EE0AD
:109F100003980088288003980296811DCDE90017D8
:109F2000838842880088214600F03AFF30B903AAAE
:109F300004A94046FFF730FF0028E9D0822800D16D
:109F4000002006B026E72DE9F0411546DDE906645C
:109F50004A1D378892B2974201D206201AE7328012
:109F6000172204F8012B0A46208065801946201D1F
:109F700010F0CCFC00200DE700220280C262831D9D
:109F80000263C36142634FF6FF734387028780F821
:109F9000201070474FF6FF720280042007F037BD93
:109FA00030B597B00D460446FFF779FF208E48B1D3
:109FB00001208DF80000E06ACDE901050021684626
:109FC000FCF7EDFA0020E062206382E70146002002
:109FD00009880A0700D5012011F0F00F01D040F0E8
:109FE0000200CA0501D540F004008A0501D540F001
:109FF0001000490501D540F0200070478C07002073
:10A000002DE9FF4FA7B01F46349E299D379C5FEA7C
:10A01000000817D02878410610D400F03F011E290F
:10A020000AD0218811F4FE6F0CD13A88172A09D37F
:10A03000A1F57F42FF3A05D0010606D500F03F00AA
:10A04000122802D004202BB06BE6FE4928984FF06E
:10A05000000908728DF810908DF834900DAA0A60EE
:10A06000359A4A60ADF81490ADF8909028780322A4
:10A0700000F03F038646711C04F1180CCB464FF0EC
:10A08000040AA8F10500CDF898C01F2B7DD2DFE8A7
:10A0900003F07C7C107C1C7C867CEF7CEE7CED7C71
:10A0A000EC7CEF7CEB7C7C7CEA7CE97C7C7C7C7CC3
:10A0B000E800B8F1030F02D08DF810A0EFE2327083
:10A0C0001720A6F801003A80BEE2B8F1050FF3D1DF
:10A0D000B5F801002083ADF81400B5F803106183D2
:10A0E00000287DD088427BD884F808B0A4F806B058
:10A0F0004FF6FF706084269800F0D4FF0520307082
:10A10000B01C00904FF0020A08AA2899269800F087
:10A11000CCFF00287ED19DF82600012803D0022024
:10A120007070102002E0012070700220834600222F
:10A1300001A909A805F0B5FA30BB9DF804008345D4
:10A1400022D13A88801CA2EB0A0181421CDB0098D4
:10A15000BDF822100AF1020A0180009909A8891CA1
:10A160000A46009101A905F09CFA9DF804000099A7
:10A1700008AA014450441FFA80FA009128992698B1
:10A1800000F093FF0028D2D000E069E2BAF1020F9C
:10A1900040D0A7F800A057E28DF8100054E2B8F1C3
:10A1A000070F89D3B5F801002083ADF81400B5F886
:10A1B00003106183A0B1884212D84FF0010A84F8DD
:10A1C00008A0B5F80500E08000202073E06900F0E9
:10A1D0000EFD90B9E16981F806A04FF4205100E02E
:10A1E00078E0E26942F601009180E16981F80AA015
:10A1F000E1690881E16900208873A8F107006084A3
:10A20000E81D6062269800F04DFF0720307006F1CF
:10A21000010A00E06FE000204FF0010BADF82200D2
:10A2200018E000BFBBF1010F0CD0E0698079012874
:10A230001FD03AF8021C00BF0BF102002AF8021BE3
:10A240001FFA80FBBDF822100BF102002AF8021B56
:10A250001FFA80FB08AA2899269800F026FF58B11B
:10A260000FE0DAE16BE10AE1AEE0D2E17BE05AE037
:10A270001EE0BDF82010DFE73988A1EB0B000428B1
:10A28000D0DABBF1010F36D0E069807901280CD01B
:10A29000BDF82010A1F57F40FF3806D03AF8021C27
:10A2A000AAF800100BF10200B1E1BDF82010F7E7A9
:10A2B000B8F1070F03D0B8F1150F7FF4FDAEB5F874
:10A2C00001102183ADF81410B5F80320628309B1A1
:10A2D000914201D901205FE701212172A4F806B063
:10A2E00084F80CB0B8F1050F07D0C0B2691DE2695F
:10A2F00005F0B8F908B10A204EE74FF6FF70608408
:10A3000004A824A9CDE90010CDE90276287800231D
:10A3100000F03F0220462899FFF730FC8146208B51
:10A32000ADF8140090E1B8F1030FC6D14020ADF8AC
:10A330009000B5F801002083ADF81400289ACDE90B
:10A3400000210AAB029339880022491E8BB294F88F
:10A35000201000F014FF8DF8100058BB0B20307057
:10A36000BDF828002EE0B8F1050FA6D18020ADF889
:10A370009000B5F801002083B5F803206284ADF8A1
:10A380001400B2F5007F01D9072005E742F47C42B2
:10A390006284289BCDE900310DF12C0CCDF808C06A
:10A3A0003988491E8BB294F8201000F0E8FE8DF831
:10A3B000100018B18328B5D10220BEE00D20307006
:10A3C000BDF82C00401C22E14FEADE1000EB4000FB
:10A3D00002EB8000404505D95FEA4E607FF56CAE28
:10A3E000584614E1B5F801C0ADF814C02978490603
:10A3F00008D505218DF834102978090605D58DF882
:10A4000034B031E106218DF83410E91C289BA8EB0B
:10A41000000ACDE90013CDF808B009911FFA8AF3BC
:10A4200094F820100022604600F0BAFC8DF810006D
:10A430008DF834B02978490610D52088C00509D593
:10A44000208B01E08C070020BDF81410884201D158
:10A45000C4F824B058468DF810B0D8E0832801D154
:10A460004FF002094FF48070ADF89000BDF8140071
:10A470002083A4F822A0099860621320C5E0B8F1F7
:10A48000050FFFF419AEB5F801C0ADF814C0218F67
:10A4900041B3A1F57F42FE3A24D007218DF8341054
:10A4A000289A6B1DCDE9003280B2CDF808B040F497
:10A4B0000043DA46B5F8032094F82010604600F017
:10A4C0006FFC4FF400718DF810008DF834A0ADF8DA
:10A4D0009010832810D0E8B1218FA1F57F40FE387D
:10A4E00007D0DCE00A218DF834104FF6FE71218789
:10A4F000D6E7A4F838A0A7E02A4641462046FFF751
:10A5000014FC8DF8100008B1832848D1BDF8140060
:10A51000208351E72A4641462046FFF706FC8DF886
:10A520001000E0BB618F606BCDE9007643185A885C
:10A53000998833F8060BFFF706FD814684E095F80D
:10A5400001A0B8F1020F7CD15FEA0A0002D0BAF193
:10A55000010F76D108208DF8340005A800908DF801
:10A5600038A094F82010534600222046FFF7B3FC91
:10A570008DF839008DF83AB050B9BAF1010F12D008
:10A58000BAF1000F04D1218FA1F57F40FF380AD026
:10A59000208F40B18DF834B04FF4806000E053E07C
:10A5A000ADF890000DE00DA83599FBF7F8FF814656
:10A5B0004FF480608DF834B0ADF89000B9F1020F1F
:10A5C00006D0FB480068807928B18DF8100043E080
:10A5D000A4F818A038E0B9F1000F03D081208DF85D
:10A5E000100043E005A8009094F820105346012283
:10A5F0002046FFF770FC8DF8100020463699FFF7D3
:10A600004EFC9DF81000F8B91920307001203880F8
:10A610001AE006208DF8100041E02078000723D5CD
:10A62000B8F1010F20D109208DF83400A088ADF8D1
:10A6300038000420369907F0EAF90820ADF89000B8
:10A6400000E011E0A7F800B09DF8340020B10DA89B
:10A650003599FBF7A4FF8146B9F1000F1CD005E046
:10A660005FEA4E607FF528AD4FF004092088BDF801
:10A67000901008432080BDF8900080050AD5218FF6
:10A68000A1F57F40FE3805D12998E062A4F830801A
:10A690004FF003094846D6E49DF8100058B1012058
:10A6A000307028787070BDF8140070809DF810002C
:10A6B0003071052038802088BDF8901088432080B4
:10A6C000E8E72DE9FF4F80460178A5B001208840DA
:10A6D0004FF60901349C0840ADF86C0021884FF01A
:10A6E0000009A1F57F42FF3A02D028B1080703D53F
:10A6F000012029B0BDE8F08F289F4FF0000A04A880
:10A7000087F800A02799269A55460988ADF87C104D
:10A71000A7498DF868A04FF0050B0A728DF810A0BC
:10A7200008603298486098F8000001282FD002286D
:10A7300009D0032874D1387820F03F001D303870DC
:10A74000B8F80400A08098F80000022804D13878F6
:10A7500020F03F001B30387021AAF81CCDF800B063
:10A76000CDE90102BDF87C0094F82010C01E83B230
:10A77000B8F80400002200F002FD0028DAD1B8F891
:10A780000400A7F80100BDF88400C01CC5E098F8DB
:10A7900005108DF8681098F804004FF4007901282E
:10A7A00002D00228C6D131E1208808F1080600F461
:10A7B000FE60ADF86C0010F0F00F1AD010F0C00F72
:10A7C00005D03088228B904201D005257AE181B9ED
:10A7D000B078C0070DD0B268CDE9002BCDF808A045
:10A7E000F388B28894F82010308800F0D9FA002855
:10A7F00071D12898BDF86C10401C802946D006DC29
:10A8000010290ED020290CD0402993D122E0B1F597
:10A81000807F61D049457DD0B1F5806F8AD1C9E094
:10A8200028E1C80601D5082000E010208146042058
:10A83000ADF814A01BA98DF8100001AB00911FAA60
:10A840001AA883E8850033884A4605212046FFF789
:10A8500095F992E09DF868104FF00A09002939D166
:10A8600021AACDF800B0CDE90102BDF87C0094F832
:10A870002010401E83B2208B002200F080FC8DF857
:10A8800068000B203870BDF884001AE09DF868104D
:10A890004FF00C0900291DD123AACDF800B0CDE955
:10A8A0000102BDF87C00628C401E83B294F8201037
:10A8B000208B00F064FC8DF868000D203870BDF826
:10A8C0008C00401CADF87C0004208DF81000208B1B
:10A8D000ADF81400B9E055E03188208B814251D1A8
:10A8E0009DF868104FF01209002918D1616A79B1FA
:10A8F000B178C90746D0B368CDE9003BCDF808A0D0
:10A90000F388B28894F8201000F04AFA8DF86800B5
:10A91000132000E004E038700120ADF87C0094E0E2
:10A920003088218B88422DD19DF868104FF0160990
:10A9300049B1606BD8B34FF6FF7100205646ADF8B1
:10A9400008A0019126E0616B61B1B078C00719D110
:10A95000608F0B181FA8CDE900075A88998833F833
:10A96000060B08E0B178C9070CD01FA9CDE9001784
:10A97000B288F188B368FFF7E6FA050065D0062DC6
:10A9800079D03EE005253CE0019121AA02A92046AC
:10A99000FFF702FA628FBDF808108A4201D0002842
:10A9A000F2D0608F616B08440680019860874CE0AC
:10A9B0008C0700209DF868004FF0180940B1208BEB
:10A9C000D0B13088208320463399FFF768FA3CE005
:10A9D00004F118000090237E94F8201001222046F4
:10A9E000FFF779FA8DF868000028ECD1192038704B
:10A9F0000120ADF87C00E6E7052520463399FFF7F6
:10AA00004EFA9DF81000032856D05BE0208800F431
:10AA10000070ADF86C0048452CD1208FA0F57F4127
:10AA2000FE397FF4D2AED8F808004FF0160948B1CD
:10AA30006063B8F80C1021874FF6FF716187A0F8AA
:10AA400000A002E04FF6FF702087BDF86C0030F4E4
:10AA5000FE6116D0782300220420339906F039FFD6
:10AA600098F80000A0702088BDF86C100843208082
:10AA70000AE000E006252088BDF86C10884320809D
:10AA800020E02188814321809DF8100028B15F4893
:10AA9000416804A8FBF783FD05469DF8680088B16E
:10AAA00087F8019001203870208B78809DF868002D
:10AAB0003871ADF87CB005E05448416804A8FBF754
:10AAC0006EFD0546208810F4FE6F23D1208E08B35A
:10AAD00027990988ADF87C10DDE932322899CDE953
:10AAE0000013CDE902241FABE26A2699FFF788FA2A
:10AAF000054603280ED001208DF81000E06A05906D
:10AB000033980690002104A8FBF749FD00B10546E3
:10AB1000A4F830A02798BDF87C1001802846E8E50D
:10AB200000B597B0042807D102208DF800000191EC
:10AB300000216846FBF733FD17B000BD70B5334CFC
:10AB4000037800222168012B02D0022B44D129E096
:10AB50000B780BB1042B03D10A7122680321117009
:10AB60002168062582880B7905EBC303CA52216848
:10AB700008230A250A7903EBC2021144C2880A801D
:10AB8000216802890B7905EBC303CA524189206809
:10AB90000C23027903EBC202815220680179491C1F
:10ABA00001711DE00A7482888A802168C288CA8087
:10ABB000226801891181226841895181C168206818
:10ABC000C1606168FBF7EBFC0146022806D02068F3
:10ABD000007C002801D119B1812070BD832070BD97
:10ABE000002070BD406B002800D0012070478178A4
:10ABF000012909D10088B0F5205F03D042F6010198
:10AC0000884201D100207047062070478C07002041
:10AC100010B58B787BB182789A4205D10B8853B1FD
:10AC200002E08B79091D43B18B789A42F9D10388F0
:10AC30000C88A342F5D1002010BD812010BD05284D
:10AC400024D012B1012A0ED103E00988C1F3812179
:10AC500002E00988C1F3013139B1012916D0022976
:10AC600008D003290CD0812070470AB10320704717
:10AC700002207047032809D0042807D020B107E03C
:10AC8000042803D0022803D0052070470020704715
:10AC90000F20704710B513880B809BB21C061FD580
:10ACA000FE4CA47A844204D843F0100008800020AF
:10ACB00010BD94682478C44064F304130B801378A7
:10ACC000917803F0030341EA032140F20123B1FB31
:10ACD000F3F403FB1411926800FB0120401C10BD2B
:10ACE000906810BD37B5BDF804101180BDF8045050
:10ACF00029061BD5E94901239468897A814209D83C
:10AD0000FE280FD1E80602D58B405B1E00E0002331
:10AD1000237007E0217883409943C5F300138340F3
:10AD200019432170108820F0100010803EBD2DE9DD
:10AD3000F0410746C81C0E4620F00300B04202D086
:10AD40008620BDE8F081082A01D90E20F9E7D34D0D
:10AD5000002034462E60AF802881AA72E8801AE075
:10AD6000E988491CE980810614D4A17800F0030029
:10AD700041EA002040F20121B0FBF1F201FB120197
:10AD8000206800F0E0FA2989084480B22881381A46
:10AD90003044A0600C3420884107E1D40020D0E783
:10ADA0002DE9FF4F85B01546DDE912B6804699467C
:10ADB00023F4404700F0B7FA04000BD020780006D7
:10ADC0000AD5B648817A0698814205D8872009B00D
:10ADD000BDE8F08F0120FAE7224669460698FFF7A2
:10ADE00059FF824600208DF80400052E18D001225C
:10ADF00021463046FFF723FF0028E8D1207840069F
:10AE00000ED502208DF80400ADF80880BDF80000D2
:10AE1000ADF80C50ADF80A00ADF80E70CDF810B0DA
:10AE20005FEA094004D500273D46B84601260CE0FC
:10AE30002178A07801F0030140EA012040F20121CD
:10AE4000B0FBF1F2804601FB12865FEA494009D56A
:10AE5000B04507D12188E078C1F3012140EA012003
:10AE6000A84201D3B54201D90720B0E778191FFAEB
:10AE700080F9B14501D90D20A9E79DF8040020B162
:10AE800001A8FBF78AFB0028A1D1B04507D1208893
:10AE90004FEA192161F30920208084F80390149867
:10AEA00000B10780BBF1000F15D00AEB05003A4650
:10AEB00059460FF02BFD224669460698FFF7EAFE39
:10AEC000BDF80000224620F01000ADF80000009907
:10AED0000698FFF707FF002079E72DE9FF4FDFF81D
:10AEE000BC9182461746B9F80610D9F8000001EB6C
:10AEF000410100EB810440F20120B2FBF0F183B08C
:10AF000000FB11764D46DDF844803146049800F090
:10AF10001AFA29682A898B46611A0C3101441144B6
:10AF2000AB8889B28B4202D8842007B050E70499DD
:10AF30008DB2290603D5A90601D58520F5E7B9F814
:10AF400006C00CF1010C1FFA8CFCA9F806C012997E
:10AF500009B1A1F800C0A90602D5C4F8088007E02D
:10AF6000104480B2A9F80800191A01EB0B00A06088
:10AF70002246FE200499FFF7B5FEA770E6702088F0
:10AF8000390A61F30100310A61F3092040F004003D
:10AF900020809AF80200A071BAF80000A080002674
:10AFA0002673280602D599F80A7000E00127A80642
:10AFB00001D54FF000084D4600244FF005090DE083
:10AFC000CDF80080CDE90196E8882146109B069ACD
:10AFD000FFF7E6FE0028A8D1641CE4B2BC42EFD320
:10AFE0000020A2E72DE9F047804600F09CF9070019
:10AFF00005D000264446294D40F2012916E00120E3
:10B00000BDE8F087204600F08EF90278817802F0E2
:10B01000030241EA0222B2FBF9F309FB13210068A3
:10B0200000F091F93044641C86B2A4B2E988601E35
:10B030008142E7DCA8F10100E8802889801B288193
:10B0400000203870DCE720B1401E10809170002095
:10B0500070470120704710B5104904460088CA881F
:10B06000904201D3822010BD096800EB400001EB43
:10B0700080029079A072908820811188D078C1F3E5
:10B08000012140EA0120A081A078211DFFF702FEE6
:10B0900020612088401C2080E08001E0980700208B
:10B0A000002010BD0121018270472DE9FC474FF6B9
:10B0B000FF780546A2F80080406817468A468078E7
:10B0C0008DF8020068680088ADF8000000208DF857
:10B0D0000600288A2C88A04200D304462C822DE04A
:10B0E000288A401C2882301D6968FFF791FD18BB33
:10B0F0003988414501D1601E38806888A04222D33A
:10B100003188F078C1F3012140EA01296946301DF8
:10B11000FFF77EFD80B96989414519D0002231468B
:10B120005046FFF78CFD38B96A894A4504D1E96871
:10B13000B0680FF0BFFB58B1641CA4B2204600F009
:10B14000F2F80600CCD1641E2C828220BDE8FC8778
:10B150007C80B079B871B088B8803178B07801F06F
:10B16000030140EA01207881A7F80C90287A324642
:10B1700007F10801FFF78EFD38610020E6E72DE9B1
:10B18000F04F85B01C4690460F468346DDF838A048
:10B19000DDF8409000F0C7F8050009D028780006D7
:10B1A00008D57048807AB84204D8872005B00FE6E9
:10B1B0000120FBE7C8F309062A4669463846FFF72F
:10B1C00069FD07465046BAF1050F1AD000222946FC
:10B1D000FFF735FD0028E9D12878400611D5012078
:10B1E0008DF80400ADF808B0BDF80000ADF80A0015
:10B1F000ADF80C60ADF80E4001A8FBF7CEF90028C1
:10B20000D4D12888A97800F0030241EA0221EA7823
:10B21000C0F3012042EA0020464507D0B1F5007F87
:10B2200004D9611E814201DD0B20BFE7864201D9AE
:10B230000720BBE7801B82B2A24200D92246B9F1A7
:10B24000000F01D0A9F800200F9810B1B9190FF024
:10B250005DFB0020AAE72DE9F0411D4617460E468A
:10B2600000F061F8040008D02078000607D53D48BA
:10B27000807AB04203D8872063E5012061E5224649
:10B2800039463046FFF706FD65B12178A07801F018
:10B29000030140EA0120B0F5007F01D8012000E061
:10B2A0000020287000204CE52DE9F0411D4617468E
:10B2B0000E4600F038F8040008D02078000607D5C4
:10B2C0002848807AB04203D887203AE5012038E543
:10B2D000224639463046FFF705FDFF2D14D0218860
:10B2E000A07801F0030240EA022040F20122B0FB04
:10B2F000F2F302FB130015B900F2012080B2A07036
:10B30000000A60F30101218000201AE510B50C4607
:10B3100000F009F828B1818821808079A070002090
:10B3200010BD012010BD0F49CA88824209D340B127
:10B33000096800EB40006FF00B0202EB800008444C
:10B3400070470020704780B2820609D4000605D5F8
:10B350000448807A4843401C80B2704708467047D2
:10B3600000207047980700201E2829D00FDC0C28E9
:10B3700022D008DC092823D2DFE800F013221522AE
:10B38000221C1C181A0012281AD1072070473028D6
:10B3900016DDA0F13A00032812D2DFE800F00F1109
:10B3A00009000020704743F20200704704207047F4
:10B3B0000D2070470F2070470820704711207047FC
:10B3C0000320704710B50C4601F079FCD0B120463F
:10B3D00000F098FA98B122780E2A0AD00F2A08D0E5
:10B3E000022A06D0032A04D0102A06D00FF05BFBF5
:10B3F0000AE0A078BDE81040B6E7112010BD0FF0BC
:10B4000052FB01E00FF04FFB002010BD00F07ABAB4
:10B4100070B50346002002466FF02F050EE09C5CDD
:10B42000A4F130060A2E02D34FF0FF3070BD00EBBE
:10B43000800005EB4000521C2044D2B28A42EED379
:10B4400070BD30B50A240AE0B0FBF4F304FB13002E
:10B450008D18303005F8010C521E1846D2B2002A61
:10B46000F2D130BD30B500234FF6FF7510E0040A6D
:10B4700044EA002084B2C85C6040C0F3031460401A
:10B4800005EA00344440E0B25B1C84EA40109BB201
:10B490009342ECD330BD000010B509F085FC0428C0
:10B4A00003D009F081FC052802D108F060FB50B9F7
:10B4B00009F09EFD032803D009F0A0FD032804D164
:10B4C00007F035FC08B1012010BD002010BD70B59B
:10B4D0000C460546062102F02AFA606008B10020F9
:10B4E00006E00721284602F022FA606018B1012028
:10B4F0002070002070BD022070BD2DE9FC5F0C465D
:10B50000064600276946FFF7E2FF00286FD19DF845
:10B51000000058B107F070FBB04268D0002221460D
:10B5200030460BF011FE00287AD116E008F0CDF875
:10B53000B0425CD00022214630460BF00FFA0028C2
:10B540006ED1019D95F89000283518B9687E08B134
:10B55000012000E00020804603E0019D95F8418035
:10B5600028354FF0010B95F82D004FF00009A0B1E0
:10B5700095F82E00800710D584F8019084F800B06B
:10B5800084F80290A68095F82F10A171298E218150
:10B59000698E618185F82D9042E0304602F07BFB98
:10B5A0005FEA000A04D10FF07EFA01E07F1CFFB2CF
:10B5B00000215046F7F71AFD0028F7D147B184F86B
:10B5C00001900D202070A680E78084F802B027E06B
:10B5D000304602F04DFB070001D10FF064FAB8F1DC
:10B5E000000F04D00021384601F02EFC10B10020DD
:10B5F000BDE8FC9F9DF8000038B90198D0F8A40080
:10B600004188B14201D180F8009084F801900A216C
:10B61000217084F80290A680A97EA17185F8199006
:10B620000120E5E710B501784068008831B10721B5
:10B6300002F087F9002800D00C2010BD0621F7E7A2
:10B640001CB504466946FFF742FF08B10FF02BFA1C
:10B65000204607F005FA08B90FF025FA6846FFF70B
:10B66000E1FF002801D00FF01EFA1CBD1CB5694691
:10B67000FFF72DFF08B10FF016FA684601F02AFC1B
:10B68000FC4900208968A1F892001CBD2DE9FC410D
:10B6900004460E46062002F0F3F80546072002F0A5
:10B6A000EFF82844C7B20025A8463E4417E020889A
:10B6B000401C80B22080B04202D34046A4F80080F3
:10B6C00080B2B84204D3B04202D20020BDE8FC816F
:10B6D0006946FFF7FCFE0028F8D06D1CEDB2AE42C3
:10B6E000E5D84FF6FF7020801220EFE70EB54FF639
:10B6F000FF70ADF800000DE001A9BDF80000FFF7F4
:10B70000E6FE08B10FF0CFF901A8FFF78BFF08B1F3
:10B710000FF0C9F900216846FFF7B8FF0028EBD009
:10B720000EBD2DE9F041D4A0D54C0679002507685F
:10B7300084F84250243401F0C4FBE5770420A08251
:10B740001020E0824FF6FF70A4F8DE0084F8E0508D
:10B75000A4F8E200657304F8245CA572257404F172
:10B760005C0084F8D85040F87D7F04F1D90106715F
:10B77000BDE8F041481E0BF09CB92DE9F041BD4CED
:10B780000D466060217007F041F9FFF7AFFFFFF74A
:10B79000C8FF207809F00CF9B949C431A1F1810042
:10B7A0000F46064608F0B4F860680BF04DF90CF04F
:10B7B000C7FC284609F0B7FF3946304607F056FA6D
:10B7C00060680BF04DFD01F07CFBAD49002081F875
:10B7D0004300BDE8F0812DE9F047040001D10FF0EE
:10B7E00062F9A74D002695F8310058B16670102017
:10B7F000207095F83200A07095F83300E07085F85D
:10B80000316071E0287840B12C22A91C20460FF04D
:10B810007DF80E2020702E7066E095F82E0060B145
:10B820000120E07095F82F00A07095F8300060704E
:10B830000F20207085F82E6056E092480221824643
:10B84000FFF724FF08B10FF02EF9B5F80691062096
:10B8500002F016F80746072002F012F83844C7B283
:10B86000781C00F0FF0800BFB5F80601B84213D1FC
:10B870000021204607F0DCFE80BB95F8340070B351
:10B880006670132020701C21A01C0FF0B6F8022057
:10B89000A07085F8346027E0404521D10021204682
:10B8A00007F07CF9D8B1207813281DD1A0783C2866
:10B8B0001AD1A088072102F03AF8050001D10FF053
:10B8C000F2F8288807F0CCF808B90FF0ECF8A08857
:10B8D000072102F036F808B10FF0E5F804E006E0C1
:10B8E0002146FFF70AFE10B10120BDE8F0870221D2
:10B8F0005046FFF7CBFE18B9B5F806114945B3D14C
:10B900000020F2E767E710B508F0C7FF08B10FF0B5
:10B91000CAF80BF097F808B10FF0C5F807F0AEFFC2
:10B9200009F0EAFE08B10FF0BEF80BF097FC08B181
:10B930000FF0B9F807F06AF908B10FF0B4F80CF09D
:10B94000F9FB08B10FF0AFF8FFF7D0FEFFF7E9FE03
:10B9500007F03EF801F0B5FA4948002180F843109D
:10B960000171012141710222C270017010BD10B538
:10B97000434C207828B10A21BDE810400E2001F088
:10B980006DBAFFF789FD08B10C2002E001F099FAC9
:10B9900000202071012060710A21E170207010BD2B
:10B9A00070B5374C0546207828B1BDE87040392184
:10B9B0000E2001F053BAFFF76FFD08B10C2012E022
:10B9C00094F8430008280DD204EB001010222946F9
:10B9D000443001F050FA94F84300401C84F84300CE
:10B9E000002000E007202071012060713921E17002
:10B9F000207070BD70B5224C0546207828B1BDE896
:10BA000070400B210E2001F029BA287818B10128C6
:10BA100001D0122016E094F8C400082819D2FFF7CC
:10BA20003BFD08B10C200DE016482B7894F8C410AB
:10BA30006A1C3E3806F041FA94F8C400401C84F8B1
:10BA4000C40000202071012060710B21E170207082
:10BA500070BD0720F6E710B5094C207828B13821D1
:10BA6000BDE810400E2001F0F9B9FFF715FD58B1FF
:10BA70000C200CE040000020FFFFFFFF1F00000033
:10BA8000A4070020AA080020002084F843002071A9
:10BA9000012060713821E170207010BDF9480178F3
:10BAA00019B10F210E2001F0D9B9002101710E2129
:10BAB00081700F21C170FF2181714FF6FF710181EB
:10BAC000F14949680A7882728A8882814988C181ED
:10BAD0000121417101707047EA490A781AB13B218E
:10BAE0000E2001F0BBB90088A1F80201012081F805
:10BAF000040100220A7148713B22CA700870704725
:10BB000010B5E04C207828B12B21BDE810400E2064
:10BB100001F0A4B90821A01D05F072FC00202071DD
:10BB2000012060712B21E170207010BD70B5D54CE3
:10BB3000217829B1BDE8704031210E2001F08EB985
:10BB400090F90000042814D098B1011D11D010F113
:10BB5000080F0ED010F10C0F0BD010F1100F08D001
:10BB600010F1140F05D010F1280F02D0122020710F
:10BB700003E0002506F0E4F925713120E070012092
:10BB80006071207070BD30B5BE4D04468DB0287810
:10BB900028B12A210E2001F061F90DB030BD10222C
:10BBA0002146684601F067F9102204F1100104A84B
:10BBB00001F061F968460DF093FD10222C46A81D96
:10BBC00008A901F058F9002020710E20A0702A2049
:10BBD000E070012060712070DFE72DE9FF41A94C82
:10BBE000207828B13A210E2001F038F9BDE8FF8114
:10BBF0004FF0000884F80680B4F80201ADF80400A4
:10BC000002A9FFF764FC20B1002101A8FFF73EFD67
:10BC1000F0BBBDF80400ADF8000002A980B2FFF748
:10BC200056FC08B10EF03FFFBDF8000002F033F8FB
:10BC3000060001D10EF037FF3046039DF7F7D0F92B
:10BC400080F0010695F84150BDF8000002F010F8B0
:10BC5000070001D10EF027FF0021384601F0F4F86B
:10BC600055EA000119D0A279BDF8001004EB420298
:10BC70001181844AA3791832995C65F300019954C3
:10BC8000A37960F341019954A07966F3820100E041
:10BC90000EE08154A079401CA07100216846FFF796
:10BCA000F5FC28B9BDF80000BDF804108842B4D1F5
:10BCB000012084F8048060713A21E170207095E7DA
:10BCC00070B5704C0546207828B1BDE8704034212D
:10BCD0000E2001F0C3B809F067F8052804D0284603
:10BCE00008F051FE002000E00C202071012060715E
:10BCF0003421E170207070BD6248017819B10E21C5
:10BD0000084601F0ABB86049CA68C0F80620098A45
:10BD1000418100210171012141710E22C270017027
:10BD2000704770B5574C0646251D207828B1BDE8F0
:10BD3000704032210E2001F091B83146002007F00A
:10BD40007DF8287058B900213246084607F0C6FE33
:10BD5000287020B94C483168C160B1880182012047
:10BD600060713221E170207070BD70B5454C0546A0
:10BD7000207828B1BDE8704030210E2001F06EB867
:10BD800008F095FE10B909F059FF68B1287809F05C
:10BD900019FD287807F01AFF00202071012060713A
:10BDA0003021E170207070BD0C20F6E72DE9F041E4
:10BDB000344C0646251D207828B1BDE8F0411721F6
:10BDC0000E2001F04BB83146012007F037F82870FB
:10BDD000012768B932460121002007F07FFE287054
:10BDE00030B93068E063B088A4F8400084F842704D
:10BDF00067711720E0702770EBE438B5214D0446D9
:10BE0000287828B1BDE8384030210E2001F026B84E
:10BE1000227961798A4215D0A079E379984211D0CC
:10BE20001F2A0FD81F290DD8002211460DF0B2FC91
:10BE300040B90022E07911460DF0ACFC10B9207A2F
:10BE4000072801D9122015E04FF6FF70ADF8000069
:10BE500009F0CEF8D0B909F0D1F8B8B908F0A4FFCC
:10BE6000A0B900216846FFF711FC78B1204605F023
:10BE700041FF00202871012068713E21E97028707F
:10BE800038BD0000A4070020400000200C20F1E78E
:10BE90002DE9FC47FE4C054694F82E0028B12821D8
:10BEA0000F2000F0DBFFBDE8FC87282084F830007D
:10BEB000012184F82E10A8784FF000091A2825D007
:10BEC0000EDC162831D2DFE800F03030303030217F
:10BED000303030303030303030303030302121218F
:10BEE0002A2822D00BDCA0F11E000C281DD2DFE88E
:10BEF00000F01C1C1C1C1C1C1C1C1C1C1C0D3A389F
:10BF0000042812D2DFE800F0110211022888B0F5EF
:10BF1000706F0AD21F20884684F82F00288869464F
:10BF2000FFF7D5FA18B1022019E0122017E09DF8AA
:10BF30000000019F002806D007F1C607019E05D129
:10BF400006F19D0604E007F19C07F7E706F1C70636
:10BF5000684600F0ABFF08B1387818B10C2084F8BF
:10BF60002F00A0E787F80080A878307084F82F9021
:10BF7000684600F0AFFF96E77CB5C54C05462078D3
:10BF800020B125210E2000F069FF7CBD288869467C
:10BF9000FFF79DFA002168B102202071BC48816042
:10BFA0000173E1800E20A0702520E07001206071F7
:10BFB00020707CBD019A104612F1280282F83610DA
:10BFC0008368A360037B237392F83630002BF5D18E
:10BFD0002888E080E6E72DE9FC41AD4C064694F860
:10BFE0002E0028B110210F2000F038FFBDE8FC81A1
:10BFF0001F2084F82F00102084F83000012784F8D7
:10C000002E7030886946FFF762FA70B9684600F012
:10C010004DFF50B1019D9DF8000028350028019882
:10C0200005D0CA30017841B904E0022006E0D0F81A
:10C03000A400F7E795F82D1019B13A2084F82F00E5
:10C04000D4E795F82E1089070CD1062101709DF8D0
:10C05000000020B901993088D1F8A41048806846C2
:10C0600000F038FF002084F82F0085F82D70BDE720
:10C070002DE9F047864D0646287828B1BDE8F047FF
:10C080001D210E2000F0EABE4FF01F0985F8049034
:10C09000012068711D21E970287008F085FE0C27C9
:10C0A00004284FD005284DD0B0791224012800D0A3
:10C0B000E8B9307808B1012819D1F07908B1012820
:10C0C00015D1708843F6FD71021F30248A420ED2CA
:10C0D000B288121F8A420AD22887B0886887B0794E
:10C0E0004FF000084446012803D050B112E02C71F3
:10C0F00007E495F8420028B3654A3C32012108461E
:10C1000002E0644A0021012007F0E8FC040001D0AD
:10C110000EF0C9FCF079012800D010B907F006FD37
:10C12000044614B185F80490E2E73078012801D084
:10C1300018B109E00021022001E00021012007F0F0
:10C140000AFD08B12F71D3E785F80480D0E770B5F8
:10C150004F4C217829B1BDE870401E210E2000F01F
:10C160007DBE1F212171012161711E22E2702170AB
:10C1700002781221012A00D01AB9407818B101289A
:10C1800001D0217170BD00260C25012A08D008F0CD
:10C190000BFE052802D008F02CFB30B1257170BDD4
:10C1A000618F208F08F090FCF7E7267170BD2DE9B4
:10C1B000F04F87B00546AFF24071D1E90001344E2F
:10C1C00001908A4696F82E0030B107B02121BDE8D3
:10C1D000F04F0F2000F042BE1F2086F82F002120D4
:10C1E00086F830004FF0010886F82E802B8843F641
:10C1F000FD711A1F30208A427ED26A88141F8C4239
:10C20000FAD29A4278D8EA8940F67B41931F8B4252
:10C21000F2D22B8A9C1F8C42EED29A42F2D8698AC3
:10C22000B1F5FA7FE8D2A98A40F67744A1F10A0273
:10C23000A242E1D2B1EBD30F5ED9E98A2A8B9142B7
:10C24000E0D82979122011B1012955D102E069798C
:10C250000029F9D1297B09B101294DD108F0A4FDAC
:10C260004FF00C0905287DD008F09EFD0428FAD077
:10C2700096F83400002875D107F027FAA0F57F4121
:10C28000FF39F8D1062105A801F023FB040003E0E3
:10C29000A40700204C0000202FD003210CF0F9FB54
:10C2A00004F10D07B4F800B00421384605F0A8F8F1
:10C2B000594638460CF0E1FCFEA03F1D0068069090
:10C2C000032106A805F027F8002006A90A5C3A54C5
:10C2D000401CC0B20328F9D3288A6080688AA080F5
:10C2E000A88AE080002784F82E7084F82F7068797F
:10C2F00028B1012807D104E068E0092066E06776EC
:10C3000001E084F81980D5F80600C4F81A0068899D
:10C31000E0830198A06084F80CA084F8AC808DF8CC
:10C320000470012101A804F0F6FF9DF8040000F05C
:10C330000701C0F3C1021144C0F3401008448DF856
:10C340000400401D2076092801D208302076002103
:10C3500020460CF09EFB20880322092106F074FB86
:10C3600018B900E05CE00EF09EFB287B20B10128AC
:10C3700006D00EF098FB2EE00021CF4A012005E008
:10C3800096F8420050B10121CC4A084607F0A6FBBE
:10C3900008B3208806F064FB70B10FE0208806F037
:10C3A0005FFB08B90EF07FFB2088062101F0C9FA77
:10C3B000B0B30EF078FB33E00EF075FB2088062159
:10C3C00001F0BFFA08B10EF06EFB1F2086F82F00B7
:10C3D00007B0BDE8F08F2879012800D010B907F028
:10C3E000A5FB50B92146032007F0B5FB28B96A88A0
:10C3F0002988204608F00BFB20B1208806F030FB8E
:10C4000028B106E084F8A07086F82F70E0E70EF0FF
:10C410004AFB2088062101F094FA08B10EF043FB94
:10C4200086F82F90D4E738B5A44C3C3C207820B156
:10C4300022210E2000F012FD22E51F20207101258F
:10C4400065712220E070257008F0AEFC052802D04E
:10C450000C20207114E500202071684608F06CFB68
:10C460000028E9D10098008806F0FAFA08B90EF021
:10C470001AFB00980621008801F063FA08B10EF05B
:10C4800012FB8D4884F834500C380078FCF7C7FF55
:10C49000F6E42DE9F041894D04463C3D95F82E0027
:10C4A00028B1BDE8F04123210F2000F0D7BC1F20A8
:10C4B00085F82F00232085F83000012085F82E0014
:10C4C000618840F67B438A1F30209A4251D2A2886D
:10C4D000961F9E424DD291424BD8E188B1F5FA7F2A
:10C4E00047D2218940F67746A1F10A03B34240D2F0
:10C4F000B1EBD20F3DD96189A289914239D84FF071
:10C5000000082088062101F012FA06004FF0020709
:10C5100007D000F0BDFC20B1D6F8A400017839B9ED
:10C5200002E085F82F7067E4D6F8B810097809B1F1
:10C530003A201EE005218171D6F8A4004146A0F8FA
:10C540000880D6F8A420A0885081D6F8A420E088DE
:10C550009081D6F8A4202089D081D6F8A400028941
:10C5600043899A4204D88279082A01D89A4203D38F
:10C57000122085F82F003FE422884280D6F8A400DC
:10C58000077085F82F1037E42DE9FE434B4C064623
:10C590003C3C207830B103B02421BDE8F0430E20AC
:10C5A00000F05CBC012565712420E07025703046E8
:10C5B0000CF086FB08B1002000E01220207100285A
:10C5C0002FD13E4884F8FC504430316840F87D1F3C
:10C5D000317901714FF0000884F8FC80694606202B
:10C5E00001F02BF908B10EF05EFA684601F0FDF893
:10C5F000A8B9BDF8047000BFBDF80400062101F021
:10C6000096F9060001D10EF04EFA86F8AC50684655
:10C6100001F0EBF818B9BDF80400B842ECD184F889
:10C620000480BDE8FE8370B5244D06463C3D95F878
:10C630002E0028B1BDE8704026210F2000F00EBC6E
:10C640001F2085F82F00262085F83000012085F86E
:10C650002E003088062101F06AF9040007D000F0AE
:10C6600017FC20B1D4F8A400017831B901E0022010
:10C670000CE0D4F8B810097809B13A2006E0072197
:10C680000170D4F8A41030884880002085F82F006D
:10C6900070BD0A483C38017819B106210E2000F01F
:10C6A000DDBB002101710E2282700622C270C0F82B
:10C6B000061005E0112233004C000020E0070020A6
:10C6C000C0F80A10817941F00101817101214171A5
:10C6D0000170704770B5F84E054696F82E0028B1E7
:10C6E000BDE870402C210F2000F0B8BB1F2086F859
:10C6F0002F002C2086F83000012086F82E00288894
:10C70000062101F014F9040007D000F0C1FB20B1AC
:10C71000D4F8A400017831B901E0022020E0D4F877
:10C72000B810097809B13A201AE094F85C10D1B138
:10C73000D5F802104160D5F80610816054F8A40FB6
:10C74000698910228181206805F10C010E300EF0FC
:10C75000DDF82168032008702168288848800020BF
:10C7600086F82F0070BD0C20FAE770B5D24E044653
:10C770000C25307828B1BDE8704018210E2000F05B
:10C780006DBB08F035FC032852D008F037FC0328B5
:10C790004ED0607908B1012829D1A07908B10128CB
:10C7A00025D1A07B28B1012803D0022801D003287D
:10C7B0001DD1607BD8B1C00819D162884FF4804088
:10C7C000824202D82188814203D9207901280ED1E2
:10C7D00018E0207930B1012814D0022805D00328B0
:10C7E00005D102E0202A0BD30CE0A0290AD220793F
:10C7F000042805D12088202802D36188884201D9E5
:10C80000122515E0207986F83600607910B10128EC
:10C8100004D00DE0A94A0021204606E096F8420027
:10C8200030B1A54A01213C32204606F087FA054680
:10C830000120357170711821F170307070BD10B524
:10C840009D4C217829B11A21BDE810400E2000F03E
:10C8500005BB01781F2902D91220207106E00021B2
:10C8600021710278411C104606F01AFB012060710C
:10C870001A21E170207010BD10B58F4C217829B1BC
:10C880002021BDE810400E2000F0E8BA01781F29F1
:10C8900002D91220207106E0002121710278411C8A
:10C8A000104606F0ECFA012060712021E170207042
:10C8B00010BDF8B5804C217829B1BDE8F8401B21A6
:10C8C0000E2000F0CBBA012767710C21217100788E
:10C8D0000026012803D0E8B3122020716EE006F094
:10C8E000F6F900286AD094F83600B0B1012814D0C7
:10C8F000042812D008F082FB00285FD108F078FBF2
:10C9000018B108F075FB022858D1002008F05DFF2F
:10C9100008B10EF0C8F8267150E008F069FBE8BBDA
:10C9200008F06CFBD0BB06F067F9A0F57F41FF393A
:10C9300044D10721684600F0CCFF604905460C3918
:10C940008860280001D10EF0AEF8032128460BF0D4
:10C95000F0FF00E012E0284606F06DFB2888062272
:10C960000D2106F071F808B90EF09DF8284608F080
:10C970002CFF0028CFD00EF096F8CCE708F038FB5B
:10C98000032803D008F03AFB032817D108F033FB43
:10C990000546002008F03EFE00B900E00EE02671DA
:10C9A00065B1288806F05CF808B90EF07CF8288894
:10C9B000072100F0C6FF08B10EF075F81B20E070EB
:10C9C0002770F8BD70B53C4C0646207828B1BDE80C
:10C9D00070402D210E2000F041BA3088072100F070
:10C9E000A6FF050022D095F8CA0040B995F834009A
:10C9F0000F2801D0102802D195F8FC0058B10C2066
:10CA000020710E20A0702D20E0703088E080012081
:10CA10006071207070BD1022B11C05F1D8000DF0BE
:10CA200075FF042085F8CA000020E9E70220E7E747
:10CA300070B5214C0546207828B1BDE870402E2104
:10CA40000E2000F00BBA2888072100F070FFC8B153
:10CA500090F8CA1029B990F834100F290DD0102978
:10CA60000BD00C2020710E20A0702E20E0702888A2
:10CA7000E08001206071207070BD052180F8CA102F
:10CA80000020EFE70220EDE77CB50B4C054620784F
:10CA900020B137210E2000F0E1F97CBD28886946DD
:10CAA000FEF715FD60B10220207101206071372171
:10CAB000E17020707CBD0000A40700204C00002025
:10CAC00001987F22014680F8302080F83120002232
:10CAD00080F83220A87801F8220FE8784870287989
:10CAE00088702271E1E71CB5F94C217821B113213E
:10CAF0000E2000F0B3F91CBD00886946FEF7E7FC84
:10CB000008B1022005E0019890F82210012902D016
:10CB10000C20207106E0302100222271095C217274
:10CB20000088E080012060711321E1700E21A17066
:10CB300020701CBD2DE9F041E54C0546207828B158
:10CB4000BDE8F04135210E2000F088B9A87808B181
:10CB5000012803D1A888B0F5FA7F01D912202071ED
:10CB60002888072100F0E3FE0126A0B1002780F805
:10CB7000C070A988A0F8C21080F89C60A97801292B
:10CB800000D0002180F8C01090F89D0008B108F096
:10CB90003CFF277101E00220207166713520E070B2
:10CBA0002670C0E42DE9F041C94C0546207828B133
:10CBB000BDE8F0413C210E2000F050B92888072143
:10CBC00000F0B5FE012358B382886D88C68841887D
:10CBD00003EB4207BD4217D342F210777E43BF10EA
:10CBE0007943B6FBF1F1491E89B24FF4FA76B142AE
:10CBF00000D931468D4200D22946491C521CB1FB56
:10CC0000F2F15143491E8AB290F8E81001B902844A
:10CC1000E2800020207163713C20E070237082E488
:10CC20000220F7E770B5AA4C0546207828B1BDE888
:10CC3000704033210E2000F011B908F0D9F908B185
:10CC40000C2017E0297889B10A290FD014290DD0BA
:10CC50001E290BD0282909D0322907D04B2905D00D
:10CC6000642903D0FF2901D0122003E0284608F0F0
:10CC700067FE00202071012060713321E170207077
:10CC800070BD70B5924C0546207828B1BDE8704063
:10CC90003D210E2000F0E2B808F0AAF910B908F022
:10CCA000ADF908B10C2003E0287806F009F900205E
:10CCB0002071012060713D21E170207070BD10B5C0
:10CCC000017801243F2923D2DFE801F0BBBB20BB60
:10CCD000BBBB90BBBBBB2326BBBB414B5DBBBB55AA
:10CCE000BBBBBB2A93BB979BBB7579BB9F7D8184E4
:10CCF00088618CBB59BB514E71A3A7BB362E32B78E
:10CD000069ABBB6D3E3A4465AFB34700FEF7FBFD30
:10CD100098E0FEF72CFE95E0801CFEF76BFE91E09C
:10CD2000801CFFF743F88DE0801CFEF7FFFE89E0D2
:10CD3000801CFEF7F6FF85E0801CFFF716F881E007
:10CD4000801CFEF72DFE7DE0FEF785FE7AE0FEF703
:10CD5000D3FF77E0FEF741FF74E0801CFFF74DF84A
:10CD600070E0FEF79BFE6DE0FEF7CAFE6AE0801CF5
:10CD7000FEF709FF66E0801CFFF7B5FE62E0801C4D
:10CD8000FFF786F85EE0801CFFF725F95AE0801C6B
:10CD9000FFF7F2F856E0801CFEF79EFE52E0801C82
:10CDA000FEF78EFF4EE0801CFFF76EFE4AE0801C0F
:10CDB000FFF790FC46E0801CFFF75AF942E0801C28
:10CDC000FFF7C5F93EE0801CFFF7F1F93AE0FFF705
:10CDD0002AFB37E0801CFFF75CFB33E0801CFFF789
:10CDE000D3FB2FE0801CFFF71EFC2BE0FFF751FC6C
:10CDF00028E0801CFFF7B9FC24E0801CFFF71FFD32
:10CE000020E0801CFFF755FD1CE0801CFFF734FD7F
:10CE100018E0801CFFF7D6FD14E0801CFFF708FE29
:10CE200010E0801CFFF786FE0CE0801CFFF7BAFEC6
:10CE300008E0801CFFF725FF04E0801CFFF7F2FEEE
:10CE400000E00024204610BD10B50C4600F036FB73
:10CE5000002802D022680021117010BD1C4A92F8EF
:10CE60003130002B06D182F8320082F833100120D5
:10CE700082F83100704730B5134606E0CC18D51A59
:10CE800014F8014C5B1E4455DBB2002BF6D130BDCB
:10CE900090F8411041B990F8901029B190F89000A5
:10CEA000042801D0012070470020704701784068B5
:10CEB00021B190F8410010B100207047E8E701204F
:10CEC000704703480021C0F8F81080F8C41070477C
:10CED000A407002001780129F9D1406890F89D103D
:10CEE0000029F4D0002180F89D1008F08EBDEEE7F7
:10CEF0000844C01D453102FB0010704770B51D4647
:10CF00000446A818049B05F14502C01D03FB002040
:10CF100086B2B14238BF0DF0C6FD60686FF30E00F7
:10CF200020F400406060A0686FF30E0020F4004021
:10CF3000A060E0686FF30E0020F40040E060002085
:10CF400020762082A0826082E0826076A576A6F1BB
:10CF500024002080012070BD008870472DE9F04F2B
:10CF600004460E4600F12409D4E902101546C0F328
:10CF70000E02C1F30E080027424509D1C0F3C033A9
:10CF8000C1F3C03193EA010F1CBF0020BDE8F08F50
:10CF9000424518D9A07EA2EB0801091AC91F09B29F
:10CFA0008D422DDCC11D08EB09000144C91E7160D2
:10CFB0003581F7603782011D31600580478001208F
:10CFC0002076BDE8F08F2188A27EA1EB0801891AA6
:10CFD000C91F0FFA81FAC0F30E0BBAF1000F0FDB75
:10CFE000BAF11B0FB8BF0DF05EFD5545D4BF284602
:10CFF0001FFA8AF0291A0A04120C18BF5A4503D9DD
:10D0000027760020BDE8F08FA17ECB1D08EB09013B
:10D010000B44DB1E7360308104F12403F360328221
:10D020000B1D336008804A8001202076BDE8F08F18
:10D030002DE9F041044600F124028068237E3BB1D3
:10D04000C0F30E0010440288438813448B4202D27E
:10D050000020BDE8F081002791429CBF01804780FD
:10D0600019D9891A0E04360C468014D0208904F18F
:10D070000808C0F30E00B04298BF0DF014FD66F32F
:10D080000E05B8F80000012121EAD03060F3CF3559
:10D09000C8F8005009E0A17E0088CB1D184481B279
:10D0A000228804F1080000F07BFA27760120BDE811
:10D0B000F0812DE9F001D0E90143C4F30E0600F13F
:10D0C0002405C3F30E08002706EB050C46450CD1DA
:10D0D000C4F3C034C3F3C033634093F0010F1FBFE8
:10D0E00087820020BDE8F0017047048ABCF8003058
:10D0F0009C4207D3BCF802C0E31AACEB0303A5F1D2
:10D10000030C05E0857E1B1B2C44A4440CF1040C8D
:10D11000C1F800C01188994288BF138011888182AC
:10D12000BDE8F001012070472DE9F04104462430AC
:10D13000A188C1F30E010D18A08A002808BFBDE820
:10D14000F081218A084480B2208229886A881144AB
:10D15000814238BF0DF0A7FC28886F88228AC11948
:10D160004FF0000891421CD18FB1A088261DC0F35A
:10D170000E00B84298BF0DF096FC67F30E0530889C
:10D18000012121EAD03060F3CF35356007E0A17E80
:10D190002288CB1D184481B2201D00F001FAA4F8AA
:10D1A0001080A4F814800120BDE8F08170B5C36838
:10D1B000044600F124058C464068C3F30E01C0F319
:10D1C0000E060D44B14209D1C3F3C031C0F3C030E3
:10D1D000484090F0010F1CBF002070BD002A1CBF0A
:10D1E000281D1060BCF1000F04D0A27E291D6046EE
:10D1F0000DF08CFB6E888EB134F80C0FC0F30E006E
:10D20000B04298BF0DF04FFC66F30E052088012157
:10D2100021EAD03060F3CF35256009E0A07E228876
:10D22000C31D2888184481B204F10C0000F0B8F93D
:10D23000012070BDD0E901104A04B2EB404F09D182
:10D24000C1F3C031C0F3C030484090F0010F1CBFA3
:10D250000120704700207047C16840684A04B2EB63
:10D26000404F09D1C1F3C031C0F3C030484090F005
:10D27000010F1CBF012070470020704770B4D0E937
:10D280000121C2F30E0300F1240CC1F30E049C44EF
:10D29000A34207D1C2F3C035C1F3C0326A4092F055
:10D2A000010F24D1028A858A5619BCF80050BCF8B7
:10D2B000022005EB020C66451CD312B1A24216D225
:10D2C00018E090F81AC0DB1D0CEB05021A44008828
:10D2D00092B2801A80B20CF12203984205D248041F
:10D2E000400C04BF70BC704704E0944202D170BC93
:10D2F0000020704770BC012070472DE9F003D0E991
:10D30000025C00F12406C5F30E04A719CCF30E0845
:10D310000023A04506D1CCF3C039C5F3C03599EA46
:10D32000050F4ED1A0450BD9857EA8EB040CACEBC4
:10D33000050CACF1070C0FFA8CF84FF000090AE06D
:10D34000058890F81A802D1BA5EB0805ED1F0FFA34
:10D3500085F8CCF30E09B8F1000F32DBB0F812C03B
:10D36000BCF1000F08BF00250ED03D887F885FB15B
:10D37000A9EB0704A4B24376944222D30CEB060334
:10D380005B1BDB1E0B600CE0A8EB05073FB243768E
:10D39000974211DB837EB444DB1D23446344DB1ED0
:10D3A0000B60C28209680A88A0F81B20897841773F
:10D3B000BDE8F00301207047914524BF0123437667
:10D3C000DCD2C382BDE8F003002070472DE9F05F96
:10D3D000044600F1240900899246C0F30E0BE08A4E
:10D3E00088460BEB090508B1404502D20020BDE894
:10D3F000F09F608A002804BF00273E4606D02F8891
:10D400006E88B919884218BF0DF04DFB607E50EA56
:10D41000060101D020B32CE0608A50B1A17E4844BF
:10D42000C91D59440844B4F81B1020F8031D617F3E
:10D430008170618A07EB08004144618200262880E0
:10D440006E80BAF1000F33D0A07E2288C31D2888D9
:10D45000184481B204F1080000F0A2F8668227E0C7
:10D46000608AB4F81B104844C01B20F8031D617F7C
:10D47000817006EB080086B2608ABAF1000F404462
:10D4800060822F806E8013D0208904F10807C0F3DA
:10D490000E00B04298BF0DF006FB66F30E0538880B
:10D4A000012121EAD03060F3CF3500203D60608259
:10D4B0000020E08220760120BDE8F09FF0B4D0E9A2
:10D4C0000143C4F30E0500F1240CC3F30E0700263C
:10D4D00005EB0C02BD4207D1C4F3C034C3F3C03323
:10D4E000634093F0010F01D1038A13B1F0BC002017
:10D4F0007047131D0B60807EC31D9818C01E4860C6
:10D5000010880881C1F80CC052880A8220B9ACF199
:10D51000030048600A810E82F0BC012070472DE9AB
:10D52000F041044600F12402D4E90110C1F30E03D6
:10D53000C0F30E0C00271A44634507D1C1F3C03174
:10D54000C0F3C030484090F0010F05D1208A002878
:10D5500004BFA08A002802D00020BDE8F081108816
:10D560005688A6B104F10408B34298BF0DF09BFAA7
:10D5700066F30E05B8F80000012121EAD03060F30F
:10D58000CF35C8F80050A7820120BDE8F081A17E08
:10D590002288CB1D184481B2201D00F001F8F2E76B
:10D5A00030B404680125214461F30E0CE10B61F3F2
:10D5B000CF3CCCF30E0191420FD2511A89B203F144
:10D5C0001B02914205D26FF30E0C25EAD43161F3B0
:10D5D000CF3CC0F800C030BC70474FEAFC31A1EB33
:10D5E00042414FEA714125EAD43262F3CF31016002
:10D5F00030BC704730B5034600255AB1181D18607D
:10D600000023521E04E0441804605B1C2046DBB279
:10D610009342F8DB056030BD024600201168002906
:10D6200002D0084609681160704702680A6001600C
:10D6300070470000F8B50E46054600F0CDF908B970
:10D640000DF031FAF44800EB8607B86A50F825006F
:10D6500008B10DF028FAB868FFF7DEFF040030D0FB
:10D66000B86A082E40F82540204628D2DFE806F0A8
:10D670000404090C0F14172221462846F7F736FD3B
:10D680001FE0F6F7ACFC1CE0F5F79CF919E0214629
:10D690002846F9F7B0F914E0F4F7D6FC11E0DE49BA
:10D6A000DE4B7A31A1F12E0200912146284609F085
:10D6B00042F906E02146284609F033FD01E00DF06D
:10D6C000F2F92046F8BD2DE9F05F8146DDF82880AB
:10D6D0001D4603EB080092468B46C4B25FEA090779
:10D6E00008D00026FF2801D90DF0DDF9BBF1000FAD
:10D6F00004D101E00126F5E70DF0D5F909F10300A9
:10D7000020F00301494501D00DF0CDF9C24501D902
:10D710000DF0C9F966B9C04900204C314FF6FF72CF
:10D7200008704A80BD490870BB497A3108704A8048
:10D73000B94880F800A045708470C47004714471C9
:10D7400080F80680C57100258246B5484FF6FC7109
:10D7500030F81500C01CFF1C00EA010827F0030781
:10D7600046B90AEB8502384697601AF8052041460B
:10D77000FFF740FF1AF805103F1D6D1C08FB0177ED
:10D78000EDB2082DE1D3FF1C4FF0040827F003058C
:10D7900036B9284622464146CAF84850FFF72AFFC4
:10D7A0002D1D18FB045000210A465346C01C20F0D2
:10D7B00003056EB903EB81070020BD6206E000BFE0
:10D7C000D7F828C04CF82020401CC0B2A042F7D3A4
:10D7D000491CC9B205EB84000829E7D3A0EB090076
:10D7E000ABF800000020BDE8F09F10B5B0F5000FC9
:10D7F00006D3B0F1805F05D38A490968884201D217
:10D80000102010BD0278844B418803EB82029B7884
:10D810000EE0946A54F8214044B14B1C438081804F
:10D82000926A52F821108160002010BD491C89B213
:10D830008B42EED84180052010BDB1F5000F06D314
:10D84000B1F1805F05D3774A1268914201D210206E
:10D850007047082801D307207047087000204880CF
:10D8600070470EB56946FFF7E8FF08B10DF01BF9E8
:10D870006846FFF7BAFF08B100200EBD01200EBDBB
:10D8800010B50446082801D30DF00DF96248005D7B
:10D8900010BD3EB5054600246946FFF7CEFF20B116
:10D8A0000DF001F901E0641CE4B26846FFF79DFF4A
:10D8B0000028F8D02846FFF7E3FF001BC0B23EBDAA
:10D8C00010B5044600F088F808B1E0B210BDFF20A2
:10D8D00010BD70B50C460546062901D0072C11D1A4
:10D8E0004D4EB06CFFF798FE4FF6FF7130B1B6F8B1
:10D8F0004820801A001FC0F38D0000E008462880F1
:10D90000884201D1002070BD2146FFF793FE04003C
:10D9100002D1288800F068F8204670BDA0F57F424B
:10D92000FF3A01D0082901D30020704782E6A0F514
:10D930007F42FF3A01D0082901D30020704700F050
:10D940005CB82DE9F0410646A0F57F400C4643F255
:10D950000207FF383ED0082C02D30720BDE8F08133
:10D96000304600F04AF8050034D0082C1CD2DFE81D
:10D9700004F00404090C11161D1D29463046F7F762
:10D98000D4FB13E0F6F73BFB10E029463046F5F7F1
:10D9900041F80BE029463046F9F767F806E02946DA
:10D9A0003046F4F756FB01E00DF07DF81A480021EF
:10D9B00000EB8407062CB86A40F8261001D0072C2B
:10D9C00002D1304600F010F82946B868FFF72DFE66
:10D9D0000020C3E73846C1E70F498978814201D961
:10D9E000012070470020704701460B48042202EBDB
:10D9F0008101806C0144FFF718BE70B50C460546E6
:10DA0000FFF7EAFF002805D0034800EB8400806A96
:10DA100050F8250070BD0000AC0800205200002026
:10DA200098AC01001C0000200146AB4800220068B1
:10DA30000260037A00EB830040F80C2F81801146CE
:10DA400000F042B92DE9F05F9946DDF82CB014469C
:10DA50008A4605004FF0000633D000208046E81CBF
:10DA600020F00300A84201D00DF01DF844B30021BE
:10DA7000084600F025F9671E00FB076600200A999A
:10DA800000F01EF948443044002286B21146104688
:10DA9000F5F79AFA00FB0766002210460C99F5F795
:10DAA00093FA5844304404EB440100EB41000C303D
:10DAB00000EB840000EB840086B2B8F1000F02D0C6
:10DAC00011E00120CAE7A6EB84000C3887B2824837
:10DAD000A10005602C7205F10C0068600CF0AFFF2E
:10DAE0003846FFF7A1FFAAF800600020BDE8F09FCC
:10DAF0002DE9FF4F784C074681B02068934608B95E
:10DB00000CF0D1FF2068017AB94203D9416851F87D
:10DB1000271021B143F2020005B0BDE8F08F006884
:10DB2000F0B358460E9900F0CBF8C51C4FF6FC76C2
:10DB30003540002204990298F5F746FAC01C00EA25
:10DB4000060808EB05002268001DA14686B20021E8
:10DB5000146801E021460446206810B1A388B3424E
:10DB6000F8D1A088B04228D311B122680A6001E040
:10DB70002068106020684FF0000A68B906F10800BC
:10DB800082B2A088904207D9821BA019C0F800A0D9
:10DB9000828000F099F8A680A0886080258000E04F
:10DBA0000BE00E9B201D0093064629465A46012392
:10DBB000FFF7A4F918B1002002E00420ACE704202C
:10DBC000A84201D90CF06FFF2088CDF800A03044A6
:10DBD0004146049B029AF5F7EFF9D9F80000406836
:10DBE00040F82740002097E770B53B4C0546206879
:10DBF00008B90CF058FF2068017AA94210D9426890
:10DC000052F8250060B14188002342F825300360B6
:10DC10008180194600F058F8216800200A7A08E04F
:10DC200043F2020070BD4B6853F820306BB9401CC2
:10DC3000C0B28242F7D8002002E08A88104480B245
:10DC400009680029F9D1FFF7EFFE002070BD70B51B
:10DC5000214D286800280AD0002404E02046FFF760
:10DC6000C3FF641CE4B22868007AA042F6D870BDF5
:10DC700070B5194E05460024306808B90CF013FF42
:10DC80003068017AA94204D9406850F8250000B1F3
:10DC9000041D204670BD70B50F4E05460024306847
:10DCA00008B90CF000FF3068017AA94206D9406833
:10DCB00050F8251011B131F8040B4418204670BDFE
:10DCC0000A460121FFF714B919B10A680260086019
:10DCD000704701490968F8E7580000202DE9F04134
:10DCE00007780D460446012F19D0072F02D00C2FBC
:10DCF00019D114E0A068216906780B2E0BD00520FD
:10DD000003F085FE052E0ED0782300220520216920
:10DD100003F0DFFD07E0782300220620F8E7052066
:10DD2000216903F074FE7DB1002028702946204649
:10DD3000F6F7BAFFF6482978C05D884202D1032081
:10DD4000BDE8F0810220FBE700212046F6F7ACFF9A
:10DD50000020F5E730B50C4691F8281089B015463B
:10DD6000012049B1012905D12978042902D10520D2
:10DD70001070002009B030BD60680590CDF818D053
:10DD80000D210DF103000CF038FEA0680188ADF8FC
:10DD9000001080788DF80200012084F82800062009
:10DDA0008DF81000606A0890294604A8FFF796FFD6
:10DDB000E0E770B50C46012091F8281086B01546B2
:10DDC000062661B3012928D12978042925D169685B
:10DDD0001022A06801F0BFFB6868C07B000606D572
:10DDE000CB4AA0681023103A014601F0A9FBD4E900
:10DDF0000210102201F0AFFBA068C07B000606D520
:10DE0000C34AE0681023103A014601F099FB2E70D6
:10DE1000A0686860E068A860002006B070BD606817
:10DE20000190BB48114620380290012084F8280058
:10DE30008DF80060606A04906846FFF74FFFECE7DA
:10DE4000027B032A06D0002281F828200B780D2BB4
:10DE500002D003E0042070470A76CA61027B930077
:10DE6000521C0273C150032070472DE9F0410C464B
:10DE700003461546012091F8281092B007224FF072
:10DE8000060861B1012925D0022930D0032904D127
:10DE90002978042901D12A70002012B050E701200E
:10DEA00084F82800606870B1A1690A7060684860F1
:10DEB000206988606069C860606A486212B018466C
:10DEC000BDE8F041BCE785F80080206968606069C2
:10DED000A8600AE029780629DFD1022084F828000A
:10DEE000042028708A48203868600320D5E7297804
:10DEF0000429D2D1A08910280CD9A0F1100080B239
:10DF0000A081A1684FF01003014468466A6801F0DF
:10DF100017FB27E004D14FF010032269A16815E038
:10DF2000C2B20DAEC2F1100707EB0600A1680CF0FB
:10DF3000EDFC17F0FF0006D0401EC1B280207054E7
:10DF400030460CF05AFD626910230DA904A801F0B7
:10DF5000F7FA102304A968466A6801F0F1FA032071
:10DF600084F8280060680990CDF828D08DF82080CA
:10DF7000606A0C90294608A8FFF7B0FE8DE72DE9EE
:10DF8000F04107460D46012091F8283008213BB1A9
:10DF9000012B04D11378072B01D111700020CFE69B
:10DFA0006C69012620222170E8686060686A6062FE
:10DFB000A168287C0870A681A068A968401C0CF0A4
:10DFC000A5FCA08920222030A081A06869682130AA
:10DFD0000CF09CFCA08921462030A08185F82860A7
:10DFE0003846BDE8F0412BE72DE9F05F0C4681464D
:10DFF000012091F82810174606464FF00808D1B1C5
:10E00000DFF80CB14FF0000AABF12C0B012924D042
:10E0100002297FD003290CD13978072909D17968E1
:10E020001022E0690CF072FC0920387018340020CE
:10E030007C60BDE8F09F216A354881F800800E3091
:10E04000486020208881606A4862E26988681060C0
:10E050006068886084F82860B6E039780729E8D1DC
:10E06000256A85F80080606A6862E0690068A860D7
:10E0700051681022E0690CF049FCE0696860A8680A
:10E08000574680F800A0AE81A8684670A889401C59
:10E0900080B2A881A968084461690A6802608A8818
:10E0A000828089798171A889C01D80B2A881A96800
:10E0B000084421690A6802608A88828089798171AE
:10E0C000A8891022C01D80B2A881A9680844E1680F
:10E0D0000CF01CFCA8891022103080B2A881A9681D
:10E0E0000844A1680CF012FCA889103080B2A88105
:10E0F000A9680144DBF808000860A889001D80B207
:10E10000A881A9680F54A889401CA881022058E062
:10E11000D4AC0100FFE7397807298AD15168102271
:10E12000A0690CF0F3FB256A85F80080E06968605F
:10E13000606A6862A96881F800A0AE81A86846702C
:10E14000A889401C80B2A881A968084461690A684E
:10E1500002608A88828089798171A889C01D80B215
:10E16000A881A968084421690A6802608A888280B7
:10E1700089798171A8891022C01D80B2A881A968FF
:10E180000844E1680CF0C2FBA8891022103080B26C
:10E19000A881A9680844A1680CF0B8FBA8891030D0
:10E1A00080B2A881A9680144DBF808000860A8894A
:10E1B000001D80B2A881A9680E54A889401CA881BE
:10E1C000032084F8280029464846BDE8F05F37E67A
:10E1D00070B50D46064691F82810012041B101297D
:10E1E00005D11178072902D10A201070002070BDD6
:10E1F0002C6A0820207068686060686A6062E9695B
:10E20000A0680A6802608A88828089798171072003
:10E21000A081A969A2680B68D01DC2F807308A885E
:10E22000828089798171A089C01D80B2A081A16896
:10E23000084469690A88028089788170A08910225F
:10E24000C01C80B2A081A168084429690CF05EFB63
:10E25000A0891022103080B2A081A1680844E9682A
:10E260000CF054FBA0891022103080B2A081A1686C
:10E270000844A9680CF04AFBA08921461030A0810F
:10E28000012085F828003046BDE87040D8E570B51B
:10E290000D46064691F82810012069B101290AD1DE
:10E2A0001178072907D15068002141608160C16061
:10E2B0000B201070084670BD6C6908201022207079
:10E2C000E8686060686A60622969A0680CF01EFBFB
:10E2D0001020A081A06820221030A9680CF016FB45
:10E2E000A0892022203080B2A081A16808446968FA
:10E2F0000CF00CFBA08921462030A081012085F87C
:10E3000028003046BDE870409AE570B50C46012003
:10E3100091F828108EB01546062659B1012931D042
:10E32000022905D12978042902D10C20107000207F
:10E330000EB070BD217D102301F00100C1F340013A
:10E340008DF800008DF80110E0686A460168CDF88C
:10E3500002108188ADF8061080798DF808002069D8
:10E360000168CDF809108188ADF80D1080798DF81D
:10E370000F006068059009A80690A16801F0E0F818
:10E3800001201BE029780429D2D1E06910236A46D4
:10E39000016800918088ADF80400A0690168CDF89B
:10E3A00006108088ADF80A00002003906068059090
:10E3B00009A80690696801F0C3F8022084F82800D3
:10E3C0008DF81060606A0890294604A8FFF786FC63
:10E3D000AEE700B591F8283089B001204BB1012B90
:10E3E00005D11178042902D10D201070002009B048
:10E3F00000BD4868019005A80290C86803680593AD
:10E400004068069088680368079340680890012078
:10E4100081F8280006208DF80000486A0490114613
:10E420006846FFF75BFCE2E700B591F8283089B059
:10E43000012043B1012BDAD111780429D7D10E2064
:10E4400010700020D3E74868019005A80290886802
:10E45000036805934068069000200790089001200B
:10E4600081F8280006208DF80000486A04901146C3
:10E470006846FFF733FCBAE700B591F8283089B059
:10E48000012043B1012BB2D111780429AFD10F2063
:10E4900010700020ABE748680590CDF818D0886868
:10E4A0000088ADF80000C8680088ADF802000020C0
:10E4B000019002900390012081F8280006208DF839
:10E4C0001000486A0890114604A8FFF707FC8EE781
:10E4D00030B4034691F8284001205CB1012C16D0DD
:10E4E000022C05D111780E2902D1102010700020C5
:10E4F00030BC7047012081F82800C86805220270EE
:10E500004A684260FD4A8260921CC2600CE0147846
:10E510000F2CEDD1022081F82800C8680424047073
:10E52000526842608A688260496A4162014630BC32
:10E53000184685E410B500F1310283799478011D05
:10E5400064F0030423408371DB070DD04B795479C9
:10E5500023404B710B79127913400B718278C97883
:10E560008A4200D9817010BD00224A710A71F5E714
:10E570002DE9F74F86B000208DF8000016460C46B6
:10E5800091F82800012518210E220B274FF0190BB6
:10E590004FF0110A4FF00A094FF01C081F2879D2DA
:10E5A000DFE800F010FCFBFAF9F8F7F6F5F4F3F207
:10E5B000F1F0EFEEEDECEBEAE9E8E7E6E5E4E3E2C3
:10E5C000E1E0DF00606910B1007813287ED0A76811
:10E5D000002F5FD001208DF80000606A04900320B6
:10E5E0008DF804008DF80590E069029020790028EC
:10E5F000EFD03A78002AE9D00C2A67D267D2DFE858
:10E6000002F066164A8FD3F8F7F6F5F4F3060228FF
:10E6100040D1606910B10078082857D102208DF8E8
:10E620000000606A049078788DF8040038E20620D3
:10E63000616A03F0ECF920790728E9D1606900F0FC
:10E64000ADFF02280BD0606900F0A8FF042806D0B7
:10E6500060690028BDD000780128D9D102E0616945
:10E66000012008703879C11F0A2902D384F8189054
:10E67000F4E361698870606939680163B9888186EB
:10E68000B97980F83610012084F8280061690320E8
:10E69000087037E03DE20728BAD16069002898D0B9
:10E6A00001780929B4D1F978890705D17979002948
:10E6B000DCD1B9790029D9D1797990F83520914305
:10E6C000D4D1B97990F83620914301E07DE2A2E1FE
:10E6D000CCD13979CA1F0A2AC8D290F824208A429C
:10E6E00002D906202076B9E3396840F8031FB988BB
:10E6F0008180B9798171012084F828006169032043
:10E7000081F800908DF80000606A049060693130F3
:10E7100001906069001D029060691C300390CEE298
:10E7200011288AD1606900F039FF042804D060699B
:10E7300000F034FF0B2890D160691022791C37302B
:10E740000CF0E4F86069017804292BD190F82410CA
:10E7500082789142C5D805210170032084F82800F1
:10E760001DE0F1E3F1E3F1E3F1E3F1E3F1E3F1E3E0
:10E77000F1E3F1E3F1E3F1E3D9E3A0E352E32BE3C7
:10E78000FAE2EDE2DCE2A7E29AE280E256E220E27F
:10E79000FBE1C8E1B7E196E183E166E13EE18DF896
:10E7A0000010E8E2082089E31128BAD1606900F07E
:10E7B000F5FE062804D0606900F0F0FE0C28B0D108
:10E7C000E068B8B12069A8B160690178062915D060
:10E7D0000D21017060691022791C57300CF096F8F9
:10E7E000606957300921A9E1E0E0B8E096E049E02E
:10E7F00027E00EE000208DF800008AE1072101707B
:10E8000060691022791C47300CF080F8606947304D
:10E81000E8E70228F1D1606900F0C0FE0028ECD0E2
:10E82000606900F0BBFE0128E7D0606900F0B6FE29
:10E830000828E2D005208DF8040078788DF80500CE
:10E8400067E11128D9D160690028D6D001780E2956
:10E85000D3D1C16A4078022812D0002000EB80009A
:10E86000142202EB800010220858791C0CF04EF89C
:10E870000520616A00F07FFE61690F200870A4E145
:10E880000120EBE70B28B8D160690028B5D00178EA
:10E890000F29B2D1C16A4078022831D05FF0000060
:10E8A00000EB80020C2000EB82000858B7F8011042
:10E8B00001806069C16A4078022824D05FF00000BE
:10E8C00000EB8000102202EB8000085857F8031F6D
:10E8D0000160796841600520616A00F04CFE606962
:10E8E0004178022912D04FF0000100BF01F1080168
:10E8F000415C21F001027BD08AE00000AAAC01005B
:10E900004FF00100CCE74FF00100D9E74FF00101D3
:10E91000ECE700BF01F1080142540EE211288FD14B
:10E92000606900288CD00278102A89D1C26A4078A8
:10E93000022812D05FF0000000EB800001EB8000A5
:10E94000791C105810220BF0E1FF0520616A00F0DD
:10E9500012FE616981F800A0DBE30120ECE70828E2
:10E9600091D16069002891D0017811298BD1C06ABA
:10E97000797801706069D7F80210C06A40F8011F09
:10E98000F98881800520616A00F0F5FD60694178B1
:10E99000022908D04FF0000101F10801415C21F08B
:10E9A00002022CD034E04FF00101F5E71128B6D176
:10E9B00060690028B6D001781229B0D1C16A4078C8
:10E9C00002281FD05FF0000000EB800008EB800001
:10E9D00010220858791C0BF099FF0520616A00F09D
:10E9E000CAFD6069417802290FD04FF0000100E0B4
:10E9F00005E001F10801415C21F0040208D14FF06B
:10EA0000010187E74FF00100DEE74FF00101EEE77B
:10EA10004FF000017EE74FF0070063E630780128F1
:10EA20009ED16069716814221C300BF0B4FF6069DC
:10EA3000017F09B12176C9E30178032901D00320C0
:10EA400094E10225C570817921F0F8018171017A84
:10EA500021F0F8010172417A21F0F80141726069F8
:10EA6000FFF768FD84F82850A5E230781328E2D13A
:10EA700007208DF80000616A0491B1688DF80400E8
:10EA800002910846616951F8032F02608A888280EA
:10EA900089798171616904200870002084F8280058
:10EAA000ADE330780328C6D1606901780529716823
:10EAB0000A6805D040F8472F49684160042055E1B5
:10EAC00040F8572FF8E730780328B4D1606901780F
:10EAD000052971680A6811D040F84F2F49684160D4
:10EAE000052084F828006069006A50B10220307067
:10EAF000002030716069006AB0609FE240F85F2FCB
:10EB0000ECE7042035E13078022894D1307908B15F
:10EB100020765BE36069B1680162606909B9FA490E
:10EB2000016206207CE23078132884D1B068E0616D
:10EB300060690178052926D04730072184F828101C
:10EB4000E16802220A706269126AC1E90120606903
:10EB50003030C8606069C01C08616069806A0278F2
:10EB6000087D62F3000008756269926A521C8A612E
:10EB70006269D26A127862F3410008756069C06AFE
:10EB8000401CC8616FE25730D7E730780C28C0D1FD
:10EB900060690178052919D0077007208DF80000F9
:10EBA000606A0490E06902908DF804A0032100F8E7
:10EBB000011B102271680BF0A9FE00216846FFF7C7
:10EBC0008DF8002084F82800E061A2E2062101709F
:10EBD000E3E7307813289CD107208DF80000606AA5
:10EBE0000490B06802908DF804A00421017061695E
:10EBF0000A78072A0BD0002284F828200C220A70F9
:10EC000061691022401C47310BF080FEF7E21022B0
:10EC1000401C57310BF07AFE00216846FFF75EF882
:10EC200084F82890E168032008706069006A4860F1
:10EC30006069573088606069473013E230780C288B
:10EC4000A5D160697168102237300BF033FE08B12E
:10EC5000042047E56069007807283FF4A3AD84F8F5
:10EC60002890E168032008706069006A4860606964
:10EC70005730886060694730C860606A48620698AB
:10EC8000FFF7DEF805466069FFF754FC8DE2307847
:10EC90000D28A0D184F828706169706889780844CB
:10ECA000C1F110010BF0A9FE08208DF80000606A88
:10ECB000049070680190606980788DF808007DE1AB
:10ECC0003078112887D160698079C0077AD00C200C
:10ECD00084F8280009204CE030781228B0D160690F
:10ECE0001422311D1C300BF056FE6069018DC06A84
:10ECF000A0F8091060698178C06AC1716169081D56
:10ED0000CA6A117A21F07F0111724379626919434D
:10ED10008378D26A03F00303012B00D0002300792B
:10ED20009B0143EAC00001431172606940780128E9
:10ED300077D002E084F8280080E184F828B07DE1F3
:10ED400060694178022901D0012100E000210831E9
:10ED5000405CC00702D084F828202CE11320E9E7AA
:10ED60003078132895D1B068E0610F2084F828002E
:10ED700005208DF8000056E13078032889D16069BC
:10ED8000C16A4078022801D0012000E0002000EB99
:10ED90008002102000EB820273688A5819681160A3
:10EDA0005968516084F82800D4E9031306220A70D8
:10EDB0006269526A4A606269D56A5278022A02D050
:10EDC000012201E0B4E1002202EB820200EB8200AA
:10EDD0002858C1E9020346E130781028C2D16069A1
:10EDE000C26A4078022801D0012000E0002000EB38
:10EDF00080010C2000EB8100022310580932716859
:10EE000000F09EFB84F828A0E16805200870606986
:10EE1000006A48606069C06A093088603A4808380A
:10EE200020E17AE130780F289CD161694A78C86A7C
:10EE3000022A01D0012200E0002202EB8202142506
:10EE400005EB820280588A7871680BF05FFD60697B
:10EE50004278C16A022A02D0012201E0B8E1002210
:10EE600002EB820205EB82028A5881785018C1F1C8
:10EE700010010BF0C2FD07208DF80000606A0490BD
:10EE8000E06902908DF804A0062101706169CA6AE8
:10EE90004978022901D0012100E0002101EB810124
:10EEA00005EB8101401C515810220BF02FFD002171
:10EEB0006846FEF713FF0020E0611220B0E03078D2
:10EEC000132877D107218DF80010606A0490B0688C
:10EED00002908DF8047001706169CA6A497802294C
:10EEE00001D0012100E0002101EB81030C2101EBA5
:10EEF000830151580988A0F801106169CA6A4978EC
:10EF0000022903D0012102E0B4AC0100002101EB91
:10EF10008101102303EB810151580A6840F8032F47
:10EF20004968416000216846FEF7D8FE16E760692F
:10EF30004178022901D0012100E000210831405C24
:10EF400080070CD514206BE0F4E0EEE0E7E02FE161
:10EF500002E1CAE08DE073E056E034E001E0162003
:10EF6000E8E63078132825D1B068E06107208DF8F5
:10EF70000000606A0490E06902908DF804A0082205
:10EF800002706269D36A5278022A01D0012200E03D
:10EF9000002202EB820201EB820110225958401C30
:10EFA0000BF0B4FC00216846FEF798FE0020E061FB
:10EFB000152035E083E08DF8009034E03146684656
:10EFC000FEF78CFE32E03078132878D107208DF8D8
:10EFD0000000606A0490B068029008208DF8040078
:10EFE0000298092101706169C969097841706169F4
:10EFF000C96951F8012FC0F802208988C180002119
:10F000006846FEF76BFEAAE760694178022901D0E5
:10F01000012200E000220832805C400708D517205A
:10F0200084F82800C7E7606A0490C7E70546BCE09B
:10F0300001293FF472AC00BF84F828800325E3E087
:10F04000307813283BD1B068E06184F82810E1687B
:10F05000052008706069006A48606069C06A09300C
:10F060008860F748C860606A48620698FEF7E8FE64
:10F07000DCE730780F2822D16069C16A4078022825
:10F0800001D0012000E0002000EB800008EB8000B0
:10F090001022085871680BF039FC07208DF8000029
:10F0A000606A0490E06902908DF804A080F80090F6
:10F0B0006169CA6A4978022902D0012101E04AE067
:10F0C000002101EB810108EB8101401C5158102205
:10F0D0000BF01CFC00216846FEF700FE0020E061FA
:10F0E000606940780128A7D127E660694378022B40
:10F0F00007D000210831415C69B1CB0703D0027011
:10F1000007E00121F6E7890701D5102100E012216F
:10F110000170002578E0012B8ED00D200AE61D201D
:10F1200084F828008DF800707DE7307814284DD1E0
:10F130001E20FFE561690878012847D0082845D0DE
:10F14000002084F82800084600F022FA0C208DF8F0
:10F150000000606A049039E030784FF01B081328F3
:10F1600005D014203070032584F828804CE0072057
:10F170008DF80000606A0490B068029002208DF85B
:10F180000400029805210170217E4170002168462B
:10F19000FEF7A4FD8DF80070606A04903146684661
:10F1A000FEF79CFD054684F82880012D0ED02BE04B
:10F1B00001208DF80000606A049004208DF804009E
:10F1C000207E8DF805000020207611E0207E78B1A9
:10F1D0006169132008701A2084F828008DF80090C7
:10F1E000606A049031466846FEF778FD05460BE0FC
:10F1F000606908B1142101709DF8000020B1002160
:10F200006846FEF76BFD84E709B02846BDE8F08F3D
:10F210002DE9F047012691F8280086B091460C466A
:10F22000B04620B1012828D002281CD19BE02079CB
:10F23000012804D0022811D0032814D10AE0A068C4
:10F24000407801280ED10620616A02F0B9FB00283F
:10F2500009D10CE0A1681320087008E0A06841788B
:10F26000022901D0052676E00078082873D184F8B9
:10F2700028800A208DF8000033E099F80000132858
:10F2800069D107208DF80000616A0491D9F808500F
:10F290000295217902274FF00B0A012904D0022997
:10F2A00027D0032957D10EE08DF8047085F800A00F
:10F2B000207B002100F0070068706846FEF70EFD15
:10F2C000A068077046E08DF8047005202870207B48
:10F2D000687000216846FEF701FD84F828708DF8FB
:10F2E00000A0606A049049466846FEF7F7FC0646AF
:10F2F00031E08DF8040085F80080207C6870607C27
:10F3000000F00100A870A07C00F00700E870E17C2C
:10F310002971C00723D0207D00F007006871607D4F
:10F3200000F00700A87100216846FEF7D7FCA0682E
:10F3300029680163A9888186A97980F83610E06878
:10F34000A168007A81F82400A16828798870A168F2
:10F3500009200870002606B03046BDE8F08700207E
:10F36000A8716871DFE7A168142008708DF800802B
:10F37000606A049004208DF80400207B8DF805005D
:10F3800000216846FEF7AAFCE4E7F0B585B00F4619
:10F3900005460124287B05EB800050F8046C30788A
:10F3A000411E0E290AD226493A46463101EB800019
:10F3B000314650F8043C2846984704460CB1012CCD
:10F3C00011D1287B401E10F0FF00287301D00324C8
:10F3D000E0E70D208DF80000706A0490002101968E
:10F3E0006846FEF77BFC032CD4D005B02046F0BD68
:10F3F00070B515460A46044629461046FFF7C5FF74
:10F40000064674B1207814280BD1207E30B100203C
:10F410002870294604F10C00FFF7B7FF204600F0E2
:10F42000B7F8304670BD704710B5012903D00229E6
:10F4300001D0052010BD417000F0AAF8002010BDD9
:10F44000AEAC010028B1027E1AB10A4600F10C01EF
:10F45000CEE70120704730B5044687B00D46062040
:10F4600002F0D5FA2946052002F0D1FA20781428B6
:10F4700006D000208DF8000069462046FFF7E2FF25
:10F4800007B030BD7FB50E4600218DF80C10017815
:10F490000D2903D00E2903D0002405E0446900E0C3
:10F4A00084680CB1217E91B16D4601462846FEF775
:10F4B000C7FC032809D1324629462046FFF798FFAA
:10F4C0009DF80C10002900D0042004B070BD04F198
:10F4D0000C05EAE700B50023012285B005280FD00E
:10F4E00006280BD102208DF8002004918DF804002D
:10F4F0008DF8053000216846FEF7F0FB05B000BD31
:10F500008DF8002004918DF80420F1E710B592B039
:10F510000C460790244808900521001D8DF818100E
:10F5200009900F92694606A8FFF7ACFF002805D1A5
:10F530001022204601990BF0E9F9002012B07EE775
:10F5400030B505E05B1EDBB2CC5CD55C6C40C454CE
:10F55000002BF7D130BD10B5002409E00B78521E06
:10F5600044EA430300F8013B11F8013BD2B2DC0945
:10F57000002AF3D163E770B50C46054602F047FA5E
:10F5800021462846BDE870407823002202F0A1B948
:10F590004178012900D008210170704708B1007836
:10F5A0007047082070470000A8AC010070B50D46F8
:10F5B000040011D085B1210128460BF01EFA10225B
:10F5C0004F4928460BF0A2F94D4801210838018027
:10F5D00044804560002070BD012070BD70B5484E6C
:10F5E00000240546083E10E07068AA7B00EB04107A
:10F5F000817B914208D1C17BEA7B914204D10C22EC
:10F6000029460BF057F930B1641C30888442EBDB9B
:10F610004FF0FF3070BD204670BD70B50D4606003E
:10F6200009D045B1364C083C20886188401C88428E
:10F6300003D9042070BD102070BD3046FFF7CEFF07
:10F64000002801DB401C0AE021886068102200EBE2
:10F65000011031460BF05AF92088401C2080287098
:10F66000002070BD70B514460D0018D0BCB100214B
:10F67000A170022802D0102811D105E0288870B1AD
:10F680000121A170108008E02846FFF7A7FF00289D
:10F6900005DB401CA070A8892080002070BD0120DF
:10F6A00070BD70B5054614460E000BD000203070BA
:10F6B000A878012808D005D91149A1F108010A88C4
:10F6C00090420AD9012070BD24B128782070288882
:10F6D000000A5070022008700FE064B149681022DF
:10F6E00001EB0011204610390BF010F92878207337
:10F6F0002888000A607310203070002070BD000060
:10F70000640000202DE9F041FE4C207EE17D88421E
:10F7100008BFBDE8F0810126FB4D0027E07D215C9C
:10F7200001EB810205EB8200037C052B10D0037CEA
:10F73000062B1BD0037C072B27D0437C012B32D018
:10F740000BF0B1F9207EE17D8842E7D1BDE8F08180
:10F750000674E07D16281ABFE07D401C0020E0758D
:10F76000481CC0B255F8222002210CE00674E07D4E
:10F7700016281ABFE07D401C0020E075481C55F893
:10F780002220C0B203219047DCE70674E07D1628F2
:10F790001ABFE07D401C0020E075481CC0B255F83F
:10F7A00022200821EFE74774E07D16281ABFE07D8C
:10F7B000401C0020E075481CC0B255F822200721EB
:10F7C000E1E770B5D14E00240C2086F82900A6F59B
:10F7D0003B70254680F8CD4180F8CC4100F5F470AF
:10F7E0000476C47506F12C0009F084FFA6F58E702E
:10F7F000057586F82B50601EB06086F8255086F897
:10F80000225086F8235086F8245086F82150C048AC
:10F8100005704570A6F1E80004EB840100EB81015E
:10F820000D74611CCCB20B2CF6D30120F9F71BFA36
:10F830000020F9F718FA012086F82600F9F7C0FD34
:10F84000B448F9F7CCFDB44C2070B448F9F7C7FDC3
:10F850006070BDE87040F9F799B910B5F9F7C4F9CF
:10F86000AD4C2078F9F7D5FD6078F9F7D2FDA74CBB
:10F8700094F82800002808BF10BDF9F7A6FB002067
:10F8800084F8280010BD70B5F9F796FA9F4C05462C
:10F8900094F8260010B10BF006F970BD94F82B0017
:10F8A000002808BF0BF0FFF86FF07F426069002668
:10F8B000291AB1F5800F24BF431BB3F5800F0BD37A
:10F8C0008A4203D2101A2844411C05E09A4239D2D8
:10F8D000511B0844401C4142002901DB0BF0E3F8B6
:10F8E000012584F8265084F82B6094F82910042010
:10F8F000854A01EB810102EB81010874A068B0F137
:10F90000FF3F04D0A81EA0600120F9F7ACF9002049
:10F91000F9F7A9F9F9F78CF909F0D8FFF9F7C8FA5E
:10F920007F48066006604FF0E0214FF40040C1F8C8
:10F930008002F3F7F5FA76480078022808D0032809
:10F9400003D008E00BF0AFF8C8E794F8230010B13B
:10F9500084F8225001E084F82260BDE87040F9F795
:10F960008BBA034668490B2000EB800201EB820250
:10F9700012F8042C22B1401E10F0FF00F4D17047A1
:10F9800000EB800201EB8201012241F8143C01F8F6
:10F99000042C7047012804D0032808BF002926D072
:10F9A00000E021B3594B4FF0000C83F821C0584AB6
:10F9B0000028907014BF022882F803C00BD00729DA
:10F9C00015D2DFE801F01404060C0E1012001B2003
:10F9D00000E03A20D070012083F8210070475820C1
:10F9E000F8E77720F6E79620F4E7B520F2E7002065
:10F9F0007047474810B54078F9F764FA80B210BDF7
:10FA0000421E10B5404900EB800001EB80040A2A39
:10FA100002D814F8040C08B90BF045F814F8040CDB
:10FA2000012818BF0BF03FF8002004F8040C10BDAB
:10FA300070B53C4C94F8CD0194F8CC1188420CBFC1
:10FA400001250025F9F7B8F9F9F73CFA94F8CD113A
:10FA500094F8CC2191420CBF01210021A942E9D1A7
:10FA600070BD2DE9F05F8046A1F1010C17460CF046
:10FA7000FF04254804EB840200EB82052E1D287C40
:10FA8000DFF8809007282BD199F8170000224B4609
:10FA900099F818A0824521D013F800A0A24508BF0C
:10FAA000012200D04AB116280CBF4FF0000A00F125
:10FAB000010A13F80AA003F800A016280CBF0020C2
:10FAC000401CC0B293F818A08245E5D132B1187E2F
:10FAD00000280EBF1620187E401E187601202874BC
:10FAE000BCF10A0F23D8084801EB810100EB81002B
:10FAF00010F8040CD8B1287C01281AD0287C0128E1
:10FB000015D011E0200B00203C0B0020240C00201D
:10FB100076000020791701007400002005F700002E
:10FB200000F5004038090020B87A012804D00AF016
:10FB3000BAFFB87A01284BD1FE4B287C022818D096
:10FB400099F8180016284BD099F8180099F8171052
:10FB5000401C884202D100BF0AF0A5FF0120687452
:10FB600099F8180009F8004099F8180016283CD0B8
:10FB70003DE0F14A92F829000146A04207D0014633
:10FB800000EB810003EB8000807CA042F7D192F86B
:10FB900029C084450CD192F8291001EB810103EBB7
:10FBA0008101897C82F82910012182F82A1009E05C
:10FBB00000EB800203EB820201EB810103EB810188
:10FBC000927C8A7400EB800003EB80000C2181742E
:10FBD000387A062825D2DFE800F012211E1B1815FE
:10FBE00099F817000028B9D1B6E7002002E099F88B
:10FBF0001800401C89F818000020BDE8F09F4FF065
:10FC0000000A12E04FF0B40A0FE04FF0730A0CE064
:10FC10004FF0320A09E04FF00A0A06E04FF0060AF8
:10FC200003E00AF040FF4FF0000A3868A0EB0A003A
:10FC30003060397A00290CBF04210221401A20F0DB
:10FC40007F423260D7E90001084420F07F407060B5
:10FC5000B87A022818BF387B7ED1387A00280CBFCA
:10FC60000420022000EB0A037868991D00EB010BC9
:10FC7000B2484078504503D9AF4991F8231011B1EB
:10FC80000BF1060003E0A0EB0A005844801DAA49CE
:10FC900091F829C0BCF10C0F24D08E4691F82910A0
:10FCA00001EB810CA34901EB8C0CDCF804C062452C
:10FCB00018D0DFF88CC29EF8292002EB820201EBFB
:10FCC00082014A688968A2EB080222F07F42A1EB18
:10FCD000080121F07F41904298BFB2F5800F48D2D1
:10FCE0008C4546D34044A0EB0B0020F07F413160AF
:10FCF0001944F86821F07F410B1A6FF07F42B3F589
:10FD0000800F24BFA0EB010CBCF5800F0BD39A42EF
:10FD100003D2101A0844431C05E0624520D2511A50
:10FD20000844401C4342002B1CDD0520287499F830
:10FD3000180016282ED099F8180099F81710401CB2
:10FD4000884201D10AF0AFFE99F8180009F8004086
:10FD500099F81800162800E00AE07FF448AF44E75D
:10FD60000AF0A1FE3068584420F07F407060002007
:10FD700030727068801D20F07F407060787AB072B9
:10FD8000387A0627707203280DD260B101F04EFA5E
:10FD900028B108E099F817000028D5D1D2E7CAF1B8
:10FDA00038074FF0320A65480178012918BF032946
:10FDB0000AD14078504507D95F4991F823100029AE
:10FDC00004BFA0EB0A000744DFF874C13068716813
:10FDD000A0EB080323F07F40A1EB080121F07F4254
:10FDE000874298BFB0F5800F1CD294451AD3524871
:10FDF00090F829200C2A34D090F829704FF00C0B81
:10FE00004FEA0B0A4B4807EB870200EB8202D2F85D
:10FE100008C0ACEB080C9C4534D8BB46977C0C2F33
:10FE2000F0D19FE00520287499F81800162813D007
:10FE300099F8180099F81710401C884202D100BFA9
:10FE40000AF031FE99F8180009F8004099F81800F6
:10FE500016287FF4CCAEC8E699F817000028F1D137
:10FE6000EEE70221297490F829100C2918BF90F8A8
:10FE70002910A97480F82940012180F82A10084629
:10FE8000BDE8F09F0C2F1CBFBA4600226AD000BF0D
:10FE90000AEB8A0300EB8303D3F804C0ACEB080C35
:10FEA0008C4529D29A7B96F80AC094451DD305202B
:10FEB000287499F81800162812D099F8180099F8A3
:10FEC0001710401C884201D10AF0EDFD99F8180086
:10FED00009F8004099F8180016287FF488AE84E6E7
:10FEE00099F817000028F1D1EEE793F812A001224B
:10FEF000BAF10C0FCCD103E0002A08BFBA4631D0CA
:10FF00003E460C4806EB860200EB8208062188F884
:10FF1000101099F81800162837D099F8180099F899
:10FF20001710401C884201D10AF0BDFD99F8180055
:10FF300008E000003C0B0020240C0020760000208C
:10FF4000FFFF3F0009F8006099F8180016280EBF5F
:10FF5000002099F81800401C89F8180098F81260E1
:10FF6000B245CED10220FE4E287406F1E80090F88A
:10FF70002910B9420ED185F812A080F8294001213C
:10FF800080F82A100120BDE8F09F99F8170000289A
:10FF9000CCD1C9E70C2F0CD0BBF10C0F08BF0AF075
:10FFA00082FD0BEB8B0006EB8000847485F812A0B9
:10FFB000E8E7BBF10C0F08BF0AF075FD0BEB8B00F7
:10FFC00006EB800084740C20A874DBE730B50D4686
:10FFD000E44A44190021101A71EB010038BF0AF0FD
:10FFE00062FDE1488542C8BF0AF05DFDDF488542F9
:10FFF000B8BF0AF058FDDE488442A8BFDD4804DAE5
:020000040001F9
:10000000002CAABF2046DA4830BD201830BD401E63
:1000100070B5C0B200EB8001D14800EB8104607B79
:10002000062810D2DFE800F0030D0B0907050020B9
:1000300037E0B4200CE073200AE0322008E00A2008
:1000400006E0062004E00AF02EFD617B002041B3AB
:10005000022108446168084420F07F40F8F732FF2D
:1000600094F90C50BF4A44190021101A71EB010099
:1000700038BF0AF018FDBC488542C8BF0AF013FD1E
:10008000BA488542B8BF0AF00EFDB9488442A8BFFD
:10009000B84804DA002CAABF2046B54870BD201825
:1000A00070BD0421D5E72DE9F04F0646B24885B072
:1000B0000068C005C00D11D0103840B20028B8BF8C
:1000C00000F00F0000F1E020B4BF90F8140D90F89C
:1000D0000004400908BF4FF0010A01D04FF0000AA8
:1000E0003078002817BF01283079002005B018BFEC
:1000F000BDE8F08F062810D2DFE800F0030D0B09F1
:100100000705002016E0B4200CE073200AE032203E
:1001100008E00A2006E0062004E00AF0C4FC317979
:10012000002039B15FF0020100EB0109BAF1000FC4
:1001300006D101E00421F7E79049002081F827006B
:100140006C4602AA2146B068F8F7C9FE9DF908205E
:10015000F068211D10440122C01C1F28B8BF019265
:1001600008DB03AAF8F7BBFE9DF80C0010B101985C
:10017000401C0190DDE900100844801D20F07F4004
:100180000190A1EB090020F07F40009070798DF87C
:100190000A0000980390F8F70FFE0099019B091AD6
:1001A000181A774A21F07F4120F07F40B1F5800F87
:1001B00010D282420ED3714890F82950009CAB4671
:1001C000191B21F07F486FF07F41091BA0F1E80760
:1001D000049101E0002082E00C2D27D005EB850082
:1001E00007EB80026FF07F435068011BB1F5800F71
:1001F00010D3A4EB000CBCF5800F0BD38B4203D2C1
:1002000004990844411C05E063450DD2181A2044A6
:10021000401C4142002909DA5848AB46957C90F8C9
:1002200027000028D8D04EE00AF03DFC5D4523D0E1
:100230000BEB8B0007EB80036FF07F429968081B84
:10024000B0F5800F10D3A4EB010CBCF5800F0BD3DD
:10025000824203D204980844401C05E0624524D23F
:10026000521A1019401C4042002805DD9DF80A0072
:100270009A7B904228BF0C460C2D1CBF9DF80A109B
:100280003E4A17D005EB850007EB800043681B1B37
:1002900023F07F4343450DD2837B994228BF846876
:1002A000857C92F8270070B902E00AF0FCFBE3E7D6
:1002B0000C2DE7D10098A04205D004EB080020F0F7
:1002C0007F400094019000990398814206D001EB91
:1002D000090020F07F40F8F7F5FDB06001202749C4
:1002E00091F82710002904BF05B0BDE8F08FBAF1DE
:1002F000000F3FF421AF05B0BDE8F08F2DE9F04FBE
:10030000814687B00C461F4809F0FCF91E490127B9
:100310004FF0000801EB090500287DD0A1F5887891
:1003200098F81400002818BF0AF0BDFB20780128B7
:1003300000F02A8288F810902078022808BF0AF07E
:10034000B2FB124E207906F10C02307260797072A5
:100350003146A068F8F7C3FD96F90C000F2817E0A6
:100360003C0B0020FF7F841E0020A10700E05EF808
:100370000080841E00807BE104ED00E0240C00205E
:10038000FFFF3F00500C0020180C0020080B00203D
:1003900004DD1F3830733068401C306096F90C0063
:1003A000E168351D0844C01C1F28B8BF2F6009DB59
:1003B0006A462946F8F793FD9DF8000010B12868B9
:1003C000401C28602078B07288F81470FA4D95F8B7
:1003D000CD0195F8CC11884204BF07B0BDE8F08F7D
:1003E000F64890F829400C2C00F0D881F8F7E4FC8E
:1003F000F34904EB840201EB82010A7C042A19BF51
:100400000A7C032A07B0BDE8F08FEE4B4A68896882
:10041000121A22F07F4200E01CE0081A20F07F4010
:10042000062A3CBF07B0BDE8F08FB2F5800F24BFAD
:1004300007B0BDE8F08F83423CBF07B0BDE8F08F46
:1004400095F8CD0195F8CC11884240F0B08107B005
:10045000BDE8F08FD84E96F8CD01162856D096F804
:10046000CD0196F8CC11401C884201D10AF01BFB4B
:10047000207801284FD0D04890F8CD1101EB8101B0
:1004800000EB810080F81090207802284CD0CA48F8
:1004900090F8CD1101EB810100EB810520792872E4
:1004A0006079687205F10C022946A068F8F717FD1B
:1004B00095F90C000F2804DD1F3828732868401CAC
:1004C000286095F90C00E1682E1D0844C01C1F2807
:1004D000B8BF376009DB6A463146F8F700FD9DF882
:1004E000000010B13068401C30602078A872B2491A
:1004F00091F8CD0116280EBF002091F8CD01401CC7
:1005000081F8CD01B04809F013F95FE796F8CC0106
:100510000028ADD1AAE715F8010C002818BF0AF091
:10052000C2FA05F8017CA6E7A8480068C005C00D1E
:1005300010D0103840B20028B8BF00F00F0000F112
:10054000E020ACBF90F8000490F8140D400908BFFB
:100550000AF0A9FA984890F8CD1101AA01EB81019F
:1005600000EB8106E068CDF800808DF804806946D4
:10057000F8F7B5FC9DF904000F28CCBF012000203E
:100580000099351D084401900220B0722079307224
:1005900060797072A068C01C1F28B8BF2F6009DB8B
:1005A0006A462946F8F79BFC9DF8000010B12868C0
:1005B000401C2860307A062810D2DFE800F0030DD6
:1005C0000B09070500200CE0B4200AE0732008E0C6
:1005D000322006E00A2004E0062002E00AF063FA76
:1005E0000020217900290CBF042102210844029037
:1005F0007168801D08440199009001440298081A0E
:1006000005906E4C002084F82700F8F7D5FB804653
:1006100030600198404420F07F40F06094F8290059
:100620000C287DD0204690F8291001EB8102A0F122
:10063000E80101EB82025468009A2746224422F026
:100640007F42039296F809B090F82950121B22F0CD
:100650007F4A6FF07F42121BA94604920C2D28D0CE
:10066000574805EB850100EB81036FF07F42586826
:10067000011BB1F5800F24BFA4EB000CBCF5800F6B
:100680000BD38A4203D204990844411C05E0624519
:100690000DD2111A0819401C4142002909DA4748B5
:1006A000A9469D7C90F827000028D7D050E00AF09A
:1006B000FAF94D4523D0424809EB890100EB81014D
:1006C0006FF07F438868021B8146B2F5800F24BF1C
:1006D000A4EB000CBCF5800F0BD3934203D2049A19
:1006E0001044421C05E0634525D21A1A1019401C1B
:1006F0004242002A03DD887B834528BF4C460C2DEF
:100700001CBF2E4BA3F1E8011AD000BF05EB8500FA
:1007100001EB80025068001B20F07F40504500E054
:100720002AE00DD2907B834528BF9468957C93F88E
:10073000270068B902E00AF0B6F9E0E70C2DE5D130
:10074000A74205D004EB0A0020F07F402746039023
:10075000039AA7EB080121F07F41A2EB080205985C
:1007600022F07F42B1F5800F06D2904204D3029866
:10077000384420F07F403060104890F8270000286F
:100780007FF43FAFB3E600BF15F8010C002818BF97
:100790000AF089F905F8017CCCE500BF95F8CD0198
:1007A00095F8CC11884204BF07B0BDE8F08F07B0C0
:1007B000BDE8F04FF8F760BB38090020240C00209A
:1007C0003C0B0020FFFF3F00500C002004ED00E038
:1007D0000020F8F737BA0120F8F734BAFE4800785D
:1007E00070472DE9F0410546022821D0FB4C94F8D2
:1007F00029000C2808BF0AF056F9002784F8267053
:10080000012684F82B6094F829100320DFF8D083A8
:1008100001EB810108EB81010874F8F734FB6DB13D
:10082000012D2DD0032D73D00AF03DF9BDE8F081E4
:10083000E9480078BDE8F041F8F7F1BD207F0028D5
:1008400018BF0AF030F984F8256000202760F8F717
:100850000AFAA168B1F1FF3F04D001230022184633
:10086000F8F746FA94F8290094F82910401CC0B211
:1008700001EB810158F82120BDE8F041012110472A
:100880000120F8F7F0F994F8250000281CBFA068B3
:10089000B0F1FF3F0DD094F8290094F82910401CC6
:1008A000C0B201EB810158F82120BDE8F0410621DA
:1008B0001047207F012809D0022813D0032828D010
:1008C00004283BD00AF0EFF8BDE8F08194F824004A
:1008D00028B184F82470F8F7DDFA84F823602777CC
:1008E000BDE8F08194F8280018B9F8F745FB84F8C2
:1008F000286094F8290094F82910401CC0B201EB3C
:10090000810158F82120002190472777BDE8F08128
:1009100033E0217B60680123411A00221846F8F772
:10092000E7F994F8240028B184F82470F8F7B2FAB3
:1009300084F8236002202077BDE8F08194F820102D
:1009400060680123411A00221846F8F7D1F994F89B
:10095000280018B9F8F710FB84F8286094F82900EB
:1009600094F82910401CC0B201EB810158F82120F5
:10097000002190472677BDE8F08194F8290094F88B
:100980002910401CC0B201EB810158F82120BDE8BC
:10099000F0410521104710B5904C94F829000C281F
:1009A00008BF0AF080F894F8290094F82910401C38
:1009B000C0B28B4A01EB810152F82120BDE8104002
:1009C000042110472DE9F05FF8F7F6F9834C8146D2
:1009D0004FF00C0B94F829000026A4F1E8084FF022
:1009E000010A0C282CD094F82910204601EB810133
:1009F00008EB8101097C042922D090F8291001EB31
:100A0000810108EB8101097C032908BFBDE8F09F43
:100A1000744922696069A2EB090222F07F42A0EBCF
:100A2000090020F07F40062A38BFBDE8F09FB2F5EC
:100A3000800F28BFBDE8F09F814238BFBDE8F09F1E
:100A4000A068B0F1FF3F18BF0AF02DF884F82560C8
:100A500094F82900644F0C2806D194F8210018B1AD
:100A6000F8787870B87838705C4890F829000C28CD
:100A70001ED05A4890F8291001EB810108EB810142
:100A8000097C042914D190F829B090F8291001EBC1
:100A9000810108EB810181F810A090F8291001EB89
:100AA000810108EB8101897C80F8291080F82AA057
:100AB0004E4C94F8CD0194F8CC1104F2DF25884215
:100AC0004FD000BF94F8CC0100EB800004EB800015
:100AD000007C405D012894F8CC0100EB800004EB21
:100AE000800004D0007C405D022873D018E0807A3A
:100AF00001280DD094F8CC11022001EB810104EB08
:100B00008101097C485594F8CC01162820D01BE0BF
:100B100094F8CC0100EB800004EB8000007C46558B
:100B200094F8CC0100EB800004EB800294F8CC0137
:100B300000EB800004EB8000017C4846FEF791FF4B
:100B400094F8CC01162803D094F8CC01401C00E0A6
:100B5000002084F8CC0194F8CD0194F8CC1188429F
:100B6000B0D1234C207D70B1207C415D012968D03B
:100B7000405D02286DD0207D28B1217C1C4A48466A
:100B8000FEF76FFF2675BBF10C0F06D00BEB8B0049
:100B900008EB8000017C012964D0104C94F82900F6
:100BA0000C2800F03E8194F82A00002800F04881CB
:100BB00084F82A6094F8290000EB800008EB800399
:100BC000A4F53B70D3E90112DB68C0F80433C0E937
:100BD000BF120FE022E0000074000020240C00206F
:100BE0003C0B0020FFFF3F0076000020380900206A
:100BF000080B0020607E00280CBF0425022594F815
:100C00002900C34600EB800108EB8100407B0628E9
:100C100051D2DFE800F0444E4C4A484694F8CC01EB
:100C200000EB800004EB8000807A012818BF09F0F7
:100C30003AFF94F8CC0100EB800004EB8000867250
:100C400066E7A17A01291DBF022141552675465547
:100C500091E7A07A012818BF09F025FFA672207C31
:100C6000465588E707210174FE4C207E162812D0D5
:100C7000207EE17D401C884202D100BF09F013FFB5
:100C8000207E04F800B0207E16280EBF0020207EB3
:100C9000401C207681E7E07D0028F1D1EEE70020BE
:100CA0000CE0B4200AE0732008E0322006E00A20BD
:100CB00004E0062002E009F0F6FE00202073617EC9
:100CC000022918BF012911D121690144A1EB0902B0
:100CD00022F07F42382A09D903206076A1F1320040
:100CE00020F07F4020613220207309E0322807D2B3
:100CF00094F8280058B9F8F73FF984F828A006E0DE
:100D000094F8280018B1F8F760F984F82860797829
:100D100084F8201038780622012818BF032806D14D
:100D200084F824A0207B814284BF081A821D94F895
:100D30002230002B18BF921C94F82400002808BF12
:100D4000002B6AD0D4F810806069A8EB0908DFF89E
:100D500018C328F07F48A0EB090020F07F404245EF
:100D600098BFB8F5800F41D284453FD3207B88429D
:100D700015D22369A1EB0002A3EB020222F07F420D
:100D80001144294421F07F412261616000280CBF99
:100D900001200320207710F0FF0F36D115E00AD98B
:100DA000226900291044284420F07F4060600CBF75
:100DB00002200420EEE7002B08BF09F074FE206932
:100DC000284420F07F40606026770120F7F74BFF32
:100DD00094F82900012300EB80010BEB810061688E
:100DE00090F90C200020F7F783FF29E084F82460B5
:100DF00084F82260207B0028E1D02169084428443F
:100E000020F07F4060600220207720690123411993
:100E100000221846F7F76CFFDAE7207B0028ECD1B8
:100E2000CDE70120F7F71FFF0020F7F71CFFF7F7CA
:100E3000FFFE94F8280018B1F8F7C7F884F8286086
:100E400094F8220028B1F8F725F884F8236084F894
:100E5000226094F8210018B1F8787870B87838706A
:100E600094F8240030B184F823603878002808BF53
:100E700084F824607B48017EC07D814203D07B489A
:100E80004078F8F7CCFA84F827A0BDE8F09F70B559
:100E9000774C054682B094F829000C2808BF09F069
:100EA00002FE94F82900734E00EB800006EB8000F0
:100EB000007C032818BF09F0F6FDA068B0F1FF3FE1
:100EC00018BF09F0F0FD94F82900002100EB800024
:100ED00006EB800001AA90F90C0000918DF8041037
:100EE00028446946F7F7FBFF9DF904000F28CCBFA3
:100EF00001200020009908446168084420F07F41E7
:100F0000A16094F82500002804BF02B070BD012341
:100F100002B00022BDE870401846F7F7E9BE564A15
:100F20000B1A02F1010CB3EB9C0F3CBF1846704743
:100F300010B5441AB4EB9C0F3CBF184610BD9A4242
:100F400003D2101A0844401C10BDA24204D2511A08
:100F50000844401C404210BD09F0A5FD002010BD12
:100F60000123002201460220F7F7C2BE0220F7F754
:100F70007ABEF7F721BFF0B53D4C054683B094F833
:100F80002B00002808BF09F08EFD642D50D33B498B
:100F90000020491B80414BD3394890F8CD1190F87F
:100FA000CC01814244D13748007D002840D194F8DB
:100FB0002900304F00EB800007EB8006206801AA73
:100FC00028446946F7F78BFF9DF90400002802DDED
:100FD0000098401C0090B268009973685018C01ABD
:100FE00020F07F40B0F5800F22D2B07C0C2809D0D1
:100FF00000EB800007EB80004068801A20F07F4003
:10100000884215D3A068B0F1FF3F05D00120F7F763
:101010002AFE4FF0FF30A060206828442060B068AE
:101020000099084420F07F40606103B00120F0BDCA
:1010300003B00020F0BD2DE9F0410646401EC5B2C8
:101040000C4805EB850100EB8104207C002808BFDB
:1010500009F029FD0A4A92F8CC1192F8CD0181429B
:1010600020D011E0200B0020FFFF3F007400002083
:10107000240C00203C0B0020FF7F841EFF1FA107D3
:1010800038090020080B002001EB810302EB8303E9
:101090001B7CB3420DD016290CBF0021491CC9B2DC
:1010A0008142DED13948017D002961D0007CB04207
:1010B0005ED10020BDE8F081217C05291FBF217C85
:1010C0000629217C07292BD12774C27D0023017EAC
:1010D000914218BF014623D011F80280A84508BFED
:1010E000012300D04BB1162A0CBF4FF0000802F1CB
:1010F000010811F8088001F80280162A0CBF0022AE
:10110000521CD2B291F818809045E5D143B10A7EC5
:10111000002A08BF81F818C002D00A7E521E0A7643
:10112000617C21B36674C27D0021037E934224D08A
:10113000835CAB4208BF012100D029B1162A0CBF45
:101140000023531CC35C8354162A0CBF0022521C7C
:10115000D2B2037E9342EBD149B1027E0146002A0E
:1011600008BF81F818C008D00A7E521E0A7604E033
:101170000127074800264FF0160C217C012904BFE7
:10118000617C002998D10120BDE8F081080B002086
:10119000200B002070B520490A68BAB100231D4613
:1011A00001244A68521C4A60092A00D34D600E7916
:1011B00004FA06F20E6816420AD072B60B68934320
:1011C0000B6062B649680160002070BD052070BDEB
:1011D0005B1C092BE5D309F066FCF7E74FF0E02133
:1011E0004FF48000C1F800027047EFF3108111F056
:1011F000010F72B64FF0010202FA00F206480368CE
:1012000042EA0302026000D162B6E7E70248002129
:1012100001604160704700007C00002001208107D0
:1012200008607047012081074860704712480068D5
:10123000C00700D0012070470F48001F0068C0079A
:1012400000D0012070470C4808300068C00700D06B
:1012500001207047084810300068704706490C317B
:101260000A68D20306D5096801F00301814201D161
:1012700001207047002070470C040040CA4911F853
:10128000210F4978884201D3401A02E0C1F12101BF
:101290000844C0B27047C449233111F8210F49787E
:1012A000884201D3401A02E0C1F121010844C0B2D2
:1012B0007047BD49463111F8210F4978884201D362
:1012C000401A02E0C1F121010844C0B27047B74999
:1012D00010B5402081F80004B3490020233101F803
:1012E000210F4870B04901F8210F4870AE494631CE
:1012F00001F8210F4870AE4808F0FCF9AC48401CDA
:1013000008F0F8F9F7F7DCFFBDE8104000F040B94D
:1013100020207047B2E770B50C4605460026FFF75F
:10132000ADFF0146A048A14212D30022641EE4B2E0
:101330000DD390F82210435C491CC9B205F8013B5B
:1013400080F822102129F1D180F82220EEE7012631
:1013500000F01EF9304670BD202070479BE770B545
:101360000C4605460026FFF796FF01468E482330BF
:10137000A14212D30022641EE4B20DD390F82210D1
:10138000435C491CC9B205F8013B80F822102129B1
:10139000F1D180F82220EEE7012600F0F9F830467E
:1013A00070BD202101700020704710B50446FFF782
:1013B00080FF2070002010BD70B50C460546FFF779
:1013C00078FF014678484630A14213D30022641EBC
:1013D000E4B20DD390F82210435C491CC9B205F861
:1013E000013B80F822102129F1D180F82220EEE77C
:1013F000002401E042F2070400F0CAF8204670BD64
:1014000070B50C460546212901D909F04CFB694805
:101410000068103840B200F0A2F8C6B20D2000F00B
:101420009EF8C0B2864205D209F03DFB02E000BF43
:10143000F7F790FF21462846FFF76DFF0028F7D009
:1014400070BD2DE9F047DFF86881574CA8F101081D
:101450000746233498F80000DFF84C91002604F189
:10146000230A38B994F8221094F82100212200F0C0
:1014700085F890B14D4699F8221099F82100212263
:1014800000F07CF8B8B155469AF822109AF821007D
:10149000212200F073F848B335E094F82100275476
:1014A00094F82100401CC0B284F8210021282AD1E0
:1014B00084F8216027E095F821002F5495F8210049
:1014C000401CC0B285F82100212801D185F8216097
:1014D00098F800004746B0B195F8221095F8210021
:1014E000212200F04BF870B13E700CE095F821001D
:1014F0002F5495F82100401CC0B285F82100212806
:1015000001D185F8216094F8221094F8210021225D
:1015100000F034F8002820D099F8221099F8210022
:10152000212200F02BF8002817D09AF822109AF800
:101530002100212200F022F800280ED0F7F7E7FE64
:101540001B4808F0DFF8B0F5005F01D009F0ABFAF6
:10155000BDE8F047164808F0EBB8BDE8F087002872
:1015600006DA00F00F0000F1E02090F8140D03E01F
:1015700000F1E02090F8000440097047401C8842C8
:1015800004D0904200D109B100207047012070477B
:1015900010B5074808F0B6F8002803D1BDE81040A0
:1015A000F7F7A0BE10BD0000540C00200DE000E0D5
:1015B0008500002004ED00E00E4908784A78401CC0
:1015C000C0B2904200D0087070470A484FF0E02146
:1015D00020BF40BF20BF427803784370D1F800326B
:1015E0002BB9D1F8043213B903789342F0D000201C
:1015F00070470000870000202DE9F04101252803F5
:101600004FF0E0210026C1F880011E4CC4F80061B3
:101610000C2000F02CF81C4801680268C94341F313
:10162000001142F010020260C4F804532560491C06
:1016300000E020BFD4F80021002AFAD019B90168CF
:1016400021F010010160114807686560C4F8085373
:10165000C4F800610C2000F00AF83846BDE8F081BB
:1016600010B50446FFF7C8FF2060002010BD00F051
:101670001F02012191404009800000F1E020C0F8E4
:101680008012704700C0004010ED00E008C5004027
:101690002DE9F047FA4C0646FF21606800EB061280
:1016A00011702178FF2916D04FF0080909EB0111BC
:1016B00009EB06174158C059491E21F07F4100F03F
:1016C000E1F918B194F80080454614E0616820788B
:1016D00001EB061108702670BDE8F087626809EB1F
:1016E0000510D159105800F0CDF930B96068A846FE
:1016F00000EB08100578FF2DF0D1606800EB0611B3
:1017000000EB08100D700670E6E7F0B5DC4B044600
:10171000002001255A680C261B7A0BE005EB001708
:10172000D75DA74204D106EB0017D7598F4204D0EA
:10173000401CC0B28342F1D8FF20F0BD70B5FFF766
:1017400018FCCF4C014608252278606805EB021290
:10175000805800F097F9012808D92178606805EBD6
:1017600001114058BDE87040FFF7FABBFFF736F8AB
:10177000BDE87040F7F753BE2DE9F041C04C257825
:10178000FFF7F7FB0146FF2D6FD04FF008086268A6
:1017900008EB0516905900F075F90228606801D928
:1017A00080595EE000EB051109782170022101EB00
:1017B0000511425C5AB1521E4254815901F5000193
:1017C00021F07F4181512846FFF762FF34E0042376
:1017D000012203EB051302EB051250F803C0875CEE
:1017E000BCF1000F10D0BCF5806F10D9CCF309020A
:1017F00050F806C00CEB423C2CF07F4C40F806C081
:10180000C3589A1A920A09E0FF2181540AE08259CA
:1018100002EB4C3222F07F42825100224254284691
:10182000FFF736FF0C21606801EB05114158E068B5
:1018300050F82720384690472078FF2815D0FFF72A
:1018400098FB01462278606808EB021245468058F2
:1018500000F018F9012891D92178606805EB011191
:101860004058BDE8F041FFF77BBBBDE8F081F0B523
:101870001D4614460E460746FF2B01D309F013F907
:10188000A00701D009F00FF97D48FF210022C760B1
:10189000446005720674017042701046012204E033
:1018A00002EB0013401CE154C0B2A842F8D3F0BDD3
:1018B00070B5734C06466578207C854201D309F0EB
:1018C000F2F8E06840F825606078401C60702846B7
:1018D00070BD2DE9FF5F1D468B460746FF24FFF7CD
:1018E00048FBDFF89C91064699F80100B84201D800
:1018F00009F0D9F800214FF001084FF00C0A99F8CF
:101900000820D9F804000EE008EB0113C35CFF2B9C
:1019100027D0BB4205D10AEB011350F803C0DC45C8
:1019200021D0491CC9B28A42EED8FF2C1BD008EB4B
:1019300004110AEB0412475440F802B00421029B40
:101940000022012B01EB041111D042504FF48068AA
:1019500008234FF0020C454519D9A905890D08D077
:1019600008E00C46DDE7FF2004B0BDE8F09F4550DD
:10197000ECE7414606EB413203EB041322F07F42D1
:10198000C250691A0CEB0412890A81540BE005B9A4
:10199000012506EB453103EB041321F07F41C150D3
:1019A0000CEB0411425499F800502046FFF770FEEA
:1019B00099F80000A84201D0FFF7C0FE3846D3E7EF
:1019C00070B50C460546FFF7D4FA06462146284670
:1019D000FFF79BFE0446FF2817D0294D082101EB95
:1019E000041168684058314600F04CF800F580500A
:1019F000400B02216A6801EB0411515C09B100EB54
:101A00008120002800D1012070BD002070BD2DE98B
:101A1000F0410F468046FFF778FEFF281BD0184E96
:101A2000357871682A462C4605E0844206D0254662
:101A300001EB05131C78FF2CF7D10CE0FF2C0AD02A
:101A4000A5420CD101EB021000783070FF2804D0C1
:101A5000FFF774FE03E0002007E7FFF787FA394637
:101A60004046FFF7ADFFFF220123716803EB04132B
:101A7000CA5401EB041201EB051112780A70F4E666
:101A8000C00C0020401A20F07F40B0F5000F00D9B4
:101A9000002070470548064A0168914201D10021A3
:101AA0000160044901200860704700008C0000209C
:101AB000BEBAFECA40E501404048002101704170B5
:101AC00010218170704770B5054616460C460220FD
:101AD000F0F783FD3949012008703949F01E08608C
:101AE00038480560001F046070BD10B50220F0F793
:101AF00074FD32490120087033480021C0F80011FC
:101B0000C0F80411C0F8081130494FF40000086013
:101B100010BD2A480178C9B12D4A4FF40001116067
:101B20002949D1F800310022002B1CBFD1F8043123
:101B3000002B02D0D1F8081111B14270102103E03E
:101B40000121417023490968817002700020F0F77B
:101B500044BD1A480178002904BF407870471A48EC
:101B6000D0F80011002904BF02207047D0F80011FE
:101B700000291CBFD0F80411002905D0D0F80801B5
:101B8000002804BF01207047002070470B480178EF
:101B9000002904BF807870470B48D0F80011002955
:101BA0001CBFD0F80411002902D0D0F8080108B1F8
:101BB0001020704707480068C0B2704790000020AE
:101BC00010F5004008F5004000F0004004F5014029
:101BD00008F5014000F400403148002101704170D7
:101BE000704770B5064614460D460120F0F7F5FC27
:101BF0002B49012008702B480660001D0460001D61
:101C0000056070BD2DE9F04104460120F0F7E5FCC8
:101C100023490120087024490C60244D0026C5F892
:101C2000046123494FF040770F60A1F104084CB1E3
:101C3000012C18BF08F037FFC5F80062C8F8007023
:101C4000BDE8F081C5F800024FF08070C8F80000D0
:101C5000BDE8F0811248017879B1154A4FF0407122
:101C600011601249D1F804210021002A08BF4170F7
:101C700002D0104A1268427001700020F0F7ADBC2B
:101C800007480178002904BF407870470748D0F81A
:101C90000401002808BF704706480068C0B27047BA
:101CA0009300002008F5004004F5004000F00040DB
:101CB00008F5014000F4004070B5F94C00250126FC
:101CC0006570257025626572A572E67284F82950E8
:101CD000256304F13C00A56307F00CFD002818BF44
:101CE00008F0E1FE84F82450EE4808F0C1FFEE4809
:101CF000066070BD30B4EA490268DFF8B4C34A61D7
:101D000042688A61007A08770A7DE84BACF10404E6
:101D100001204AB10A7E00FA02F21A608D7D002D80
:101D20000CBF2260CCF800204A7D002A04BF30BCE2
:101D300070474A7E90401860C97D00290CBF206022
:101D4000CCF8000030BC7047DA4900B50A1D20B15C
:101D5000012806D008F0A7FE00BDD7480860D74884
:101D600002E0D7480860D748106000BDF0B50226F1
:101D70004FF0E02701240025C7F88061D2490D60AB
:101D80000C604A07D1490A60D208926DB2F1FF3F58
:101D90001ED1CF4B40F21B121A601B1DCD4A1A6098
:101DA000CE4BCD4A1A60CE4B42F28A021A60CD4A1F
:101DB0000A60CD4943F27D030A6822F47F4242F46F
:101DC000B0520A600A1F11686FF30F0119431160C6
:101DD000B8490A1DD8B101281DD008F064FE00BF23
:101DE000C24940F25B600860091F40F203100860BE
:101DF000081F0460BE4903200860BE4996200860A1
:101E0000A74890F9240010F0030F09D033E0AA4846
:101E10000860AA4802E0AA480860AA481060DFE704
:101E200080100A300C2826D2DFE800F02125252575
:101E3000251D1915110D0A06AF49042008601CE084
:101E4000AD48056019E0AC49FC20086015E0AA49DE
:101E5000F820086011E0A849F42008600DE0A649C8
:101E6000F020086009E0A449EC20086005E0A249E0
:101E7000D820086001E008F016FEA1499F480860DC
:101E8000A149A0480860091FA0480860C7F88062FF
:101E90009F491020C1F80403F0BD814A0368C2F8CD
:101EA00002308088D080117270477D4890F82900F8
:101EB00070477B4A517010707047F0B50D4604466C
:101EC00004EB4501908808841078D2F801100127AE
:101ED00040EA012044F8250005F1080007FA00F661
:101EE000002B04BF206BB04305D0012B18BF08F0B6
:101EF000DAFD206B304307FA05F108432063F0BD9B
:101F000030B50D460446082988BF08F0CCFD0022F4
:101F1000002D11D954F82210900000F1804000F5F6
:101F20008050C0F8001604EB4201098CC0F820165E
:101F3000501CC2B29542EDD8206B7649086030BD86
:101F400010B5044610F0030F2BD1A0100A300C2856
:101F500027D2DFE800F022262626261E1A16120EA9
:101F60000A066549042008601DE0634900200860F6
:101F700019E06149FC20086015E05F49F82008601D
:101F800011E05D49F42008600DE05B49F020086035
:101F900009E05949EC20086005E05749D82008605D
:101FA00001E008F080FD3E4880F8244010BD3C4828
:101FB00090F834007047584AC1781160006857495A
:101FC000000208607047252808BF02210ED026288D
:101FD00008BF1A210AD0272808BF502106D00A2896
:101FE00094BF0422062202EB4001C9B24C4A1160A0
:101FF0004C49086070472A490862704728498A7A24
:10200000012A4AD0022A18BF70474B7D002B08BF17
:102010007047DFF814C1012A40D0CA7D4B7E002AE8
:1020200018BF012210F17D00CCF80000DFF8FCC0E1
:102030000020CCF84C01180282F0010240EA025064
:1020400040F00312087F830003F1804303F5C0438F
:10205000C3F81025364A02EB8002887EC30003F1E4
:10206000804303F5F833C3F81425DFF8C8C0C3F87C
:1020700010C5C97ECB0003F1804303F5F833C3F8E4
:102080001425224AC3F81025012202FA00F002FAB0
:1020900001F108432849086070474FE053E0000011
:1020A000D40C0020E80C0020A005004018050050CA
:1020B0000C05005014150040060102002500030223
:1020C000050103001F000302FC1F004074170040BD
:1020D0008C150040700B103E206011009C150040D4
:1020E00034170040010300804017004038150040BD
:1020F00010150040441500400C150040004000043D
:1021000008F501404080004084F501401011004076
:102110000010004040160040241500401C150040EF
:1021200008150040541500404C85004000800040D8
:10213000006000404C81004004F501400B7D002B05
:102140007FF467AF70478A7D0B7E002A18BF01229B
:102150007E3069E72DE9F84F00280CBF01200220EE
:10216000FE4CFF4D0322A072C5F80022FE4FFD4A2F
:102170003A604FF0010839B1012922D0022939D043
:1021800008F091FCBDE8F88F012813D0C5F8048051
